Archive member included to satisfy reference by file (symbol)

../cmd/cmds.lib(alias.obj)    cmdtable.obj (cmd_alias)
../cmd/cmds.lib(beep.obj)     cmdtable.obj (cmd_beep)
../cmd/cmds.lib(break.obj)    cmdtable.obj (cmd_break)
../cmd/cmds.lib(call.obj)     cmdtable.obj (cmd_call)
../cmd/cmds.lib(cdd.obj)      cmdtable.obj (cmd_cdd)
../cmd/cmds.lib(chcp.obj)     cmdtable.obj (cmd_chcp)
../cmd/cmds.lib(chdir.obj)    cmdtable.obj (cmd_chdir)
../cmd/cmds.lib(cls.obj)      cmdtable.obj (cmd_cls)
../cmd/cmds.lib(copy.obj)     cmdtable.obj (cmd_copy)
../cmd/cmds.lib(ctty.obj)     cmdtable.obj (cmd_ctty)
../cmd/cmds.lib(date.obj)     cmdtable.obj (cmd_date)
../cmd/cmds.lib(del.obj)      cmdtable.obj (cmd_del)
../cmd/cmds.lib(dir.obj)      cmdtable.obj (cmd_dir)
../cmd/cmds.lib(dirs.obj)     cmdtable.obj (cmd_dirs)
../cmd/cmds.lib(doskey.obj)   cmdtable.obj (cmd_doskey)
../cmd/cmds.lib(echo.obj)     cmdtable.obj (cmd_echo)
../cmd/cmds.lib(exit.obj)     cmdtable.obj (internal_exit)
../cmd/cmds.lib(for.obj)      cmdtable.obj (cmd_for)
../cmd/cmds.lib(goto.obj)     cmdtable.obj (cmd_goto)
../cmd/cmds.lib(history.obj)  cmdtable.obj (cmd_history)
../cmd/cmds.lib(if.obj)       cmdtable.obj (cmd_if)
../cmd/cmds.lib(lfnfor.obj)   cmdtable.obj (cmd_lfnfor)
../cmd/cmds.lib(memory.obj)   cmdtable.obj (cmd_memory)
../cmd/cmds.lib(mkdir.obj)    cmdtable.obj (cmd_mkdir)
../cmd/cmds.lib(path.obj)     cmdtable.obj (cmd_path)
../cmd/cmds.lib(pause.obj)    cmdtable.obj (cmd_pause)
../cmd/cmds.lib(popd.obj)     cmdtable.obj (cmd_popd)
../cmd/cmds.lib(prompt.obj)   cmdtable.obj (cmd_prompt)
../cmd/cmds.lib(pushd.obj)    cmdtable.obj (cmd_pushd)
../cmd/cmds.lib(rem.obj)      cmdtable.obj (cmd_rem)
../cmd/cmds.lib(ren.obj)      cmdtable.obj (cmd_rename)
../cmd/cmds.lib(rmdir.obj)    cmdtable.obj (cmd_rmdir)
../cmd/cmds.lib(set.obj)      cmdtable.obj (cmd_set)
../cmd/cmds.lib(shift.obj)    cmdtable.obj (cmd_shift)
../cmd/cmds.lib(time.obj)     cmdtable.obj (cmd_time)
../cmd/cmds.lib(truename.obj)
                              cmdtable.obj (cmd_truename)
../cmd/cmds.lib(type.obj)     cmdtable.obj (cmd_type)
../cmd/cmds.lib(verify.obj)   cmdtable.obj (cmd_verify)
../cmd/cmds.lib(which.obj)    cmdtable.obj (cmd_which)
../lib/freecom.lib(absfile.obj)
                              batch.obj (abspath)
../lib/freecom.lib(app_get.obj)
                              ../cmd/cmds.lib(dir.obj) (appendDisable)
../lib/freecom.lib(app_set.obj)
                              ../cmd/cmds.lib(dir.obj) (appendRestore)
../lib/freecom.lib(beep_n.obj)
                              command.obj (beep)
../lib/freecom.lib(brk_get.obj)
                              ../cmd/cmds.lib(break.obj) (getbreak)
../lib/freecom.lib(brk_set.obj)
                              ../cmd/cmds.lib(break.obj) (setbreak)
../lib/freecom.lib(cbreak.obj)
                              ../cmd/cmds.lib(ctty.obj) (setCurrentConDev)
../lib/freecom.lib(cd_dir.obj)
                              ../cmd/cmds.lib(cdd.obj) (cd_dir)
../lib/freecom.lib(cgetch.obj)
                              command.obj (cgetchar)
../lib/freecom.lib(chgctxt.obj)
                              ../cmd/cmds.lib(alias.obj) (chgCtxt)
../lib/freecom.lib(chgdrv.obj)
                              command.obj (changeDrive)
../lib/freecom.lib(chgenv.obj)
                              command.obj (chgEnv)
../lib/freecom.lib(chgenvc.obj)
                              ../cmd/cmds.lib(set.obj) (chgEnvCase)
../lib/freecom.lib(chgenvr.obj)
                              ../cmd/cmds.lib(path.obj) (chgEnvRemove)
../lib/freecom.lib(cmdinput.obj)
                              command.obj (mywherex)
../lib/freecom.lib(critrchk.obj)
                              init.obj (registerCriterRepeatCheckAddr)
../lib/freecom.lib(ctxt.obj)  expalias.obj (ctxt)
../lib/freecom.lib(ctxt_clr.obj)
                              ../cmd/cmds.lib(popd.obj) (ctxtClear)
../lib/freecom.lib(ctxt_get.obj)
                              ../lib/freecom.lib(chgctxt.obj) (ctxtGet)
../lib/freecom.lib(ctxt_inf.obj)
                              ../cmd/cmds.lib(memory.obj) (ctxt_info)
../lib/freecom.lib(ctxt_mk.obj)
                              init.obj (ctxtCreate)
../lib/freecom.lib(ctxt_mkb.obj)
                              ../lib/freecom.lib(ctxt_mk.obj) (ctxtCreateMemBlock)
../lib/freecom.lib(ctxt_mkn.obj)
                              ../lib/freecom.lib(ctxt_get.obj) (ctxtMkItemName)
../lib/freecom.lib(ctxt_pop.obj)
                              ../cmd/cmds.lib(popd.obj) (ctxtPop)
../lib/freecom.lib(ctxt_psh.obj)
                              ../cmd/cmds.lib(pushd.obj) (ctxtPush)
../lib/freecom.lib(ctxt_rnu.obj)
                              ../lib/freecom.lib(ctxt_psh.obj) (ctxtRenumberItems)
../lib/freecom.lib(ctxt_set.obj)
                              ../lib/freecom.lib(ctxt_psh.obj) (ctxtSet)
../lib/freecom.lib(ctxt_vw.obj)
                              ../cmd/cmds.lib(dirs.obj) (ctxtView)
../lib/freecom.lib(curdatel.obj)
                              ../cmd/cmds.lib(date.obj) (curDateLong)
../lib/freecom.lib(curtime.obj)
                              ../cmd/cmds.lib(time.obj) (curTime)
../lib/freecom.lib(cwd.obj)   command.obj (cwd)
../lib/freecom.lib(dateget.obj)
                              ../lib/freecom.lib(curdatel.obj) (_dos_getdate)
../lib/freecom.lib(dateset.obj)
                              ../cmd/cmds.lib(date.obj) (_dos_setdate)
../lib/freecom.lib(devopen.obj)
                              command.obj (devopen)
../lib/freecom.lib(dfn_err.obj)
                              ../lib/freecom.lib(absfile.obj) (display_errno_fnam_error)
../lib/freecom.lib(dispcnt.obj)
                              ../cmd/cmds.lib(del.obj) (dispCount)
../lib/freecom.lib(drvnum.obj)
                              ../lib/freecom.lib(chgdrv.obj) (drvNum)
../lib/freecom.lib(exec.obj)  command.obj (exec)
../lib/freecom.lib(exec1.obj)
                              command.obj (setErrorLevel)
../lib/freecom.lib(farread.obj)
                              ../cmd/cmds.lib(copy.obj) (farread)
../lib/freecom.lib(filecomp.obj)
                              ../lib/freecom.lib(cmdinput.obj) (complete_filename)
../lib/freecom.lib(fdattr.obj)
                              command.obj (fdattr)
../lib/freecom.lib(fdsattr.obj)
                              ../cmd/cmds.lib(copy.obj) (fdsetattr)
../lib/freecom.lib(fillcomp.obj)
                              ../cmd/cmds.lib(copy.obj) (fillFnam)
../lib/freecom.lib(find.obj)  command.obj (skip_word)
../lib/freecom.lib(freep.obj)
                              batch.obj (freep)
../lib/freecom.lib(gallstr.obj)
                              loadhigh.obj (dosGetAllocStrategy)
../lib/freecom.lib(get1mcb.obj)
                              loadhigh.obj (GetFirstMCB)
../lib/freecom.lib(getenv.obj)
                              command.obj (getEnv)
../lib/freecom.lib(goxy.obj)  ../cmd/cmds.lib(cls.obj) (goxy)
../lib/freecom.lib(grabfcom.obj)
                              init.obj (grabComFilename)
../lib/freecom.lib(gumblink.obj)
                              loadhigh.obj (dosGetUMBLinkState)
../lib/freecom.lib(hdlrctxt.obj)
                              ../cmd/cmds.lib(alias.obj) (breakVarAssign)
../lib/freecom.lib(hist_get.obj)
                              ../lib/freecom.lib(cmdinput.obj) (histGet)
../lib/freecom.lib(hist_set.obj)
                              ../lib/freecom.lib(cmdinput.obj) (histSet)
../lib/freecom.lib(is_empty.obj)
                              ../cmd/cmds.lib(set.obj) (is_empty)
../lib/freecom.lib(is_fnamc.obj)
                              command.obj (is_fnchar)
../lib/freecom.lib(is_fnstr.obj)
                              ../cmd/cmds.lib(alias.obj) (is_fnstr)
../lib/freecom.lib(is_pchr.obj)
                              expalias.obj (is_pathdelim)
../lib/freecom.lib(isadev.obj)
                              ../cmd/cmds.lib(copy.obj) (isadev)
../lib/freecom.lib(lastdget.obj)
                              ../lib/freecom.lib(cd_dir.obj) (lastDirGet)
../lib/freecom.lib(lastdset.obj)
                              ../lib/freecom.lib(cd_dir.obj) (lastDirSet)
../lib/freecom.lib(leadopt.obj)
                              init.obj (leadOptions)
../lib/freecom.lib(lfnfuncs.obj)
                              command.obj (getshortfilename)
../lib/freecom.lib(lowexec.obj)
                              ../lib/freecom.lib(exec.obj) (lowLevelExec)
../lib/freecom.lib(ltrimcl.obj)
                              batch.obj (ltrimcl)
../lib/freecom.lib(match.obj)
                              command.obj (match_)
../lib/freecom.lib(messages.obj)
                              command.obj (unloadMsgs)
../lib/freecom.lib(mk_rddir.obj)
                              ../cmd/cmds.lib(mkdir.obj) (mk_rd_dir)
../lib/freecom.lib(msg_dps.obj)
                              command.obj (displayString)
../lib/freecom.lib(msg_fstr.obj)
                              ../cmd/cmds.lib(copy.obj) (getString)
../lib/freecom.lib(msg_gpt.obj)
                              ../lib/freecom.lib(cbreak.obj) (getPromptString)
../lib/freecom.lib(msg_mkey.obj)
                              ../lib/freecom.lib(cbreak.obj) (mapMetakey)
../lib/freecom.lib(msg_prmp.obj)
                              command.obj (userprompt)
../lib/freecom.lib(mux_ae.obj)
                              command.obj (runExtension)
../lib/freecom.lib(myperror.obj)
                              ../cmd/cmds.lib(del.obj) (myperror)
../lib/freecom.lib(nls.obj)   ../cmd/cmds.lib(date.obj) (refreshNLS)
../lib/freecom.lib(nls_date.obj)
                              ../cmd/cmds.lib(dir.obj) (nls_makedate)
../lib/freecom.lib(nls_time.obj)
                              ../cmd/cmds.lib(dir.obj) (nls_maketime)
../lib/freecom.lib(num_fmt.obj)
                              ../cmd/cmds.lib(dir.obj) (convert)
../lib/freecom.lib(onoff.obj)
                              ../cmd/cmds.lib(break.obj) (onoffStr)
../lib/freecom.lib(openf.obj)
                              ../cmd/cmds.lib(copy.obj) (isDeviceName)
../lib/freecom.lib(optsb.obj)
                              init.obj (optScanBool_)
../lib/freecom.lib(optsi.obj)
                              init.obj (optScanInteger_)
../lib/freecom.lib(optss.obj)
                              init.obj (optScanString_)
../lib/freecom.lib(pr_date.obj)
                              ../cmd/cmds.lib(date.obj) (parsedate)
../lib/freecom.lib(pr_prmpt.obj)
                              command.obj (printprompt)
../lib/freecom.lib(pr_time.obj)
                              ../cmd/cmds.lib(time.obj) (parsetime)
../lib/freecom.lib(prf.obj)   ../lib/freecom.lib(cbreak.obj) (vsprintf)
../lib/freecom.lib(prprompt.obj)
                              ../lib/freecom.lib(pr_prmpt.obj) (displayPrompt)
../lib/freecom.lib(readcmd.obj)
                              ../cmd/cmds.lib(ctty.obj) (set_readcommandType)
../lib/freecom.lib(realnum.obj)
                              ../lib/freecom.lib(hist_get.obj) (realNum)
../lib/freecom.lib(res.obj)   ../lib/freecom.lib(messages.obj) (enumResources)
../lib/freecom.lib(res_r.obj)
                              ../lib/freecom.lib(res.obj) (enumFileResources)
../lib/freecom.lib(res_vald.obj)
                              ../lib/freecom.lib(grabfcom.obj) (validResFile)
../lib/freecom.lib(resfile.obj)
                              ../lib/freecom.lib(res.obj) (comResFile)
../lib/freecom.lib(rmtmpfil.obj)
                              command.obj (killtmpfn)
../lib/freecom.lib(rtrimcl.obj)
                              ../cmd/cmds.lib(dir.obj) (rtrimcl)
../lib/freecom.lib(rtrimsp.obj)
                              ../cmd/cmds.lib(alias.obj) (rtrimsp)
../lib/freecom.lib(salloc.obj)
                              loadhigh.obj (dosSetAllocStrategy)
../lib/freecom.lib(samefile.obj)
                              ../cmd/cmds.lib(copy.obj) (samefile)
../lib/freecom.lib(scancmd.obj)
                              ver.obj (scanCmdline)
../lib/freecom.lib(scanopt.obj)
                              ../lib/freecom.lib(leadopt.obj) (scanOption)
../lib/freecom.lib(session.obj)
                              ../lib/freecom.lib(exec.obj) (saveSession)
../lib/freecom.lib(showcmds.obj)
                              cmdtable.obj (showcmds)
../lib/freecom.lib(skqwd.obj)
                              ../cmd/cmds.lib(if.obj) (skipqword)
../lib/freecom.lib(spfnam.obj)
                              ../cmd/cmds.lib(for.obj) (skipfnam)
../lib/freecom.lib(split.obj)
                              ../lib/freecom.lib(scancmd.obj) (split)
../lib/freecom.lib(sumblink.obj)
                              loadhigh.obj (dosSetUMBLinkState)
../lib/freecom.lib(timeget.obj)
                              ../lib/freecom.lib(curtime.obj) (_dos_gettime)
../lib/freecom.lib(timeset.obj)
                              ../cmd/cmds.lib(time.obj) (_dos_settime)
../lib/freecom.lib(tmpnam.obj)
                              command.obj (tmpfn)
../lib/freecom.lib(trimsp.obj)
                              ../cmd/cmds.lib(alias.obj) (trimsp)
../lib/freecom.lib(truepath.obj)
                              ../cmd/cmds.lib(truename.obj) (truepath)
../lib/freecom.lib(truncate.obj)
                              ../cmd/cmds.lib(copy.obj) (truncate)
../lib/freecom.lib(txtlend.obj)
                              batch.obj (textlineEnd)
../lib/freecom.lib(unquote.obj)
                              command.obj (unquote)
../lib/freecom.lib(vcgetch.obj)
                              ../lib/freecom.lib(msg_prmp.obj) (vcgetchar)
../lib/freecom.lib(where.obj)
                              command.obj (find_which)
../lib/freecom.lib(delay.obj)
                              command.obj (delay)
../lib/freecom.lib(err2.obj)  init.obj (error_invalid_lswitch)
../lib/freecom.lib(err3.obj)  init.obj (error_too_many_parameters)
../lib/freecom.lib(err5.obj)  loadhigh.obj (error_file_not_found)
../lib/freecom.lib(err6.obj)  init.obj (error_sfile_not_found)
../lib/freecom.lib(err7.obj)  ../cmd/cmds.lib(del.obj) (error_req_param_missing)
../lib/freecom.lib(err8.obj)  command.obj (error_bad_command)
../lib/freecom.lib(err10.obj)
                              batch.obj (error_out_of_memory)
../lib/freecom.lib(err11.obj)
                              command.obj (error_syntax)
../lib/freecom.lib(err13.obj)
                              ../cmd/cmds.lib(copy.obj) (error_selfcopy)
../lib/freecom.lib(err14.obj)
                              batch.obj (error_long_batchline)
../lib/freecom.lib(err15.obj)
                              batch.obj (error_bfile_vanished)
../lib/freecom.lib(err16.obj)
                              batch.obj (error_bfile_no_such_label)
../lib/freecom.lib(err17.obj)
                              ../cmd/cmds.lib(time.obj) (error_invalid_time)
../lib/freecom.lib(err18.obj)
                              ../lib/freecom.lib(chgenv.obj) (error_env_var)
../lib/freecom.lib(err19.obj)
                              ../cmd/cmds.lib(set.obj) (error_env_var_not_found)
../lib/freecom.lib(err20.obj)
                              ../cmd/cmds.lib(del.obj) (error_filename_too_long)
../lib/freecom.lib(err21.obj)
                              expalias.obj (error_command_too_long)
../lib/freecom.lib(err22.obj)
                              command.obj (error_line_too_long)
../lib/freecom.lib(err23.obj)
                              ../lib/freecom.lib(tmpnam.obj) (error_tempfile)
../lib/freecom.lib(err25.obj)
                              ../cmd/cmds.lib(dir.obj) (error_illformed_option)
../lib/freecom.lib(err26.obj)
                              ../lib/freecom.lib(optsb.obj) (error_opt_arg)
../lib/freecom.lib(err27.obj)
                              ../lib/freecom.lib(optsi.obj) (error_opt_noarg)
../lib/freecom.lib(err28.obj)
                              ../cmd/cmds.lib(copy.obj) (error_leading_plus)
../lib/freecom.lib(err29.obj)
                              ../cmd/cmds.lib(copy.obj) (error_trailing_plus)
../lib/freecom.lib(err30.obj)
                              ../cmd/cmds.lib(copy.obj) (error_open_file)
../lib/freecom.lib(err31.obj)
                              ../cmd/cmds.lib(copy.obj) (error_read_file)
../lib/freecom.lib(err32.obj)
                              ../cmd/cmds.lib(copy.obj) (error_write_file)
../lib/freecom.lib(err33.obj)
                              ../cmd/cmds.lib(copy.obj) (error_write_file_disc_full)
../lib/freecom.lib(err34.obj)
                              ../cmd/cmds.lib(copy.obj) (error_copy)
../lib/freecom.lib(err35.obj)
                              ../cmd/cmds.lib(copy.obj) (error_nothing_to_do)
../lib/freecom.lib(err36.obj)
                              ../lib/freecom.lib(optsi.obj) (error_invalid_number)
../lib/freecom.lib(err37.obj)
                              ../lib/freecom.lib(grabfcom.obj) (error_init_fully_qualified)
../lib/freecom.lib(err38.obj)
                              init.obj (error_corrupt_command_line)
../lib/freecom.lib(err39.obj)
                              init.obj (error_quoted_c_k)
../lib/freecom.lib(err41.obj)
                              init.obj (error_l_notimplemented)
../lib/freecom.lib(err42.obj)
                              init.obj (error_u_notimplemented)
../lib/freecom.lib(err45.obj)
                              ../cmd/cmds.lib(ctty.obj) (error_no_rw_device)
../lib/freecom.lib(err46.obj)
                              ../cmd/cmds.lib(ctty.obj) (error_ctty_dup)
../lib/freecom.lib(err47.obj)
                              ../lib/freecom.lib(cwd.obj) (error_no_cwd)
../lib/freecom.lib(err50.obj)
                              ../cmd/cmds.lib(if.obj) (error_if_exist)
../lib/freecom.lib(err51.obj)
                              ../cmd/cmds.lib(if.obj) (error_if_errorlevel)
../lib/freecom.lib(err53.obj)
                              ../cmd/cmds.lib(if.obj) (error_if_command)
../lib/freecom.lib(err54.obj)
                              ../lib/freecom.lib(chgctxt.obj) (error_alias_out_of_memory)
../lib/freecom.lib(err58.obj)
                              ../lib/freecom.lib(cd_dir.obj) (error_dirfct_failed)
../lib/freecom.lib(err59.obj)
                              ../cmd/cmds.lib(alias.obj) (error_no_alias_name)
../lib/freecom.lib(err60.obj)
                              ../cmd/cmds.lib(history.obj) (error_history_size)
../lib/freecom.lib(err61.obj)
                              ../lib/freecom.lib(chgctxt.obj) (error_context_out_of_memory)
../lib/freecom.lib(err63.obj)
                              ../cmd/cmds.lib(dir.obj) (error_out_of_dos_memory)
../lib/freecom.lib(err64.obj)
                              ../lib/freecom.lib(ctxt_mk.obj) (error_context_length)
../lib/freecom.lib(err65.obj)
                              ../lib/freecom.lib(ctxt_mk.obj) (error_context_add_status)
../lib/freecom.lib(err67.obj)
                              command.obj (error_redirect_from_file)
../lib/freecom.lib(err68.obj)
                              command.obj (error_redirect_to_file)
../lib/freecom.lib(err69.obj)
                              loadhigh.obj (error_bad_mcb_chain)
../lib/freecom.lib(err70.obj)
                              loadhigh.obj (error_unknown)
../lib/freecom.lib(err71.obj)
                              ../cmd/cmds.lib(copy.obj) (error_invalid_drive)
../lib/freecom.lib(err72.obj)
                              ../lib/freecom.lib(chgenv.obj) (error_no_env)
../lib/freecom.lib(err73.obj)
                              ../cmd/cmds.lib(break.obj) (error_on_off)
../lib/freecom.lib(err74.obj)
                              ../cmd/cmds.lib(date.obj) (error_invalid_date)
../lib/freecom.lib(err75.obj)
                              ../cmd/cmds.lib(for.obj) (error_for_bad_var)
../lib/freecom.lib(err76.obj)
                              ../cmd/cmds.lib(for.obj) (error_for_in)
../lib/freecom.lib(err77.obj)
                              ../cmd/cmds.lib(for.obj) (error_for_parens)
../lib/freecom.lib(err78.obj)
                              ../cmd/cmds.lib(for.obj) (error_for_do)
../lib/freecom.lib(err79.obj)
                              ../cmd/cmds.lib(for.obj) (error_for_no_command)
../lib/freecom.lib(err80.obj)
                              ../cmd/cmds.lib(goto.obj) (error_goto_label)
../lib/freecom.lib(err81.obj)
                              ../cmd/cmds.lib(chcp.obj) (error_get_codepage)
../lib/freecom.lib(err82.obj)
                              ../cmd/cmds.lib(chcp.obj) (error_set_codepage)
../lib/freecom.lib(err83.obj)
                              ../cmd/cmds.lib(copy.obj) (error_copy_plus_destination)
../lib/freecom.lib(err84.obj)
                              ../cmd/cmds.lib(copy.obj) (error_invalid_parameter)
../lib/freecom.lib(err85.obj)
                              ../lib/freecom.lib(grabfcom.obj) (error_fcom_is_device)
../lib/freecom.lib(err86.obj)
                              ../lib/freecom.lib(grabfcom.obj) (error_fcom_invalid)
../lib/freecom.lib(err87.obj)
                              ../lib/freecom.lib(exec1.obj) (error_exe_corrupt)
../lib/freecom.lib(almemblk.obj)
                              ../lib/freecom.lib(messages.obj) (allocMemBlk)
../lib/freecom.lib(beep_l.obj)
                              ../lib/freecom.lib(filecomp.obj) (beep_low)
../lib/freecom.lib(cbs.obj)   ../lib/freecom.lib(mk_rddir.obj) (cutBackslash)
../lib/freecom.lib(comfile.obj)
                              ../lib/freecom.lib(resfile.obj) (comFile)
../lib/freecom.lib(ctxt_as.obj)
                              ../lib/freecom.lib(ctxt_mk.obj) (ctxtAddStatus)
../lib/freecom.lib(dispexit.obj)
                              ../lib/freecom.lib(exec1.obj) (displayExitcode)
../lib/freecom.lib(inputdos.obj)
                              ../lib/freecom.lib(readcmd.obj) (readcommandDOS)
../lib/freecom.lib(ltrimsp.obj)
                              ../lib/freecom.lib(nls_time.obj) (ltrimsp)
../lib/freecom.lib(mktmpfil.obj)
                              ../lib/freecom.lib(tmpnam.obj) (mktempfile)
../lib/freecom.lib(msg_dflt.obj)
                              ../lib/freecom.lib(msg_fstr.obj) (defaultMessage)
../lib/freecom.lib(msg_get.obj)
                              ../lib/freecom.lib(dispexit.obj) (getMessage)
../lib/freecom.lib(parsenum.obj)
                              ../lib/freecom.lib(pr_date.obj) (parsenum)
../strings/strings.lib(str0011.obj)
                              ../lib/freecom.lib(messages.obj) (TEXT_ERROR_OUT_OF_MEMORY)
../strings/strings.lib(str0018.obj)
                              ../lib/freecom.lib(msg_dflt.obj) (TEXT_ERROR_SET_ENV_VAR)
../strings/strings.lib(str003c.obj)
                              ../lib/freecom.lib(msg_dflt.obj) (TEXT_ERROR_OPEN_FILE)
../strings/strings.lib(str00b1.obj)
                              command.obj (TEXT_MSG_REBOOT_NOW)
../strings/strings.lib(str00b2.obj)
                              init.obj (TEXT_MSG_FREECOM_NOT_FOUND)
../strings/strings.lib(str00f4.obj)
                              ../lib/freecom.lib(msg_dflt.obj) (TEXT_ERROR_FCOM_INVALID)
../strings/strings.lib(str00f5.obj)
                              ../lib/freecom.lib(messages.obj) (TEXT_ERROR_LOADING_STRINGS)
../strings/strings.lib(str00f6.obj)
                              init.obj (TEXT_TERMINATING)
../suppl/suppl_s.lib(byte2par.obj)
                              ../lib/freecom.lib(almemblk.obj) (BLK_byte2para)
../suppl/suppl_s.lib(cntry.obj)
                              ../lib/freecom.lib(nls.obj) (nlsNewInfo)
../suppl/suppl_s.lib(dfnfnam.obj)
                              batch.obj (dfnfilename)
../suppl/suppl_s.lib(dfnfullp.obj)
                              ../lib/freecom.lib(absfile.obj) (dfnfullpath)
../suppl/suppl_s.lib(dfnmerge.obj)
                              ../cmd/cmds.lib(copy.obj) (dfnmerge)
../suppl/suppl_s.lib(dfnpath.obj)
                              ../lib/freecom.lib(cwd.obj) (dfnpath)
../suppl/suppl_s.lib(dfnstat.obj)
                              init.obj (dfnstat)
../suppl/suppl_s.lib(dfntruen.obj)
                              ../lib/freecom.lib(truepath.obj) (dfntruename)
../suppl/suppl_s.lib(dosalloc.obj)
                              cswapc.obj (DOSalloc)
../suppl/suppl_s.lib(dosfree.obj)
                              cswapc.obj (DOSfree)
../suppl/suppl_s.lib(dossize.obj)
                              loadhigh.obj (DOSresize)
../suppl/suppl_s.lib(dstrfupr.obj)
                              expalias.obj (StrFUpr)
../suppl/suppl_s.lib(dstrtrim.obj)
                              ../suppl/suppl_s.lib(dfnfullp.obj) (StrTrim)
../suppl/suppl_s.lib(dstrupr.obj)
                              ../cmd/cmds.lib(set.obj) (StrUpr)
../suppl/suppl_s.lib(enoallc.obj)
                              ../suppl/suppl_s.lib(dfnmerge.obj) (eno_malloc)
../suppl/suppl_s.lib(enoreal.obj)
                              ../suppl/suppl_s.lib(dstrtrim.obj) (eno_realloc)
../suppl/suppl_s.lib(enosetos.obj)
                              ../suppl/suppl_s.lib(dfnstat.obj) (eno_setOSerror)
../suppl/suppl_s.lib(env_chg.obj)
                              ../lib/freecom.lib(chgctxt.obj) (env_change)
../suppl/suppl_s.lib(env_dvar.obj)
                              ../lib/freecom.lib(getenv.obj) (dupvar)
../suppl/suppl_s.lib(env_find.obj)
                              expalias.obj (env_findVar)
../suppl/suppl_s.lib(env_fora.obj)
                              ../lib/freecom.lib(ctxt_clr.obj) (env_forAll)
../suppl/suppl_s.lib(env_free.obj)
                              init.obj (env_freeCount)
../suppl/suppl_s.lib(env_insv.obj)
                              ../suppl/suppl_s.lib(env_chg.obj) (env_appVar)
../suppl/suppl_s.lib(env_len.obj)
                              ../lib/freecom.lib(chgctxt.obj) (env_varlen)
../suppl/suppl_s.lib(env_mtch.obj)
                              init.obj (env_matchVar)
../suppl/suppl_s.lib(env_new.obj)
                              ../lib/freecom.lib(ctxt_mkb.obj) (env_create)
../suppl/suppl_s.lib(env_nost.obj)
                              command.obj (env_nullStrings)
../suppl/suppl_s.lib(env_ovrw.obj)
                              ../suppl/suppl_s.lib(env_chg.obj) (env_ovrVarOffset)
../suppl/suppl_s.lib(env_repl.obj)
                              init.obj (env_replace)
../suppl/suppl_s.lib(env_rlsg.obj)
                              ../suppl/suppl_s.lib(env_repl.obj) (env_relocateSegment)
../suppl/suppl_s.lib(env_scnt.obj)
                              ../suppl/suppl_s.lib(env_free.obj) (env_strcounter)
../suppl/suppl_s.lib(env_size.obj)
                              init.obj (env_setsize)
../suppl/suppl_s.lib(env_strg.obj)
                              init.obj (env_string)
../suppl/suppl_s.lib(env_sub.obj)
                              ../lib/freecom.lib(ctxt_clr.obj) (env_subVarOffset)
../suppl/suppl_s.lib(env_var1.obj)
                              init.obj (env_resizeCtrl)
../suppl/suppl_s.lib(env_var2.obj)
                              init.obj (suppl_dfltEnvSegm)
../suppl/suppl_s.lib(fstrdup.obj)
                              init.obj (_fdupstr)
../suppl/suppl_s.lib(mcb_is.obj)
                              init.obj (isMCB)
../suppl/suppl_s.lib(mcb_leng.obj)
                              ../cmd/cmds.lib(memory.obj) (mcb_length)
../suppl/suppl_s.lib(mcb_nxt.obj)
                              loadhigh.obj (nxtMCB)
../suppl/suppl_s.lib(mcb_walk.obj)
                              ../suppl/suppl_s.lib(mcb_is.obj) (mcb_walk)
../suppl/suppl_s.lib(toupperx.obj)
                              ../suppl/suppl_s.lib(dstrfupr.obj) (toFUpper)
../suppl/suppl_s.lib(filefind.obj)
                              batch.obj (findfirst)
../suppl/suppl_s.lib(invokedo.obj)
                              ../suppl/suppl_s.lib(filefind.obj) (invokeDOS)
../suppl/suppl_s.lib(intr.obj)
                              cswapc.obj (_intrf)
../suppl/suppl_s.lib(addu.obj)
                              ../suppl/suppl_s.lib(env_repl.obj) (addu)
../suppl/suppl_s.lib(dfndeli2.obj)
                              ../suppl/suppl_s.lib(dfnfnam.obj) (dfndelim2)
../suppl/suppl_s.lib(dfndelim.obj)
                              ../suppl/suppl_s.lib(dfnmerge.obj) (dfndelim)
../suppl/suppl_s.lib(dfnexpan.obj)
                              ../suppl/suppl_s.lib(dfnfullp.obj) (dfnexpand)
../suppl/suppl_s.lib(dfnsplit.obj)
                              ../suppl/suppl_s.lib(dfnexpan.obj) (dfnsplit)
../suppl/suppl_s.lib(dfnsquee.obj)
                              ../suppl/suppl_s.lib(dfnexpan.obj) (dfnsqueeze)
../suppl/suppl_s.lib(dmemcmpf.obj)
                              ../suppl/suppl_s.lib(env_mtch.obj) (_fMemiCmp)
../suppl/suppl_s.lib(dstrchar.obj)
                              ../suppl/suppl_s.lib(dfnexpan.obj) (StrChar)
../suppl/suppl_s.lib(dstrleft.obj)
                              ../suppl/suppl_s.lib(dfnsplit.obj) (StrLeft)
../suppl/suppl_s.lib(dstrrepl.obj)
                              ../suppl/suppl_s.lib(dfnexpan.obj) (StrRepl_)
../suppl/suppl_s.lib(enosdup.obj)
                              ../suppl/suppl_s.lib(dfnsplit.obj) (eno_strdup)
../suppl/suppl_s.lib(env_del.obj)
                              ../suppl/suppl_s.lib(env_repl.obj) (env_delete)
../suppl/suppl_s.lib(mcb_1st.obj)
                              ../suppl/suppl_s.lib(mcb_walk.obj) (mcb_first)
/home/evln/proj/build-ia16.202501/prefix/bin/../lib/gcc/ia16-elf/6.3.0/../../../../ia16-elf/lib/regparmcall/libi86.a(fmemchr.o)
                              ../cmd/cmds.lib(copy.obj) (_fmemchr)
/home/evln/proj/build-ia16.202501/prefix/bin/../lib/gcc/ia16-elf/6.3.0/../../../../ia16-elf/lib/regparmcall/libi86.a(fmemcmp.o)
                              loadhigh.obj (_fmemcmp)
/home/evln/proj/build-ia16.202501/prefix/bin/../lib/gcc/ia16-elf/6.3.0/../../../../ia16-elf/lib/regparmcall/libi86.a(fmemcpy.o)
                              init.obj (_fmemcpy)
/home/evln/proj/build-ia16.202501/prefix/bin/../lib/gcc/ia16-elf/6.3.0/../../../../ia16-elf/lib/regparmcall/libi86.a(fmemmove.o)
                              ../suppl/suppl_s.lib(env_insv.obj) (_fmemmove)
/home/evln/proj/build-ia16.202501/prefix/bin/../lib/gcc/ia16-elf/6.3.0/../../../../ia16-elf/lib/regparmcall/libi86.a(fstrcpy.o)
                              expalias.obj (_fstrcpy)
/home/evln/proj/build-ia16.202501/prefix/bin/../lib/gcc/ia16-elf/6.3.0/../../../../ia16-elf/lib/regparmcall/libi86.a(fstrlen.o)
                              expalias.obj (_fstrlen)
/home/evln/proj/build-ia16.202501/prefix/bin/../lib/gcc/ia16-elf/6.3.0/../../../../ia16-elf/lib/regparmcall/libi86.a(libi86-fmemmove-backward.o)
                              /home/evln/proj/build-ia16.202501/prefix/bin/../lib/gcc/ia16-elf/6.3.0/../../../../ia16-elf/lib/regparmcall/libi86.a(fmemmove.o) (__libi86_fmemmove_backward)
/home/evln/proj/build-ia16.202501/prefix/bin/../lib/gcc/ia16-elf/6.3.0/../../../../ia16-elf/lib/regparmcall/libi86.a(getdcwd.o)
                              ../suppl/suppl_s.lib(dfnpath.obj) (_getdcwd)
/home/evln/proj/build-ia16.202501/prefix/bin/../lib/gcc/ia16-elf/6.3.0/../../../../ia16-elf/lib/regparmcall/libi86.a(getdrive.o)
                              /home/evln/proj/build-ia16.202501/prefix/bin/../lib/gcc/ia16-elf/6.3.0/../../../../ia16-elf/lib/regparmcall/libi86.a(getdcwd.o) (_getdrive)
/home/evln/proj/build-ia16.202501/prefix/bin/../lib/gcc/ia16-elf/6.3.0/../../../../ia16-elf/lib/regparmcall/libc.a(lib_a-atexit.o)
                              init.obj (atexit)
/home/evln/proj/build-ia16.202501/prefix/bin/../lib/gcc/ia16-elf/6.3.0/../../../../ia16-elf/lib/regparmcall/libc.a(lib_a-atol.o)
                              ../cmd/cmds.lib(history.obj) (atol)
/home/evln/proj/build-ia16.202501/prefix/bin/../lib/gcc/ia16-elf/6.3.0/../../../../ia16-elf/lib/regparmcall/libc.a(lib_a-ctype_.o)
                              batch.obj (__ctype_ptr__)
/home/evln/proj/build-ia16.202501/prefix/bin/../lib/gcc/ia16-elf/6.3.0/../../../../ia16-elf/lib/regparmcall/libc.a(lib_a-errno.o)
                              command.obj (__errno)
/home/evln/proj/build-ia16.202501/prefix/bin/../lib/gcc/ia16-elf/6.3.0/../../../../ia16-elf/lib/regparmcall/libc.a(lib_a-exit.o)
                              /home/evln/proj/build-ia16.202501/prefix/bin/../lib/gcc/ia16-elf/6.3.0/../../../../ia16-elf/lib/regparmcall/dos-s-c0.o (exit)
/home/evln/proj/build-ia16.202501/prefix/bin/../lib/gcc/ia16-elf/6.3.0/../../../../ia16-elf/lib/regparmcall/libc.a(lib_a-impure.o)
                              /home/evln/proj/build-ia16.202501/prefix/bin/../lib/gcc/ia16-elf/6.3.0/../../../../ia16-elf/lib/regparmcall/libc.a(lib_a-exit.o) (_global_impure_ptr)
/home/evln/proj/build-ia16.202501/prefix/bin/../lib/gcc/ia16-elf/6.3.0/../../../../ia16-elf/lib/regparmcall/libc.a(lib_a-malloc.o)
                              batch.obj (malloc)
/home/evln/proj/build-ia16.202501/prefix/bin/../lib/gcc/ia16-elf/6.3.0/../../../../ia16-elf/lib/regparmcall/libc.a(lib_a-memchr.o)
                              batch.obj (memchr)
/home/evln/proj/build-ia16.202501/prefix/bin/../lib/gcc/ia16-elf/6.3.0/../../../../ia16-elf/lib/regparmcall/libc.a(lib_a-memcmp.o)
                              batch.obj (memcmp)
/home/evln/proj/build-ia16.202501/prefix/bin/../lib/gcc/ia16-elf/6.3.0/../../../../ia16-elf/lib/regparmcall/libc.a(lib_a-memcpy.o)
                              loadhigh.obj (memcpy)
/home/evln/proj/build-ia16.202501/prefix/bin/../lib/gcc/ia16-elf/6.3.0/../../../../ia16-elf/lib/regparmcall/libc.a(lib_a-memmove.o)
                              batch.obj (memmove)
/home/evln/proj/build-ia16.202501/prefix/bin/../lib/gcc/ia16-elf/6.3.0/../../../../ia16-elf/lib/regparmcall/libc.a(lib_a-memset.o)
                              batch.obj (memset)
/home/evln/proj/build-ia16.202501/prefix/bin/../lib/gcc/ia16-elf/6.3.0/../../../../ia16-elf/lib/regparmcall/libc.a(lib_a-nano-freer.o)
                              /home/evln/proj/build-ia16.202501/prefix/bin/../lib/gcc/ia16-elf/6.3.0/../../../../ia16-elf/lib/regparmcall/libc.a(lib_a-malloc.o) (_free_r)
/home/evln/proj/build-ia16.202501/prefix/bin/../lib/gcc/ia16-elf/6.3.0/../../../../ia16-elf/lib/regparmcall/libc.a(lib_a-nano-mallocr.o)
                              /home/evln/proj/build-ia16.202501/prefix/bin/../lib/gcc/ia16-elf/6.3.0/../../../../ia16-elf/lib/regparmcall/libc.a(lib_a-malloc.o) (_malloc_r)
/home/evln/proj/build-ia16.202501/prefix/bin/../lib/gcc/ia16-elf/6.3.0/../../../../ia16-elf/lib/regparmcall/libc.a(lib_a-qsort.o)
                              ../cmd/cmds.lib(dir.obj) (qsort)
/home/evln/proj/build-ia16.202501/prefix/bin/../lib/gcc/ia16-elf/6.3.0/../../../../ia16-elf/lib/regparmcall/libc.a(lib_a-realloc.o)
                              expalias.obj (realloc)
/home/evln/proj/build-ia16.202501/prefix/bin/../lib/gcc/ia16-elf/6.3.0/../../../../ia16-elf/lib/regparmcall/libc.a(lib_a-remove.o)
                              ../lib/freecom.lib(rmtmpfil.obj) (remove)
/home/evln/proj/build-ia16.202501/prefix/bin/../lib/gcc/ia16-elf/6.3.0/../../../../ia16-elf/lib/regparmcall/libc.a(lib_a-setjmp.o)
                              command.obj (setjmp)
/home/evln/proj/build-ia16.202501/prefix/bin/../lib/gcc/ia16-elf/6.3.0/../../../../ia16-elf/lib/regparmcall/libc.a(lib_a-stpcpy.o)
                              batch.obj (stpcpy)
/home/evln/proj/build-ia16.202501/prefix/bin/../lib/gcc/ia16-elf/6.3.0/../../../../ia16-elf/lib/regparmcall/libc.a(lib_a-strcasecmp.o)
                              batch.obj (strcasecmp)
/home/evln/proj/build-ia16.202501/prefix/bin/../lib/gcc/ia16-elf/6.3.0/../../../../ia16-elf/lib/regparmcall/libc.a(lib_a-strcat.o)
                              expalias.obj (strcat)
/home/evln/proj/build-ia16.202501/prefix/bin/../lib/gcc/ia16-elf/6.3.0/../../../../ia16-elf/lib/regparmcall/libc.a(lib_a-strchr.o)
                              command.obj (strchr)
/home/evln/proj/build-ia16.202501/prefix/bin/../lib/gcc/ia16-elf/6.3.0/../../../../ia16-elf/lib/regparmcall/libc.a(lib_a-strcmp.o)
                              command.obj (strcmp)
/home/evln/proj/build-ia16.202501/prefix/bin/../lib/gcc/ia16-elf/6.3.0/../../../../ia16-elf/lib/regparmcall/libc.a(lib_a-strcpy.o)
                              command.obj (strcpy)
/home/evln/proj/build-ia16.202501/prefix/bin/../lib/gcc/ia16-elf/6.3.0/../../../../ia16-elf/lib/regparmcall/libc.a(lib_a-strdup.o)
                              batch.obj (strdup)
/home/evln/proj/build-ia16.202501/prefix/bin/../lib/gcc/ia16-elf/6.3.0/../../../../ia16-elf/lib/regparmcall/libc.a(lib_a-strdup_r.o)
                              /home/evln/proj/build-ia16.202501/prefix/bin/../lib/gcc/ia16-elf/6.3.0/../../../../ia16-elf/lib/regparmcall/libc.a(lib_a-strdup.o) (_strdup_r)
/home/evln/proj/build-ia16.202501/prefix/bin/../lib/gcc/ia16-elf/6.3.0/../../../../ia16-elf/lib/regparmcall/libc.a(lib_a-strlen.o)
                              batch.obj (strlen)
/home/evln/proj/build-ia16.202501/prefix/bin/../lib/gcc/ia16-elf/6.3.0/../../../../ia16-elf/lib/regparmcall/libc.a(lib_a-strlwr.o)
                              ../cmd/cmds.lib(dir.obj) (strlwr)
/home/evln/proj/build-ia16.202501/prefix/bin/../lib/gcc/ia16-elf/6.3.0/../../../../ia16-elf/lib/regparmcall/libc.a(lib_a-strncasecmp.o)
                              ../cmd/cmds.lib(if.obj) (strncasecmp)
/home/evln/proj/build-ia16.202501/prefix/bin/../lib/gcc/ia16-elf/6.3.0/../../../../ia16-elf/lib/regparmcall/libc.a(lib_a-strncpy.o)
                              ../lib/freecom.lib(hist_get.obj) (strncpy)
/home/evln/proj/build-ia16.202501/prefix/bin/../lib/gcc/ia16-elf/6.3.0/../../../../ia16-elf/lib/regparmcall/libc.a(lib_a-strpbrk.o)
                              batch.obj (strpbrk)
/home/evln/proj/build-ia16.202501/prefix/bin/../lib/gcc/ia16-elf/6.3.0/../../../../ia16-elf/lib/regparmcall/libc.a(lib_a-strrchr.o)
                              command.obj (strrchr)
/home/evln/proj/build-ia16.202501/prefix/bin/../lib/gcc/ia16-elf/6.3.0/../../../../ia16-elf/lib/regparmcall/libc.a(lib_a-strspn.o)
                              ../suppl/suppl_s.lib(dfnfullp.obj) (strspn)
/home/evln/proj/build-ia16.202501/prefix/bin/../lib/gcc/ia16-elf/6.3.0/../../../../ia16-elf/lib/regparmcall/libc.a(lib_a-strtok.o)
                              ../cmd/cmds.lib(copy.obj) (strtok)
/home/evln/proj/build-ia16.202501/prefix/bin/../lib/gcc/ia16-elf/6.3.0/../../../../ia16-elf/lib/regparmcall/libc.a(lib_a-strtok_r.o)
                              /home/evln/proj/build-ia16.202501/prefix/bin/../lib/gcc/ia16-elf/6.3.0/../../../../ia16-elf/lib/regparmcall/libc.a(lib_a-strtok.o) (__strtok_r)
/home/evln/proj/build-ia16.202501/prefix/bin/../lib/gcc/ia16-elf/6.3.0/../../../../ia16-elf/lib/regparmcall/libc.a(lib_a-strtol.o)
                              /home/evln/proj/build-ia16.202501/prefix/bin/../lib/gcc/ia16-elf/6.3.0/../../../../ia16-elf/lib/regparmcall/libc.a(lib_a-atol.o) (_strtol_r)
/home/evln/proj/build-ia16.202501/prefix/bin/../lib/gcc/ia16-elf/6.3.0/../../../../ia16-elf/lib/regparmcall/libc.a(lib_a-sysisatty.o)
                              ../cmd/cmds.lib(copy.obj) (isatty)
/home/evln/proj/build-ia16.202501/prefix/bin/../lib/gcc/ia16-elf/6.3.0/../../../../ia16-elf/lib/regparmcall/libc.a(lib_a-syslseek.o)
                              batch.obj (lseek)
/home/evln/proj/build-ia16.202501/prefix/bin/../lib/gcc/ia16-elf/6.3.0/../../../../ia16-elf/lib/regparmcall/libc.a(lib_a-sysunlink.o)
                              ../cmd/cmds.lib(copy.obj) (unlink)
/home/evln/proj/build-ia16.202501/prefix/bin/../lib/gcc/ia16-elf/6.3.0/../../../../ia16-elf/lib/regparmcall/libc.a(lib_a-syswrite.o)
                              /home/evln/proj/build-ia16.202501/prefix/bin/../lib/gcc/ia16-elf/6.3.0/../../../../ia16-elf/lib/regparmcall/libc.a(lib_a-nano-freer.o) (write)
/home/evln/proj/build-ia16.202501/prefix/bin/../lib/gcc/ia16-elf/6.3.0/../../../../ia16-elf/lib/regparmcall/libc.a(lib_a-toupper.o)
                              ../suppl/suppl_s.lib(toupperx.obj) (toupper)
/home/evln/proj/build-ia16.202501/prefix/bin/../lib/gcc/ia16-elf/6.3.0/../../../../ia16-elf/lib/regparmcall/libc.a(lib_a-__atexit.o)
                              /home/evln/proj/build-ia16.202501/prefix/bin/../lib/gcc/ia16-elf/6.3.0/../../../../ia16-elf/lib/regparmcall/libc.a(lib_a-atexit.o) (__register_exitproc)
/home/evln/proj/build-ia16.202501/prefix/bin/../lib/gcc/ia16-elf/6.3.0/../../../../ia16-elf/lib/regparmcall/libc.a(lib_a-__call_atexit.o)
                              /home/evln/proj/build-ia16.202501/prefix/bin/../lib/gcc/ia16-elf/6.3.0/../../../../ia16-elf/lib/regparmcall/libc.a(lib_a-exit.o) (__call_exitprocs)
/home/evln/proj/build-ia16.202501/prefix/bin/../lib/gcc/ia16-elf/6.3.0/../../../../ia16-elf/lib/regparmcall/libc.a(lib_a-nano-reallocr.o)
                              /home/evln/proj/build-ia16.202501/prefix/bin/../lib/gcc/ia16-elf/6.3.0/../../../../ia16-elf/lib/regparmcall/libc.a(lib_a-realloc.o) (_realloc_r)
/home/evln/proj/build-ia16.202501/prefix/bin/../lib/gcc/ia16-elf/6.3.0/../../../../ia16-elf/lib/regparmcall/libc.a(lib_a-nano-msizer.o)
                              /home/evln/proj/build-ia16.202501/prefix/bin/../lib/gcc/ia16-elf/6.3.0/../../../../ia16-elf/lib/regparmcall/libc.a(lib_a-nano-reallocr.o) (_malloc_usable_size_r)
/home/evln/proj/build-ia16.202501/prefix/bin/../lib/gcc/ia16-elf/6.3.0/regparmcall/libgcc.a(udivsi3.o)
                              ../cmd/cmds.lib(dir.obj) (__udivsi3)
/home/evln/proj/build-ia16.202501/prefix/bin/../lib/gcc/ia16-elf/6.3.0/regparmcall/libgcc.a(umodsi3.o)
                              ../cmd/cmds.lib(dir.obj) (__umodsi3)
/home/evln/proj/build-ia16.202501/prefix/bin/../lib/gcc/ia16-elf/6.3.0/regparmcall/libgcc.a(ia16-ldivmodu.o)
                              /home/evln/proj/build-ia16.202501/prefix/bin/../lib/gcc/ia16-elf/6.3.0/regparmcall/libgcc.a(udivsi3.o) (__ia16_ldivmodu)
/home/evln/proj/build-ia16.202501/prefix/bin/../lib/gcc/ia16-elf/6.3.0/../../../../ia16-elf/lib/regparmcall/libdos-s.a(dos-isattyr.o)
                              /home/evln/proj/build-ia16.202501/prefix/bin/../lib/gcc/ia16-elf/6.3.0/../../../../ia16-elf/lib/regparmcall/libc.a(lib_a-sysisatty.o) (_isatty_r)
/home/evln/proj/build-ia16.202501/prefix/bin/../lib/gcc/ia16-elf/6.3.0/../../../../ia16-elf/lib/regparmcall/libdos-s.a(dos-lseekr.o)
                              /home/evln/proj/build-ia16.202501/prefix/bin/../lib/gcc/ia16-elf/6.3.0/../../../../ia16-elf/lib/regparmcall/libc.a(lib_a-syslseek.o) (_lseek_r)
/home/evln/proj/build-ia16.202501/prefix/bin/../lib/gcc/ia16-elf/6.3.0/../../../../ia16-elf/lib/regparmcall/libdos-s.a(dos-sbrkr.o)
                              /home/evln/proj/build-ia16.202501/prefix/bin/../lib/gcc/ia16-elf/6.3.0/../../../../ia16-elf/lib/regparmcall/libc.a(lib_a-nano-mallocr.o) (_sbrk_r)
/home/evln/proj/build-ia16.202501/prefix/bin/../lib/gcc/ia16-elf/6.3.0/../../../../ia16-elf/lib/regparmcall/libdos-s.a(dos-unlinkr.o)
                              /home/evln/proj/build-ia16.202501/prefix/bin/../lib/gcc/ia16-elf/6.3.0/../../../../ia16-elf/lib/regparmcall/libc.a(lib_a-remove.o) (_unlink_r)
/home/evln/proj/build-ia16.202501/prefix/bin/../lib/gcc/ia16-elf/6.3.0/../../../../ia16-elf/lib/regparmcall/libdos-s.a(dos-writer.o)
                              /home/evln/proj/build-ia16.202501/prefix/bin/../lib/gcc/ia16-elf/6.3.0/../../../../ia16-elf/lib/regparmcall/libc.a(lib_a-syswrite.o) (_write_r)
/home/evln/proj/build-ia16.202501/prefix/bin/../lib/gcc/ia16-elf/6.3.0/../../../../ia16-elf/lib/regparmcall/libdos-s.a(dos-msmmabort.o)
                              /home/evln/proj/build-ia16.202501/prefix/bin/../lib/gcc/ia16-elf/6.3.0/../../../../ia16-elf/lib/regparmcall/libc.a(lib_a-nano-freer.o) (abort)
/home/evln/proj/build-ia16.202501/prefix/bin/../lib/gcc/ia16-elf/6.3.0/../../../../ia16-elf/lib/regparmcall/libdos-s.a(dos-heaplen.o)
                              /home/evln/proj/build-ia16.202501/prefix/bin/../lib/gcc/ia16-elf/6.3.0/../../../../ia16-elf/lib/regparmcall/libdos-s.a(dos-sbrkr.o) (_heaplen)
/home/evln/proj/build-ia16.202501/prefix/bin/../lib/gcc/ia16-elf/6.3.0/../../../../ia16-elf/lib/regparmcall/libdos-s.a(dos-near-data-segment.o)
                              /home/evln/proj/build-ia16.202501/prefix/bin/../lib/gcc/ia16-elf/6.3.0/../../../../ia16-elf/lib/regparmcall/libdos-s.a(dos-msmmabort.o) (__ia16_near_data_segment)
/home/evln/proj/build-ia16.202501/prefix/bin/../lib/gcc/ia16-elf/6.3.0/../../../../ia16-elf/lib/regparmcall/libc.a(lib_a-abort.o)
                              /home/evln/proj/build-ia16.202501/prefix/bin/../lib/gcc/ia16-elf/6.3.0/../../../../ia16-elf/lib/regparmcall/libdos-s.a(dos-msmmabort.o) (__ia16_abort_impl)

Allocating common symbols
Common symbol       size              file

ComPath             0x2               init.obj
exitReason          0x2               ../lib/freecom.lib(dispexit.obj)
jmp_beginning       0x14              command.obj

Discarded input sections

 .comment       0x0000000000000000       0x12 cswapc.obj
 .comment       0x0000000000000000       0x12 batch.obj
 .comment       0x0000000000000000       0x12 cmdtable.obj
 .comment       0x0000000000000000       0x12 command.obj
 .comment       0x0000000000000000       0x12 expalias.obj
 .comment       0x0000000000000000       0x12 init.obj
 .comment       0x0000000000000000       0x12 kswap.obj
 .comment       0x0000000000000000       0x12 loadhigh.obj
 .comment       0x0000000000000000       0x12 module.obj
 .comment       0x0000000000000000       0x12 redir.obj
 .comment       0x0000000000000000       0x12 ver.obj
 .comment       0x0000000000000000       0x12 ../cmd/cmds.lib(alias.obj)
 .comment       0x0000000000000000       0x12 ../cmd/cmds.lib(beep.obj)
 .comment       0x0000000000000000       0x12 ../cmd/cmds.lib(break.obj)
 .comment       0x0000000000000000       0x12 ../cmd/cmds.lib(call.obj)
 .comment       0x0000000000000000       0x12 ../cmd/cmds.lib(cdd.obj)
 .comment       0x0000000000000000       0x12 ../cmd/cmds.lib(chcp.obj)
 .comment       0x0000000000000000       0x12 ../cmd/cmds.lib(chdir.obj)
 .comment       0x0000000000000000       0x12 ../cmd/cmds.lib(cls.obj)
 .comment       0x0000000000000000       0x12 ../cmd/cmds.lib(copy.obj)
 .comment       0x0000000000000000       0x12 ../cmd/cmds.lib(ctty.obj)
 .comment       0x0000000000000000       0x12 ../cmd/cmds.lib(date.obj)
 .comment       0x0000000000000000       0x12 ../cmd/cmds.lib(del.obj)
 .comment       0x0000000000000000       0x12 ../cmd/cmds.lib(dir.obj)
 .comment       0x0000000000000000       0x12 ../cmd/cmds.lib(dirs.obj)
 .comment       0x0000000000000000       0x12 ../cmd/cmds.lib(doskey.obj)
 .comment       0x0000000000000000       0x12 ../cmd/cmds.lib(echo.obj)
 .comment       0x0000000000000000       0x12 ../cmd/cmds.lib(exit.obj)
 .comment       0x0000000000000000       0x12 ../cmd/cmds.lib(for.obj)
 .comment       0x0000000000000000       0x12 ../cmd/cmds.lib(goto.obj)
 .comment       0x0000000000000000       0x12 ../cmd/cmds.lib(history.obj)
 .comment       0x0000000000000000       0x12 ../cmd/cmds.lib(if.obj)
 .comment       0x0000000000000000       0x12 ../cmd/cmds.lib(lfnfor.obj)
 .comment       0x0000000000000000       0x12 ../cmd/cmds.lib(memory.obj)
 .comment       0x0000000000000000       0x12 ../cmd/cmds.lib(mkdir.obj)
 .comment       0x0000000000000000       0x12 ../cmd/cmds.lib(path.obj)
 .comment       0x0000000000000000       0x12 ../cmd/cmds.lib(pause.obj)
 .comment       0x0000000000000000       0x12 ../cmd/cmds.lib(popd.obj)
 .comment       0x0000000000000000       0x12 ../cmd/cmds.lib(prompt.obj)
 .comment       0x0000000000000000       0x12 ../cmd/cmds.lib(pushd.obj)
 .comment       0x0000000000000000       0x12 ../cmd/cmds.lib(rem.obj)
 .comment       0x0000000000000000       0x12 ../cmd/cmds.lib(ren.obj)
 .comment       0x0000000000000000       0x12 ../cmd/cmds.lib(rmdir.obj)
 .comment       0x0000000000000000       0x12 ../cmd/cmds.lib(set.obj)
 .comment       0x0000000000000000       0x12 ../cmd/cmds.lib(shift.obj)
 .comment       0x0000000000000000       0x12 ../cmd/cmds.lib(time.obj)
 .comment       0x0000000000000000       0x12 ../cmd/cmds.lib(truename.obj)
 .comment       0x0000000000000000       0x12 ../cmd/cmds.lib(type.obj)
 .comment       0x0000000000000000       0x12 ../cmd/cmds.lib(verify.obj)
 .comment       0x0000000000000000       0x12 ../cmd/cmds.lib(which.obj)
 .comment       0x0000000000000000       0x12 ../lib/freecom.lib(absfile.obj)
 .comment       0x0000000000000000       0x12 ../lib/freecom.lib(app_get.obj)
 .comment       0x0000000000000000       0x12 ../lib/freecom.lib(app_set.obj)
 .comment       0x0000000000000000       0x12 ../lib/freecom.lib(beep_n.obj)
 .comment       0x0000000000000000       0x12 ../lib/freecom.lib(brk_get.obj)
 .comment       0x0000000000000000       0x12 ../lib/freecom.lib(brk_set.obj)
 .comment       0x0000000000000000       0x12 ../lib/freecom.lib(cbreak.obj)
 .comment       0x0000000000000000       0x12 ../lib/freecom.lib(cd_dir.obj)
 .comment       0x0000000000000000       0x12 ../lib/freecom.lib(cgetch.obj)
 .comment       0x0000000000000000       0x12 ../lib/freecom.lib(chgctxt.obj)
 .comment       0x0000000000000000       0x12 ../lib/freecom.lib(chgdrv.obj)
 .comment       0x0000000000000000       0x12 ../lib/freecom.lib(chgenv.obj)
 .comment       0x0000000000000000       0x12 ../lib/freecom.lib(chgenvc.obj)
 .comment       0x0000000000000000       0x12 ../lib/freecom.lib(chgenvr.obj)
 .comment       0x0000000000000000       0x12 ../lib/freecom.lib(cmdinput.obj)
 .comment       0x0000000000000000       0x12 ../lib/freecom.lib(critrchk.obj)
 .comment       0x0000000000000000       0x12 ../lib/freecom.lib(ctxt.obj)
 .comment       0x0000000000000000       0x12 ../lib/freecom.lib(ctxt_clr.obj)
 .comment       0x0000000000000000       0x12 ../lib/freecom.lib(ctxt_get.obj)
 .comment       0x0000000000000000       0x12 ../lib/freecom.lib(ctxt_inf.obj)
 .comment       0x0000000000000000       0x12 ../lib/freecom.lib(ctxt_mk.obj)
 .comment       0x0000000000000000       0x12 ../lib/freecom.lib(ctxt_mkb.obj)
 .comment       0x0000000000000000       0x12 ../lib/freecom.lib(ctxt_mkn.obj)
 .comment       0x0000000000000000       0x12 ../lib/freecom.lib(ctxt_pop.obj)
 .comment       0x0000000000000000       0x12 ../lib/freecom.lib(ctxt_psh.obj)
 .comment       0x0000000000000000       0x12 ../lib/freecom.lib(ctxt_rnu.obj)
 .comment       0x0000000000000000       0x12 ../lib/freecom.lib(ctxt_set.obj)
 .comment       0x0000000000000000       0x12 ../lib/freecom.lib(ctxt_vw.obj)
 .comment       0x0000000000000000       0x12 ../lib/freecom.lib(curdatel.obj)
 .comment       0x0000000000000000       0x12 ../lib/freecom.lib(curtime.obj)
 .comment       0x0000000000000000       0x12 ../lib/freecom.lib(cwd.obj)
 .comment       0x0000000000000000       0x12 ../lib/freecom.lib(dateget.obj)
 .comment       0x0000000000000000       0x12 ../lib/freecom.lib(dateset.obj)
 .comment       0x0000000000000000       0x12 ../lib/freecom.lib(devopen.obj)
 .comment       0x0000000000000000       0x12 ../lib/freecom.lib(dfn_err.obj)
 .comment       0x0000000000000000       0x12 ../lib/freecom.lib(dispcnt.obj)
 .comment       0x0000000000000000       0x12 ../lib/freecom.lib(drvnum.obj)
 .comment       0x0000000000000000       0x12 ../lib/freecom.lib(exec.obj)
 .comment       0x0000000000000000       0x12 ../lib/freecom.lib(exec1.obj)
 .comment       0x0000000000000000       0x12 ../lib/freecom.lib(farread.obj)
 .comment       0x0000000000000000       0x12 ../lib/freecom.lib(filecomp.obj)
 .comment       0x0000000000000000       0x12 ../lib/freecom.lib(fdattr.obj)
 .comment       0x0000000000000000       0x12 ../lib/freecom.lib(fdsattr.obj)
 .comment       0x0000000000000000       0x12 ../lib/freecom.lib(fillcomp.obj)
 .comment       0x0000000000000000       0x12 ../lib/freecom.lib(find.obj)
 .comment       0x0000000000000000       0x12 ../lib/freecom.lib(freep.obj)
 .comment       0x0000000000000000       0x12 ../lib/freecom.lib(gallstr.obj)
 .comment       0x0000000000000000       0x12 ../lib/freecom.lib(get1mcb.obj)
 .comment       0x0000000000000000       0x12 ../lib/freecom.lib(getenv.obj)
 .comment       0x0000000000000000       0x12 ../lib/freecom.lib(goxy.obj)
 .comment       0x0000000000000000       0x12 ../lib/freecom.lib(grabfcom.obj)
 .comment       0x0000000000000000       0x12 ../lib/freecom.lib(gumblink.obj)
 .comment       0x0000000000000000       0x12 ../lib/freecom.lib(hdlrctxt.obj)
 .comment       0x0000000000000000       0x12 ../lib/freecom.lib(hist_get.obj)
 .comment       0x0000000000000000       0x12 ../lib/freecom.lib(hist_set.obj)
 .comment       0x0000000000000000       0x12 ../lib/freecom.lib(is_empty.obj)
 .comment       0x0000000000000000       0x12 ../lib/freecom.lib(is_fnamc.obj)
 .comment       0x0000000000000000       0x12 ../lib/freecom.lib(is_fnstr.obj)
 .comment       0x0000000000000000       0x12 ../lib/freecom.lib(is_pchr.obj)
 .comment       0x0000000000000000       0x12 ../lib/freecom.lib(isadev.obj)
 .comment       0x0000000000000000       0x12 ../lib/freecom.lib(lastdget.obj)
 .comment       0x0000000000000000       0x12 ../lib/freecom.lib(lastdset.obj)
 .comment       0x0000000000000000       0x12 ../lib/freecom.lib(leadopt.obj)
 .comment       0x0000000000000000       0x12 ../lib/freecom.lib(lfnfuncs.obj)
 .comment       0x0000000000000000       0x12 ../lib/freecom.lib(ltrimcl.obj)
 .comment       0x0000000000000000       0x12 ../lib/freecom.lib(match.obj)
 .comment       0x0000000000000000       0x12 ../lib/freecom.lib(messages.obj)
 .comment       0x0000000000000000       0x12 ../lib/freecom.lib(mk_rddir.obj)
 .comment       0x0000000000000000       0x12 ../lib/freecom.lib(msg_dps.obj)
 .comment       0x0000000000000000       0x12 ../lib/freecom.lib(msg_fstr.obj)
 .comment       0x0000000000000000       0x12 ../lib/freecom.lib(msg_gpt.obj)
 .comment       0x0000000000000000       0x12 ../lib/freecom.lib(msg_mkey.obj)
 .comment       0x0000000000000000       0x12 ../lib/freecom.lib(msg_prmp.obj)
 .comment       0x0000000000000000       0x12 ../lib/freecom.lib(mux_ae.obj)
 .comment       0x0000000000000000       0x12 ../lib/freecom.lib(myperror.obj)
 .comment       0x0000000000000000       0x12 ../lib/freecom.lib(nls.obj)
 .comment       0x0000000000000000       0x12 ../lib/freecom.lib(nls_date.obj)
 .comment       0x0000000000000000       0x12 ../lib/freecom.lib(nls_time.obj)
 .comment       0x0000000000000000       0x12 ../lib/freecom.lib(num_fmt.obj)
 .comment       0x0000000000000000       0x12 ../lib/freecom.lib(onoff.obj)
 .comment       0x0000000000000000       0x12 ../lib/freecom.lib(openf.obj)
 .comment       0x0000000000000000       0x12 ../lib/freecom.lib(optsb.obj)
 .comment       0x0000000000000000       0x12 ../lib/freecom.lib(optsi.obj)
 .comment       0x0000000000000000       0x12 ../lib/freecom.lib(optss.obj)
 .comment       0x0000000000000000       0x12 ../lib/freecom.lib(pr_date.obj)
 .comment       0x0000000000000000       0x12 ../lib/freecom.lib(pr_prmpt.obj)
 .comment       0x0000000000000000       0x12 ../lib/freecom.lib(pr_time.obj)
 .comment       0x0000000000000000       0x12 ../lib/freecom.lib(prf.obj)
 .comment       0x0000000000000000       0x12 ../lib/freecom.lib(prprompt.obj)
 .comment       0x0000000000000000       0x12 ../lib/freecom.lib(readcmd.obj)
 .comment       0x0000000000000000       0x12 ../lib/freecom.lib(realnum.obj)
 .comment       0x0000000000000000       0x12 ../lib/freecom.lib(res.obj)
 .comment       0x0000000000000000       0x12 ../lib/freecom.lib(res_r.obj)
 .comment       0x0000000000000000       0x12 ../lib/freecom.lib(res_vald.obj)
 .comment       0x0000000000000000       0x12 ../lib/freecom.lib(resfile.obj)
 .comment       0x0000000000000000       0x12 ../lib/freecom.lib(rmtmpfil.obj)
 .comment       0x0000000000000000       0x12 ../lib/freecom.lib(rtrimcl.obj)
 .comment       0x0000000000000000       0x12 ../lib/freecom.lib(rtrimsp.obj)
 .comment       0x0000000000000000       0x12 ../lib/freecom.lib(salloc.obj)
 .comment       0x0000000000000000       0x12 ../lib/freecom.lib(samefile.obj)
 .comment       0x0000000000000000       0x12 ../lib/freecom.lib(scancmd.obj)
 .comment       0x0000000000000000       0x12 ../lib/freecom.lib(scanopt.obj)
 .comment       0x0000000000000000       0x12 ../lib/freecom.lib(session.obj)
 .comment       0x0000000000000000       0x12 ../lib/freecom.lib(showcmds.obj)
 .comment       0x0000000000000000       0x12 ../lib/freecom.lib(skqwd.obj)
 .comment       0x0000000000000000       0x12 ../lib/freecom.lib(spfnam.obj)
 .comment       0x0000000000000000       0x12 ../lib/freecom.lib(split.obj)
 .comment       0x0000000000000000       0x12 ../lib/freecom.lib(sumblink.obj)
 .comment       0x0000000000000000       0x12 ../lib/freecom.lib(timeget.obj)
 .comment       0x0000000000000000       0x12 ../lib/freecom.lib(timeset.obj)
 .comment       0x0000000000000000       0x12 ../lib/freecom.lib(tmpnam.obj)
 .comment       0x0000000000000000       0x12 ../lib/freecom.lib(trimsp.obj)
 .comment       0x0000000000000000       0x12 ../lib/freecom.lib(truepath.obj)
 .comment       0x0000000000000000       0x12 ../lib/freecom.lib(truncate.obj)
 .comment       0x0000000000000000       0x12 ../lib/freecom.lib(txtlend.obj)
 .comment       0x0000000000000000       0x12 ../lib/freecom.lib(unquote.obj)
 .comment       0x0000000000000000       0x12 ../lib/freecom.lib(vcgetch.obj)
 .comment       0x0000000000000000       0x12 ../lib/freecom.lib(where.obj)
 .comment       0x0000000000000000       0x12 ../lib/freecom.lib(delay.obj)
 .comment       0x0000000000000000       0x12 ../lib/freecom.lib(err2.obj)
 .comment       0x0000000000000000       0x12 ../lib/freecom.lib(err3.obj)
 .comment       0x0000000000000000       0x12 ../lib/freecom.lib(err5.obj)
 .comment       0x0000000000000000       0x12 ../lib/freecom.lib(err6.obj)
 .comment       0x0000000000000000       0x12 ../lib/freecom.lib(err7.obj)
 .comment       0x0000000000000000       0x12 ../lib/freecom.lib(err8.obj)
 .comment       0x0000000000000000       0x12 ../lib/freecom.lib(err10.obj)
 .comment       0x0000000000000000       0x12 ../lib/freecom.lib(err11.obj)
 .comment       0x0000000000000000       0x12 ../lib/freecom.lib(err13.obj)
 .comment       0x0000000000000000       0x12 ../lib/freecom.lib(err14.obj)
 .comment       0x0000000000000000       0x12 ../lib/freecom.lib(err15.obj)
 .comment       0x0000000000000000       0x12 ../lib/freecom.lib(err16.obj)
 .comment       0x0000000000000000       0x12 ../lib/freecom.lib(err17.obj)
 .comment       0x0000000000000000       0x12 ../lib/freecom.lib(err18.obj)
 .comment       0x0000000000000000       0x12 ../lib/freecom.lib(err19.obj)
 .comment       0x0000000000000000       0x12 ../lib/freecom.lib(err20.obj)
 .comment       0x0000000000000000       0x12 ../lib/freecom.lib(err21.obj)
 .comment       0x0000000000000000       0x12 ../lib/freecom.lib(err22.obj)
 .comment       0x0000000000000000       0x12 ../lib/freecom.lib(err23.obj)
 .comment       0x0000000000000000       0x12 ../lib/freecom.lib(err25.obj)
 .comment       0x0000000000000000       0x12 ../lib/freecom.lib(err26.obj)
 .comment       0x0000000000000000       0x12 ../lib/freecom.lib(err27.obj)
 .comment       0x0000000000000000       0x12 ../lib/freecom.lib(err28.obj)
 .comment       0x0000000000000000       0x12 ../lib/freecom.lib(err29.obj)
 .comment       0x0000000000000000       0x12 ../lib/freecom.lib(err30.obj)
 .comment       0x0000000000000000       0x12 ../lib/freecom.lib(err31.obj)
 .comment       0x0000000000000000       0x12 ../lib/freecom.lib(err32.obj)
 .comment       0x0000000000000000       0x12 ../lib/freecom.lib(err33.obj)
 .comment       0x0000000000000000       0x12 ../lib/freecom.lib(err34.obj)
 .comment       0x0000000000000000       0x12 ../lib/freecom.lib(err35.obj)
 .comment       0x0000000000000000       0x12 ../lib/freecom.lib(err36.obj)
 .comment       0x0000000000000000       0x12 ../lib/freecom.lib(err37.obj)
 .comment       0x0000000000000000       0x12 ../lib/freecom.lib(err38.obj)
 .comment       0x0000000000000000       0x12 ../lib/freecom.lib(err39.obj)
 .comment       0x0000000000000000       0x12 ../lib/freecom.lib(err41.obj)
 .comment       0x0000000000000000       0x12 ../lib/freecom.lib(err42.obj)
 .comment       0x0000000000000000       0x12 ../lib/freecom.lib(err45.obj)
 .comment       0x0000000000000000       0x12 ../lib/freecom.lib(err46.obj)
 .comment       0x0000000000000000       0x12 ../lib/freecom.lib(err47.obj)
 .comment       0x0000000000000000       0x12 ../lib/freecom.lib(err50.obj)
 .comment       0x0000000000000000       0x12 ../lib/freecom.lib(err51.obj)
 .comment       0x0000000000000000       0x12 ../lib/freecom.lib(err53.obj)
 .comment       0x0000000000000000       0x12 ../lib/freecom.lib(err54.obj)
 .comment       0x0000000000000000       0x12 ../lib/freecom.lib(err58.obj)
 .comment       0x0000000000000000       0x12 ../lib/freecom.lib(err59.obj)
 .comment       0x0000000000000000       0x12 ../lib/freecom.lib(err60.obj)
 .comment       0x0000000000000000       0x12 ../lib/freecom.lib(err61.obj)
 .comment       0x0000000000000000       0x12 ../lib/freecom.lib(err63.obj)
 .comment       0x0000000000000000       0x12 ../lib/freecom.lib(err64.obj)
 .comment       0x0000000000000000       0x12 ../lib/freecom.lib(err65.obj)
 .comment       0x0000000000000000       0x12 ../lib/freecom.lib(err67.obj)
 .comment       0x0000000000000000       0x12 ../lib/freecom.lib(err68.obj)
 .comment       0x0000000000000000       0x12 ../lib/freecom.lib(err69.obj)
 .comment       0x0000000000000000       0x12 ../lib/freecom.lib(err70.obj)
 .comment       0x0000000000000000       0x12 ../lib/freecom.lib(err71.obj)
 .comment       0x0000000000000000       0x12 ../lib/freecom.lib(err72.obj)
 .comment       0x0000000000000000       0x12 ../lib/freecom.lib(err73.obj)
 .comment       0x0000000000000000       0x12 ../lib/freecom.lib(err74.obj)
 .comment       0x0000000000000000       0x12 ../lib/freecom.lib(err75.obj)
 .comment       0x0000000000000000       0x12 ../lib/freecom.lib(err76.obj)
 .comment       0x0000000000000000       0x12 ../lib/freecom.lib(err77.obj)
 .comment       0x0000000000000000       0x12 ../lib/freecom.lib(err78.obj)
 .comment       0x0000000000000000       0x12 ../lib/freecom.lib(err79.obj)
 .comment       0x0000000000000000       0x12 ../lib/freecom.lib(err80.obj)
 .comment       0x0000000000000000       0x12 ../lib/freecom.lib(err81.obj)
 .comment       0x0000000000000000       0x12 ../lib/freecom.lib(err82.obj)
 .comment       0x0000000000000000       0x12 ../lib/freecom.lib(err83.obj)
 .comment       0x0000000000000000       0x12 ../lib/freecom.lib(err84.obj)
 .comment       0x0000000000000000       0x12 ../lib/freecom.lib(err85.obj)
 .comment       0x0000000000000000       0x12 ../lib/freecom.lib(err86.obj)
 .comment       0x0000000000000000       0x12 ../lib/freecom.lib(err87.obj)
 .comment       0x0000000000000000       0x12 ../lib/freecom.lib(almemblk.obj)
 .comment       0x0000000000000000       0x12 ../lib/freecom.lib(beep_l.obj)
 .comment       0x0000000000000000       0x12 ../lib/freecom.lib(cbs.obj)
 .comment       0x0000000000000000       0x12 ../lib/freecom.lib(comfile.obj)
 .comment       0x0000000000000000       0x12 ../lib/freecom.lib(ctxt_as.obj)
 .comment       0x0000000000000000       0x12 ../lib/freecom.lib(dispexit.obj)
 .comment       0x0000000000000000       0x12 ../lib/freecom.lib(inputdos.obj)
 .comment       0x0000000000000000       0x12 ../lib/freecom.lib(ltrimsp.obj)
 .comment       0x0000000000000000       0x12 ../lib/freecom.lib(mktmpfil.obj)
 .comment       0x0000000000000000       0x12 ../lib/freecom.lib(msg_dflt.obj)
 .comment       0x0000000000000000       0x12 ../lib/freecom.lib(msg_get.obj)
 .comment       0x0000000000000000       0x12 ../lib/freecom.lib(parsenum.obj)
 .comment       0x0000000000000000       0x12 ../strings/strings.lib(str0011.obj)
 .comment       0x0000000000000000       0x12 ../strings/strings.lib(str0018.obj)
 .comment       0x0000000000000000       0x12 ../strings/strings.lib(str003c.obj)
 .comment       0x0000000000000000       0x12 ../strings/strings.lib(str00b1.obj)
 .comment       0x0000000000000000       0x12 ../strings/strings.lib(str00b2.obj)
 .comment       0x0000000000000000       0x12 ../strings/strings.lib(str00f4.obj)
 .comment       0x0000000000000000       0x12 ../strings/strings.lib(str00f5.obj)
 .comment       0x0000000000000000       0x12 ../strings/strings.lib(str00f6.obj)
 .comment       0x0000000000000000       0x12 ../suppl/suppl_s.lib(byte2par.obj)
 .comment       0x0000000000000000       0x12 ../suppl/suppl_s.lib(cntry.obj)
 .comment       0x0000000000000000       0x12 ../suppl/suppl_s.lib(dfnfnam.obj)
 .comment       0x0000000000000000       0x12 ../suppl/suppl_s.lib(dfnfullp.obj)
 .comment       0x0000000000000000       0x12 ../suppl/suppl_s.lib(dfnmerge.obj)
 .comment       0x0000000000000000       0x12 ../suppl/suppl_s.lib(dfnpath.obj)
 .comment       0x0000000000000000       0x12 ../suppl/suppl_s.lib(dfnstat.obj)
 .comment       0x0000000000000000       0x12 ../suppl/suppl_s.lib(dfntruen.obj)
 .comment       0x0000000000000000       0x12 ../suppl/suppl_s.lib(dosalloc.obj)
 .comment       0x0000000000000000       0x12 ../suppl/suppl_s.lib(dosfree.obj)
 .comment       0x0000000000000000       0x12 ../suppl/suppl_s.lib(dossize.obj)
 .comment       0x0000000000000000       0x12 ../suppl/suppl_s.lib(dstrfupr.obj)
 .comment       0x0000000000000000       0x12 ../suppl/suppl_s.lib(dstrtrim.obj)
 .comment       0x0000000000000000       0x12 ../suppl/suppl_s.lib(dstrupr.obj)
 .comment       0x0000000000000000       0x12 ../suppl/suppl_s.lib(enoallc.obj)
 .comment       0x0000000000000000       0x12 ../suppl/suppl_s.lib(enoreal.obj)
 .comment       0x0000000000000000       0x12 ../suppl/suppl_s.lib(enosetos.obj)
 .comment       0x0000000000000000       0x12 ../suppl/suppl_s.lib(env_chg.obj)
 .comment       0x0000000000000000       0x12 ../suppl/suppl_s.lib(env_dvar.obj)
 .comment       0x0000000000000000       0x12 ../suppl/suppl_s.lib(env_find.obj)
 .comment       0x0000000000000000       0x12 ../suppl/suppl_s.lib(env_fora.obj)
 .comment       0x0000000000000000       0x12 ../suppl/suppl_s.lib(env_free.obj)
 .comment       0x0000000000000000       0x12 ../suppl/suppl_s.lib(env_insv.obj)
 .comment       0x0000000000000000       0x12 ../suppl/suppl_s.lib(env_len.obj)
 .comment       0x0000000000000000       0x12 ../suppl/suppl_s.lib(env_mtch.obj)
 .comment       0x0000000000000000       0x12 ../suppl/suppl_s.lib(env_new.obj)
 .comment       0x0000000000000000       0x12 ../suppl/suppl_s.lib(env_nost.obj)
 .comment       0x0000000000000000       0x12 ../suppl/suppl_s.lib(env_ovrw.obj)
 .comment       0x0000000000000000       0x12 ../suppl/suppl_s.lib(env_repl.obj)
 .comment       0x0000000000000000       0x12 ../suppl/suppl_s.lib(env_rlsg.obj)
 .comment       0x0000000000000000       0x12 ../suppl/suppl_s.lib(env_scnt.obj)
 .comment       0x0000000000000000       0x12 ../suppl/suppl_s.lib(env_size.obj)
 .comment       0x0000000000000000       0x12 ../suppl/suppl_s.lib(env_strg.obj)
 .comment       0x0000000000000000       0x12 ../suppl/suppl_s.lib(env_sub.obj)
 .comment       0x0000000000000000       0x12 ../suppl/suppl_s.lib(env_var1.obj)
 .comment       0x0000000000000000       0x12 ../suppl/suppl_s.lib(env_var2.obj)
 .comment       0x0000000000000000       0x12 ../suppl/suppl_s.lib(fstrdup.obj)
 .comment       0x0000000000000000       0x12 ../suppl/suppl_s.lib(mcb_is.obj)
 .comment       0x0000000000000000       0x12 ../suppl/suppl_s.lib(mcb_leng.obj)
 .comment       0x0000000000000000       0x12 ../suppl/suppl_s.lib(mcb_nxt.obj)
 .comment       0x0000000000000000       0x12 ../suppl/suppl_s.lib(mcb_walk.obj)
 .comment       0x0000000000000000       0x12 ../suppl/suppl_s.lib(toupperx.obj)
 .comment       0x0000000000000000       0x12 ../suppl/suppl_s.lib(filefind.obj)
 .comment       0x0000000000000000       0x12 ../suppl/suppl_s.lib(invokedo.obj)
 .comment       0x0000000000000000       0x12 ../suppl/suppl_s.lib(addu.obj)
 .comment       0x0000000000000000       0x12 ../suppl/suppl_s.lib(dfndeli2.obj)
 .comment       0x0000000000000000       0x12 ../suppl/suppl_s.lib(dfndelim.obj)
 .comment       0x0000000000000000       0x12 ../suppl/suppl_s.lib(dfnexpan.obj)
 .comment       0x0000000000000000       0x12 ../suppl/suppl_s.lib(dfnsplit.obj)
 .comment       0x0000000000000000       0x12 ../suppl/suppl_s.lib(dfnsquee.obj)
 .comment       0x0000000000000000       0x12 ../suppl/suppl_s.lib(dmemcmpf.obj)
 .comment       0x0000000000000000       0x12 ../suppl/suppl_s.lib(dstrchar.obj)
 .comment       0x0000000000000000       0x12 ../suppl/suppl_s.lib(dstrleft.obj)
 .comment       0x0000000000000000       0x12 ../suppl/suppl_s.lib(dstrrepl.obj)
 .comment       0x0000000000000000       0x12 ../suppl/suppl_s.lib(enosdup.obj)
 .comment       0x0000000000000000       0x12 ../suppl/suppl_s.lib(env_del.obj)
 .comment       0x0000000000000000       0x12 ../suppl/suppl_s.lib(mcb_1st.obj)
 .debug_frame   0x0000000000000000       0x32 /home/evln/proj/build-ia16.202501/prefix/bin/../lib/gcc/ia16-elf/6.3.0/../../../../ia16-elf/lib/regparmcall/libi86.a(fmemmove.o)
 .debug_info    0x0000000000000000      0x9a1 /home/evln/proj/build-ia16.202501/prefix/bin/../lib/gcc/ia16-elf/6.3.0/../../../../ia16-elf/lib/regparmcall/libi86.a(fmemmove.o)
 .debug_abbrev  0x0000000000000000      0x1ed /home/evln/proj/build-ia16.202501/prefix/bin/../lib/gcc/ia16-elf/6.3.0/../../../../ia16-elf/lib/regparmcall/libi86.a(fmemmove.o)
 .debug_loc     0x0000000000000000       0xbe /home/evln/proj/build-ia16.202501/prefix/bin/../lib/gcc/ia16-elf/6.3.0/../../../../ia16-elf/lib/regparmcall/libi86.a(fmemmove.o)
 .debug_aranges
                0x0000000000000000       0x14 /home/evln/proj/build-ia16.202501/prefix/bin/../lib/gcc/ia16-elf/6.3.0/../../../../ia16-elf/lib/regparmcall/libi86.a(fmemmove.o)
 .debug_line    0x0000000000000000      0x233 /home/evln/proj/build-ia16.202501/prefix/bin/../lib/gcc/ia16-elf/6.3.0/../../../../ia16-elf/lib/regparmcall/libi86.a(fmemmove.o)
 .debug_str     0x0000000000000000      0x678 /home/evln/proj/build-ia16.202501/prefix/bin/../lib/gcc/ia16-elf/6.3.0/../../../../ia16-elf/lib/regparmcall/libi86.a(fmemmove.o)
 .comment       0x0000000000000000       0x12 /home/evln/proj/build-ia16.202501/prefix/bin/../lib/gcc/ia16-elf/6.3.0/../../../../ia16-elf/lib/regparmcall/libi86.a(fmemmove.o)
 .debug_frame   0x0000000000000000       0x46 /home/evln/proj/build-ia16.202501/prefix/bin/../lib/gcc/ia16-elf/6.3.0/../../../../ia16-elf/lib/regparmcall/libi86.a(getdcwd.o)
 .debug_info    0x0000000000000000      0xb69 /home/evln/proj/build-ia16.202501/prefix/bin/../lib/gcc/ia16-elf/6.3.0/../../../../ia16-elf/lib/regparmcall/libi86.a(getdcwd.o)
 .debug_abbrev  0x0000000000000000      0x27b /home/evln/proj/build-ia16.202501/prefix/bin/../lib/gcc/ia16-elf/6.3.0/../../../../ia16-elf/lib/regparmcall/libi86.a(getdcwd.o)
 .debug_loc     0x0000000000000000      0x22d /home/evln/proj/build-ia16.202501/prefix/bin/../lib/gcc/ia16-elf/6.3.0/../../../../ia16-elf/lib/regparmcall/libi86.a(getdcwd.o)
 .debug_aranges
                0x0000000000000000       0x14 /home/evln/proj/build-ia16.202501/prefix/bin/../lib/gcc/ia16-elf/6.3.0/../../../../ia16-elf/lib/regparmcall/libi86.a(getdcwd.o)
 .debug_ranges  0x0000000000000000       0x18 /home/evln/proj/build-ia16.202501/prefix/bin/../lib/gcc/ia16-elf/6.3.0/../../../../ia16-elf/lib/regparmcall/libi86.a(getdcwd.o)
 .debug_line    0x0000000000000000      0x28f /home/evln/proj/build-ia16.202501/prefix/bin/../lib/gcc/ia16-elf/6.3.0/../../../../ia16-elf/lib/regparmcall/libi86.a(getdcwd.o)
 .debug_str     0x0000000000000000      0x6f5 /home/evln/proj/build-ia16.202501/prefix/bin/../lib/gcc/ia16-elf/6.3.0/../../../../ia16-elf/lib/regparmcall/libi86.a(getdcwd.o)
 .comment       0x0000000000000000       0x12 /home/evln/proj/build-ia16.202501/prefix/bin/../lib/gcc/ia16-elf/6.3.0/../../../../ia16-elf/lib/regparmcall/libi86.a(getdcwd.o)
 .comment       0x0000000000000000       0x12 /home/evln/proj/build-ia16.202501/prefix/bin/../lib/gcc/ia16-elf/6.3.0/regparmcall/crtbegin.o
 .comment       0x0000000000000000       0x12 /home/evln/proj/build-ia16.202501/prefix/bin/../lib/gcc/ia16-elf/6.3.0/regparmcall/crtend.o
 .debug_frame   0x0000000000000000       0x2c /home/evln/proj/build-ia16.202501/prefix/bin/../lib/gcc/ia16-elf/6.3.0/../../../../ia16-elf/lib/regparmcall/libc.a(lib_a-atexit.o)
 .debug_info    0x0000000000000000      0x8f9 /home/evln/proj/build-ia16.202501/prefix/bin/../lib/gcc/ia16-elf/6.3.0/../../../../ia16-elf/lib/regparmcall/libc.a(lib_a-atexit.o)
 .debug_abbrev  0x0000000000000000      0x19f /home/evln/proj/build-ia16.202501/prefix/bin/../lib/gcc/ia16-elf/6.3.0/../../../../ia16-elf/lib/regparmcall/libc.a(lib_a-atexit.o)
 .debug_loc     0x0000000000000000       0x26 /home/evln/proj/build-ia16.202501/prefix/bin/../lib/gcc/ia16-elf/6.3.0/../../../../ia16-elf/lib/regparmcall/libc.a(lib_a-atexit.o)
 .debug_aranges
                0x0000000000000000       0x14 /home/evln/proj/build-ia16.202501/prefix/bin/../lib/gcc/ia16-elf/6.3.0/../../../../ia16-elf/lib/regparmcall/libc.a(lib_a-atexit.o)
 .debug_line    0x0000000000000000      0x1cd /home/evln/proj/build-ia16.202501/prefix/bin/../lib/gcc/ia16-elf/6.3.0/../../../../ia16-elf/lib/regparmcall/libc.a(lib_a-atexit.o)
 .debug_str     0x0000000000000000      0x5e0 /home/evln/proj/build-ia16.202501/prefix/bin/../lib/gcc/ia16-elf/6.3.0/../../../../ia16-elf/lib/regparmcall/libc.a(lib_a-atexit.o)
 .comment       0x0000000000000000       0x12 /home/evln/proj/build-ia16.202501/prefix/bin/../lib/gcc/ia16-elf/6.3.0/../../../../ia16-elf/lib/regparmcall/libc.a(lib_a-atexit.o)
 .debug_frame   0x0000000000000000       0x38 /home/evln/proj/build-ia16.202501/prefix/bin/../lib/gcc/ia16-elf/6.3.0/../../../../ia16-elf/lib/regparmcall/libc.a(lib_a-atol.o)
 .debug_info    0x0000000000000000      0x93c /home/evln/proj/build-ia16.202501/prefix/bin/../lib/gcc/ia16-elf/6.3.0/../../../../ia16-elf/lib/regparmcall/libc.a(lib_a-atol.o)
 .debug_abbrev  0x0000000000000000      0x193 /home/evln/proj/build-ia16.202501/prefix/bin/../lib/gcc/ia16-elf/6.3.0/../../../../ia16-elf/lib/regparmcall/libc.a(lib_a-atol.o)
 .debug_loc     0x0000000000000000       0x4e /home/evln/proj/build-ia16.202501/prefix/bin/../lib/gcc/ia16-elf/6.3.0/../../../../ia16-elf/lib/regparmcall/libc.a(lib_a-atol.o)
 .debug_aranges
                0x0000000000000000       0x14 /home/evln/proj/build-ia16.202501/prefix/bin/../lib/gcc/ia16-elf/6.3.0/../../../../ia16-elf/lib/regparmcall/libc.a(lib_a-atol.o)
 .debug_line    0x0000000000000000      0x1c1 /home/evln/proj/build-ia16.202501/prefix/bin/../lib/gcc/ia16-elf/6.3.0/../../../../ia16-elf/lib/regparmcall/libc.a(lib_a-atol.o)
 .debug_str     0x0000000000000000      0x5b1 /home/evln/proj/build-ia16.202501/prefix/bin/../lib/gcc/ia16-elf/6.3.0/../../../../ia16-elf/lib/regparmcall/libc.a(lib_a-atol.o)
 .comment       0x0000000000000000       0x12 /home/evln/proj/build-ia16.202501/prefix/bin/../lib/gcc/ia16-elf/6.3.0/../../../../ia16-elf/lib/regparmcall/libc.a(lib_a-atol.o)
 .debug_frame   0x0000000000000000       0x1e /home/evln/proj/build-ia16.202501/prefix/bin/../lib/gcc/ia16-elf/6.3.0/../../../../ia16-elf/lib/regparmcall/libc.a(lib_a-ctype_.o)
 .debug_info    0x0000000000000000      0x10f /home/evln/proj/build-ia16.202501/prefix/bin/../lib/gcc/ia16-elf/6.3.0/../../../../ia16-elf/lib/regparmcall/libc.a(lib_a-ctype_.o)
 .debug_abbrev  0x0000000000000000       0xa3 /home/evln/proj/build-ia16.202501/prefix/bin/../lib/gcc/ia16-elf/6.3.0/../../../../ia16-elf/lib/regparmcall/libc.a(lib_a-ctype_.o)
 .debug_aranges
                0x0000000000000000       0x14 /home/evln/proj/build-ia16.202501/prefix/bin/../lib/gcc/ia16-elf/6.3.0/../../../../ia16-elf/lib/regparmcall/libc.a(lib_a-ctype_.o)
 .debug_line    0x0000000000000000       0xb3 /home/evln/proj/build-ia16.202501/prefix/bin/../lib/gcc/ia16-elf/6.3.0/../../../../ia16-elf/lib/regparmcall/libc.a(lib_a-ctype_.o)
 .debug_str     0x0000000000000000      0x1bf /home/evln/proj/build-ia16.202501/prefix/bin/../lib/gcc/ia16-elf/6.3.0/../../../../ia16-elf/lib/regparmcall/libc.a(lib_a-ctype_.o)
 .comment       0x0000000000000000       0x12 /home/evln/proj/build-ia16.202501/prefix/bin/../lib/gcc/ia16-elf/6.3.0/../../../../ia16-elf/lib/regparmcall/libc.a(lib_a-ctype_.o)
 .debug_frame   0x0000000000000000       0x1e /home/evln/proj/build-ia16.202501/prefix/bin/../lib/gcc/ia16-elf/6.3.0/../../../../ia16-elf/lib/regparmcall/libc.a(lib_a-errno.o)
 .debug_info    0x0000000000000000      0x89a /home/evln/proj/build-ia16.202501/prefix/bin/../lib/gcc/ia16-elf/6.3.0/../../../../ia16-elf/lib/regparmcall/libc.a(lib_a-errno.o)
 .debug_abbrev  0x0000000000000000      0x151 /home/evln/proj/build-ia16.202501/prefix/bin/../lib/gcc/ia16-elf/6.3.0/../../../../ia16-elf/lib/regparmcall/libc.a(lib_a-errno.o)
 .debug_aranges
                0x0000000000000000       0x14 /home/evln/proj/build-ia16.202501/prefix/bin/../lib/gcc/ia16-elf/6.3.0/../../../../ia16-elf/lib/regparmcall/libc.a(lib_a-errno.o)
 .debug_line    0x0000000000000000      0x172 /home/evln/proj/build-ia16.202501/prefix/bin/../lib/gcc/ia16-elf/6.3.0/../../../../ia16-elf/lib/regparmcall/libc.a(lib_a-errno.o)
 .debug_str     0x0000000000000000      0x59b /home/evln/proj/build-ia16.202501/prefix/bin/../lib/gcc/ia16-elf/6.3.0/../../../../ia16-elf/lib/regparmcall/libc.a(lib_a-errno.o)
 .comment       0x0000000000000000       0x12 /home/evln/proj/build-ia16.202501/prefix/bin/../lib/gcc/ia16-elf/6.3.0/../../../../ia16-elf/lib/regparmcall/libc.a(lib_a-errno.o)
 .debug_frame   0x0000000000000000       0x26 /home/evln/proj/build-ia16.202501/prefix/bin/../lib/gcc/ia16-elf/6.3.0/../../../../ia16-elf/lib/regparmcall/libc.a(lib_a-exit.o)
 .debug_info    0x0000000000000000      0x92c /home/evln/proj/build-ia16.202501/prefix/bin/../lib/gcc/ia16-elf/6.3.0/../../../../ia16-elf/lib/regparmcall/libc.a(lib_a-exit.o)
 .debug_abbrev  0x0000000000000000      0x193 /home/evln/proj/build-ia16.202501/prefix/bin/../lib/gcc/ia16-elf/6.3.0/../../../../ia16-elf/lib/regparmcall/libc.a(lib_a-exit.o)
 .debug_loc     0x0000000000000000       0x17 /home/evln/proj/build-ia16.202501/prefix/bin/../lib/gcc/ia16-elf/6.3.0/../../../../ia16-elf/lib/regparmcall/libc.a(lib_a-exit.o)
 .debug_aranges
                0x0000000000000000       0x14 /home/evln/proj/build-ia16.202501/prefix/bin/../lib/gcc/ia16-elf/6.3.0/../../../../ia16-elf/lib/regparmcall/libc.a(lib_a-exit.o)
 .debug_line    0x0000000000000000      0x1d9 /home/evln/proj/build-ia16.202501/prefix/bin/../lib/gcc/ia16-elf/6.3.0/../../../../ia16-elf/lib/regparmcall/libc.a(lib_a-exit.o)
 .debug_str     0x0000000000000000      0x5e1 /home/evln/proj/build-ia16.202501/prefix/bin/../lib/gcc/ia16-elf/6.3.0/../../../../ia16-elf/lib/regparmcall/libc.a(lib_a-exit.o)
 .comment       0x0000000000000000       0x12 /home/evln/proj/build-ia16.202501/prefix/bin/../lib/gcc/ia16-elf/6.3.0/../../../../ia16-elf/lib/regparmcall/libc.a(lib_a-exit.o)
 .debug_info    0x0000000000000000      0x875 /home/evln/proj/build-ia16.202501/prefix/bin/../lib/gcc/ia16-elf/6.3.0/../../../../ia16-elf/lib/regparmcall/libc.a(lib_a-impure.o)
 .debug_abbrev  0x0000000000000000      0x135 /home/evln/proj/build-ia16.202501/prefix/bin/../lib/gcc/ia16-elf/6.3.0/../../../../ia16-elf/lib/regparmcall/libc.a(lib_a-impure.o)
 .debug_aranges
                0x0000000000000000       0x10 /home/evln/proj/build-ia16.202501/prefix/bin/../lib/gcc/ia16-elf/6.3.0/../../../../ia16-elf/lib/regparmcall/libc.a(lib_a-impure.o)
 .debug_line    0x0000000000000000      0x103 /home/evln/proj/build-ia16.202501/prefix/bin/../lib/gcc/ia16-elf/6.3.0/../../../../ia16-elf/lib/regparmcall/libc.a(lib_a-impure.o)
 .debug_str     0x0000000000000000      0x589 /home/evln/proj/build-ia16.202501/prefix/bin/../lib/gcc/ia16-elf/6.3.0/../../../../ia16-elf/lib/regparmcall/libc.a(lib_a-impure.o)
 .comment       0x0000000000000000       0x12 /home/evln/proj/build-ia16.202501/prefix/bin/../lib/gcc/ia16-elf/6.3.0/../../../../ia16-elf/lib/regparmcall/libc.a(lib_a-impure.o)
 .debug_frame   0x0000000000000000       0x2a /home/evln/proj/build-ia16.202501/prefix/bin/../lib/gcc/ia16-elf/6.3.0/../../../../ia16-elf/lib/regparmcall/libc.a(lib_a-malloc.o)
 .debug_info    0x0000000000000000      0x90e /home/evln/proj/build-ia16.202501/prefix/bin/../lib/gcc/ia16-elf/6.3.0/../../../../ia16-elf/lib/regparmcall/libc.a(lib_a-malloc.o)
 .debug_abbrev  0x0000000000000000      0x1a2 /home/evln/proj/build-ia16.202501/prefix/bin/../lib/gcc/ia16-elf/6.3.0/../../../../ia16-elf/lib/regparmcall/libc.a(lib_a-malloc.o)
 .debug_loc     0x0000000000000000       0x4c /home/evln/proj/build-ia16.202501/prefix/bin/../lib/gcc/ia16-elf/6.3.0/../../../../ia16-elf/lib/regparmcall/libc.a(lib_a-malloc.o)
 .debug_aranges
                0x0000000000000000       0x14 /home/evln/proj/build-ia16.202501/prefix/bin/../lib/gcc/ia16-elf/6.3.0/../../../../ia16-elf/lib/regparmcall/libc.a(lib_a-malloc.o)
 .debug_line    0x0000000000000000      0x1cf /home/evln/proj/build-ia16.202501/prefix/bin/../lib/gcc/ia16-elf/6.3.0/../../../../ia16-elf/lib/regparmcall/libc.a(lib_a-malloc.o)
 .debug_str     0x0000000000000000      0x5c6 /home/evln/proj/build-ia16.202501/prefix/bin/../lib/gcc/ia16-elf/6.3.0/../../../../ia16-elf/lib/regparmcall/libc.a(lib_a-malloc.o)
 .comment       0x0000000000000000       0x12 /home/evln/proj/build-ia16.202501/prefix/bin/../lib/gcc/ia16-elf/6.3.0/../../../../ia16-elf/lib/regparmcall/libc.a(lib_a-malloc.o)
 .debug_frame   0x0000000000000000       0x38 /home/evln/proj/build-ia16.202501/prefix/bin/../lib/gcc/ia16-elf/6.3.0/../../../../ia16-elf/lib/regparmcall/libc.a(lib_a-nano-freer.o)
 .debug_info    0x0000000000000000      0xb65 /home/evln/proj/build-ia16.202501/prefix/bin/../lib/gcc/ia16-elf/6.3.0/../../../../ia16-elf/lib/regparmcall/libc.a(lib_a-nano-freer.o)
 .debug_abbrev  0x0000000000000000      0x222 /home/evln/proj/build-ia16.202501/prefix/bin/../lib/gcc/ia16-elf/6.3.0/../../../../ia16-elf/lib/regparmcall/libc.a(lib_a-nano-freer.o)
 .debug_loc     0x0000000000000000       0x90 /home/evln/proj/build-ia16.202501/prefix/bin/../lib/gcc/ia16-elf/6.3.0/../../../../ia16-elf/lib/regparmcall/libc.a(lib_a-nano-freer.o)
 .debug_aranges
                0x0000000000000000       0x14 /home/evln/proj/build-ia16.202501/prefix/bin/../lib/gcc/ia16-elf/6.3.0/../../../../ia16-elf/lib/regparmcall/libc.a(lib_a-nano-freer.o)
 .debug_line    0x0000000000000000      0x26c /home/evln/proj/build-ia16.202501/prefix/bin/../lib/gcc/ia16-elf/6.3.0/../../../../ia16-elf/lib/regparmcall/libc.a(lib_a-nano-freer.o)
 .debug_str     0x0000000000000000      0x6ea /home/evln/proj/build-ia16.202501/prefix/bin/../lib/gcc/ia16-elf/6.3.0/../../../../ia16-elf/lib/regparmcall/libc.a(lib_a-nano-freer.o)
 .comment       0x0000000000000000       0x12 /home/evln/proj/build-ia16.202501/prefix/bin/../lib/gcc/ia16-elf/6.3.0/../../../../ia16-elf/lib/regparmcall/libc.a(lib_a-nano-freer.o)
 .debug_frame   0x0000000000000000       0x32 /home/evln/proj/build-ia16.202501/prefix/bin/../lib/gcc/ia16-elf/6.3.0/../../../../ia16-elf/lib/regparmcall/libc.a(lib_a-nano-mallocr.o)
 .debug_info    0x0000000000000000      0xc6a /home/evln/proj/build-ia16.202501/prefix/bin/../lib/gcc/ia16-elf/6.3.0/../../../../ia16-elf/lib/regparmcall/libc.a(lib_a-nano-mallocr.o)
 .debug_abbrev  0x0000000000000000      0x286 /home/evln/proj/build-ia16.202501/prefix/bin/../lib/gcc/ia16-elf/6.3.0/../../../../ia16-elf/lib/regparmcall/libc.a(lib_a-nano-mallocr.o)
 .debug_loc     0x0000000000000000      0x25a /home/evln/proj/build-ia16.202501/prefix/bin/../lib/gcc/ia16-elf/6.3.0/../../../../ia16-elf/lib/regparmcall/libc.a(lib_a-nano-mallocr.o)
 .debug_aranges
                0x0000000000000000       0x14 /home/evln/proj/build-ia16.202501/prefix/bin/../lib/gcc/ia16-elf/6.3.0/../../../../ia16-elf/lib/regparmcall/libc.a(lib_a-nano-mallocr.o)
 .debug_ranges  0x0000000000000000       0x20 /home/evln/proj/build-ia16.202501/prefix/bin/../lib/gcc/ia16-elf/6.3.0/../../../../ia16-elf/lib/regparmcall/libc.a(lib_a-nano-mallocr.o)
 .debug_line    0x0000000000000000      0x2f6 /home/evln/proj/build-ia16.202501/prefix/bin/../lib/gcc/ia16-elf/6.3.0/../../../../ia16-elf/lib/regparmcall/libc.a(lib_a-nano-mallocr.o)
 .debug_str     0x0000000000000000      0x72d /home/evln/proj/build-ia16.202501/prefix/bin/../lib/gcc/ia16-elf/6.3.0/../../../../ia16-elf/lib/regparmcall/libc.a(lib_a-nano-mallocr.o)
 .comment       0x0000000000000000       0x12 /home/evln/proj/build-ia16.202501/prefix/bin/../lib/gcc/ia16-elf/6.3.0/../../../../ia16-elf/lib/regparmcall/libc.a(lib_a-nano-mallocr.o)
 .debug_frame   0x0000000000000000       0x7a /home/evln/proj/build-ia16.202501/prefix/bin/../lib/gcc/ia16-elf/6.3.0/../../../../ia16-elf/lib/regparmcall/libc.a(lib_a-qsort.o)
 .debug_info    0x0000000000000000      0xf91 /home/evln/proj/build-ia16.202501/prefix/bin/../lib/gcc/ia16-elf/6.3.0/../../../../ia16-elf/lib/regparmcall/libc.a(lib_a-qsort.o)
 .debug_abbrev  0x0000000000000000      0x2cb /home/evln/proj/build-ia16.202501/prefix/bin/../lib/gcc/ia16-elf/6.3.0/../../../../ia16-elf/lib/regparmcall/libc.a(lib_a-qsort.o)
 .debug_loc     0x0000000000000000      0x6fe /home/evln/proj/build-ia16.202501/prefix/bin/../lib/gcc/ia16-elf/6.3.0/../../../../ia16-elf/lib/regparmcall/libc.a(lib_a-qsort.o)
 .debug_aranges
                0x0000000000000000       0x14 /home/evln/proj/build-ia16.202501/prefix/bin/../lib/gcc/ia16-elf/6.3.0/../../../../ia16-elf/lib/regparmcall/libc.a(lib_a-qsort.o)
 .debug_ranges  0x0000000000000000        0xc /home/evln/proj/build-ia16.202501/prefix/bin/../lib/gcc/ia16-elf/6.3.0/../../../../ia16-elf/lib/regparmcall/libc.a(lib_a-qsort.o)
 .debug_line    0x0000000000000000      0x2de /home/evln/proj/build-ia16.202501/prefix/bin/../lib/gcc/ia16-elf/6.3.0/../../../../ia16-elf/lib/regparmcall/libc.a(lib_a-qsort.o)
 .debug_str     0x0000000000000000      0x5dd /home/evln/proj/build-ia16.202501/prefix/bin/../lib/gcc/ia16-elf/6.3.0/../../../../ia16-elf/lib/regparmcall/libc.a(lib_a-qsort.o)
 .comment       0x0000000000000000       0x12 /home/evln/proj/build-ia16.202501/prefix/bin/../lib/gcc/ia16-elf/6.3.0/../../../../ia16-elf/lib/regparmcall/libc.a(lib_a-qsort.o)
 .debug_frame   0x0000000000000000       0x1e /home/evln/proj/build-ia16.202501/prefix/bin/../lib/gcc/ia16-elf/6.3.0/../../../../ia16-elf/lib/regparmcall/libc.a(lib_a-realloc.o)
 .debug_info    0x0000000000000000      0x8e8 /home/evln/proj/build-ia16.202501/prefix/bin/../lib/gcc/ia16-elf/6.3.0/../../../../ia16-elf/lib/regparmcall/libc.a(lib_a-realloc.o)
 .debug_abbrev  0x0000000000000000      0x197 /home/evln/proj/build-ia16.202501/prefix/bin/../lib/gcc/ia16-elf/6.3.0/../../../../ia16-elf/lib/regparmcall/libc.a(lib_a-realloc.o)
 .debug_loc     0x0000000000000000       0x4c /home/evln/proj/build-ia16.202501/prefix/bin/../lib/gcc/ia16-elf/6.3.0/../../../../ia16-elf/lib/regparmcall/libc.a(lib_a-realloc.o)
 .debug_aranges
                0x0000000000000000       0x14 /home/evln/proj/build-ia16.202501/prefix/bin/../lib/gcc/ia16-elf/6.3.0/../../../../ia16-elf/lib/regparmcall/libc.a(lib_a-realloc.o)
 .debug_line    0x0000000000000000      0x1cd /home/evln/proj/build-ia16.202501/prefix/bin/../lib/gcc/ia16-elf/6.3.0/../../../../ia16-elf/lib/regparmcall/libc.a(lib_a-realloc.o)
 .debug_str     0x0000000000000000      0x5b7 /home/evln/proj/build-ia16.202501/prefix/bin/../lib/gcc/ia16-elf/6.3.0/../../../../ia16-elf/lib/regparmcall/libc.a(lib_a-realloc.o)
 .comment       0x0000000000000000       0x12 /home/evln/proj/build-ia16.202501/prefix/bin/../lib/gcc/ia16-elf/6.3.0/../../../../ia16-elf/lib/regparmcall/libc.a(lib_a-realloc.o)
 .debug_frame   0x0000000000000000       0x2a /home/evln/proj/build-ia16.202501/prefix/bin/../lib/gcc/ia16-elf/6.3.0/../../../../ia16-elf/lib/regparmcall/libc.a(lib_a-remove.o)
 .debug_info    0x0000000000000000      0x8f1 /home/evln/proj/build-ia16.202501/prefix/bin/../lib/gcc/ia16-elf/6.3.0/../../../../ia16-elf/lib/regparmcall/libc.a(lib_a-remove.o)
 .debug_abbrev  0x0000000000000000      0x1ad /home/evln/proj/build-ia16.202501/prefix/bin/../lib/gcc/ia16-elf/6.3.0/../../../../ia16-elf/lib/regparmcall/libc.a(lib_a-remove.o)
 .debug_loc     0x0000000000000000       0x5a /home/evln/proj/build-ia16.202501/prefix/bin/../lib/gcc/ia16-elf/6.3.0/../../../../ia16-elf/lib/regparmcall/libc.a(lib_a-remove.o)
 .debug_aranges
                0x0000000000000000       0x14 /home/evln/proj/build-ia16.202501/prefix/bin/../lib/gcc/ia16-elf/6.3.0/../../../../ia16-elf/lib/regparmcall/libc.a(lib_a-remove.o)
 .debug_line    0x0000000000000000      0x168 /home/evln/proj/build-ia16.202501/prefix/bin/../lib/gcc/ia16-elf/6.3.0/../../../../ia16-elf/lib/regparmcall/libc.a(lib_a-remove.o)
 .debug_str     0x0000000000000000      0x5a1 /home/evln/proj/build-ia16.202501/prefix/bin/../lib/gcc/ia16-elf/6.3.0/../../../../ia16-elf/lib/regparmcall/libc.a(lib_a-remove.o)
 .comment       0x0000000000000000       0x12 /home/evln/proj/build-ia16.202501/prefix/bin/../lib/gcc/ia16-elf/6.3.0/../../../../ia16-elf/lib/regparmcall/libc.a(lib_a-remove.o)
 .debug_frame   0x0000000000000000       0x32 /home/evln/proj/build-ia16.202501/prefix/bin/../lib/gcc/ia16-elf/6.3.0/../../../../ia16-elf/lib/regparmcall/libc.a(lib_a-strcasecmp.o)
 .debug_info    0x0000000000000000      0x93b /home/evln/proj/build-ia16.202501/prefix/bin/../lib/gcc/ia16-elf/6.3.0/../../../../ia16-elf/lib/regparmcall/libc.a(lib_a-strcasecmp.o)
 .debug_abbrev  0x0000000000000000      0x190 /home/evln/proj/build-ia16.202501/prefix/bin/../lib/gcc/ia16-elf/6.3.0/../../../../ia16-elf/lib/regparmcall/libc.a(lib_a-strcasecmp.o)
 .debug_loc     0x0000000000000000      0x1e1 /home/evln/proj/build-ia16.202501/prefix/bin/../lib/gcc/ia16-elf/6.3.0/../../../../ia16-elf/lib/regparmcall/libc.a(lib_a-strcasecmp.o)
 .debug_aranges
                0x0000000000000000       0x14 /home/evln/proj/build-ia16.202501/prefix/bin/../lib/gcc/ia16-elf/6.3.0/../../../../ia16-elf/lib/regparmcall/libc.a(lib_a-strcasecmp.o)
 .debug_ranges  0x0000000000000000       0x24 /home/evln/proj/build-ia16.202501/prefix/bin/../lib/gcc/ia16-elf/6.3.0/../../../../ia16-elf/lib/regparmcall/libc.a(lib_a-strcasecmp.o)
 .debug_line    0x0000000000000000      0x19a /home/evln/proj/build-ia16.202501/prefix/bin/../lib/gcc/ia16-elf/6.3.0/../../../../ia16-elf/lib/regparmcall/libc.a(lib_a-strcasecmp.o)
 .debug_str     0x0000000000000000      0x5ae /home/evln/proj/build-ia16.202501/prefix/bin/../lib/gcc/ia16-elf/6.3.0/../../../../ia16-elf/lib/regparmcall/libc.a(lib_a-strcasecmp.o)
 .comment       0x0000000000000000       0x12 /home/evln/proj/build-ia16.202501/prefix/bin/../lib/gcc/ia16-elf/6.3.0/../../../../ia16-elf/lib/regparmcall/libc.a(lib_a-strcasecmp.o)
 .debug_frame   0x0000000000000000       0x28 /home/evln/proj/build-ia16.202501/prefix/bin/../lib/gcc/ia16-elf/6.3.0/../../../../ia16-elf/lib/regparmcall/libc.a(lib_a-strcat.o)
 .debug_info    0x0000000000000000      0x8a0 /home/evln/proj/build-ia16.202501/prefix/bin/../lib/gcc/ia16-elf/6.3.0/../../../../ia16-elf/lib/regparmcall/libc.a(lib_a-strcat.o)
 .debug_abbrev  0x0000000000000000      0x160 /home/evln/proj/build-ia16.202501/prefix/bin/../lib/gcc/ia16-elf/6.3.0/../../../../ia16-elf/lib/regparmcall/libc.a(lib_a-strcat.o)
 .debug_loc     0x0000000000000000       0x7b /home/evln/proj/build-ia16.202501/prefix/bin/../lib/gcc/ia16-elf/6.3.0/../../../../ia16-elf/lib/regparmcall/libc.a(lib_a-strcat.o)
 .debug_aranges
                0x0000000000000000       0x14 /home/evln/proj/build-ia16.202501/prefix/bin/../lib/gcc/ia16-elf/6.3.0/../../../../ia16-elf/lib/regparmcall/libc.a(lib_a-strcat.o)
 .debug_line    0x0000000000000000      0x167 /home/evln/proj/build-ia16.202501/prefix/bin/../lib/gcc/ia16-elf/6.3.0/../../../../ia16-elf/lib/regparmcall/libc.a(lib_a-strcat.o)
 .debug_str     0x0000000000000000      0x586 /home/evln/proj/build-ia16.202501/prefix/bin/../lib/gcc/ia16-elf/6.3.0/../../../../ia16-elf/lib/regparmcall/libc.a(lib_a-strcat.o)
 .comment       0x0000000000000000       0x12 /home/evln/proj/build-ia16.202501/prefix/bin/../lib/gcc/ia16-elf/6.3.0/../../../../ia16-elf/lib/regparmcall/libc.a(lib_a-strcat.o)
 .debug_frame   0x0000000000000000       0x1e /home/evln/proj/build-ia16.202501/prefix/bin/../lib/gcc/ia16-elf/6.3.0/../../../../ia16-elf/lib/regparmcall/libc.a(lib_a-strdup.o)
 .debug_info    0x0000000000000000      0x8c3 /home/evln/proj/build-ia16.202501/prefix/bin/../lib/gcc/ia16-elf/6.3.0/../../../../ia16-elf/lib/regparmcall/libc.a(lib_a-strdup.o)
 .debug_abbrev  0x0000000000000000      0x188 /home/evln/proj/build-ia16.202501/prefix/bin/../lib/gcc/ia16-elf/6.3.0/../../../../ia16-elf/lib/regparmcall/libc.a(lib_a-strdup.o)
 .debug_loc     0x0000000000000000       0x26 /home/evln/proj/build-ia16.202501/prefix/bin/../lib/gcc/ia16-elf/6.3.0/../../../../ia16-elf/lib/regparmcall/libc.a(lib_a-strdup.o)
 .debug_aranges
                0x0000000000000000       0x14 /home/evln/proj/build-ia16.202501/prefix/bin/../lib/gcc/ia16-elf/6.3.0/../../../../ia16-elf/lib/regparmcall/libc.a(lib_a-strdup.o)
 .debug_line    0x0000000000000000      0x1ca /home/evln/proj/build-ia16.202501/prefix/bin/../lib/gcc/ia16-elf/6.3.0/../../../../ia16-elf/lib/regparmcall/libc.a(lib_a-strdup.o)
 .debug_str     0x0000000000000000      0x5a6 /home/evln/proj/build-ia16.202501/prefix/bin/../lib/gcc/ia16-elf/6.3.0/../../../../ia16-elf/lib/regparmcall/libc.a(lib_a-strdup.o)
 .comment       0x0000000000000000       0x12 /home/evln/proj/build-ia16.202501/prefix/bin/../lib/gcc/ia16-elf/6.3.0/../../../../ia16-elf/lib/regparmcall/libc.a(lib_a-strdup.o)
 .debug_frame   0x0000000000000000       0x30 /home/evln/proj/build-ia16.202501/prefix/bin/../lib/gcc/ia16-elf/6.3.0/../../../../ia16-elf/lib/regparmcall/libc.a(lib_a-strdup_r.o)
 .debug_info    0x0000000000000000      0x965 /home/evln/proj/build-ia16.202501/prefix/bin/../lib/gcc/ia16-elf/6.3.0/../../../../ia16-elf/lib/regparmcall/libc.a(lib_a-strdup_r.o)
 .debug_abbrev  0x0000000000000000      0x1d0 /home/evln/proj/build-ia16.202501/prefix/bin/../lib/gcc/ia16-elf/6.3.0/../../../../ia16-elf/lib/regparmcall/libc.a(lib_a-strdup_r.o)
 .debug_loc     0x0000000000000000       0x65 /home/evln/proj/build-ia16.202501/prefix/bin/../lib/gcc/ia16-elf/6.3.0/../../../../ia16-elf/lib/regparmcall/libc.a(lib_a-strdup_r.o)
 .debug_aranges
                0x0000000000000000       0x14 /home/evln/proj/build-ia16.202501/prefix/bin/../lib/gcc/ia16-elf/6.3.0/../../../../ia16-elf/lib/regparmcall/libc.a(lib_a-strdup_r.o)
 .debug_line    0x0000000000000000      0x1d0 /home/evln/proj/build-ia16.202501/prefix/bin/../lib/gcc/ia16-elf/6.3.0/../../../../ia16-elf/lib/regparmcall/libc.a(lib_a-strdup_r.o)
 .debug_str     0x0000000000000000      0x5cf /home/evln/proj/build-ia16.202501/prefix/bin/../lib/gcc/ia16-elf/6.3.0/../../../../ia16-elf/lib/regparmcall/libc.a(lib_a-strdup_r.o)
 .comment       0x0000000000000000       0x12 /home/evln/proj/build-ia16.202501/prefix/bin/../lib/gcc/ia16-elf/6.3.0/../../../../ia16-elf/lib/regparmcall/libc.a(lib_a-strdup_r.o)
 .debug_frame   0x0000000000000000       0x28 /home/evln/proj/build-ia16.202501/prefix/bin/../lib/gcc/ia16-elf/6.3.0/../../../../ia16-elf/lib/regparmcall/libc.a(lib_a-strlwr.o)
 .debug_info    0x0000000000000000      0x8c4 /home/evln/proj/build-ia16.202501/prefix/bin/../lib/gcc/ia16-elf/6.3.0/../../../../ia16-elf/lib/regparmcall/libc.a(lib_a-strlwr.o)
 .debug_abbrev  0x0000000000000000      0x176 /home/evln/proj/build-ia16.202501/prefix/bin/../lib/gcc/ia16-elf/6.3.0/../../../../ia16-elf/lib/regparmcall/libc.a(lib_a-strlwr.o)
 .debug_loc     0x0000000000000000       0x40 /home/evln/proj/build-ia16.202501/prefix/bin/../lib/gcc/ia16-elf/6.3.0/../../../../ia16-elf/lib/regparmcall/libc.a(lib_a-strlwr.o)
 .debug_aranges
                0x0000000000000000       0x14 /home/evln/proj/build-ia16.202501/prefix/bin/../lib/gcc/ia16-elf/6.3.0/../../../../ia16-elf/lib/regparmcall/libc.a(lib_a-strlwr.o)
 .debug_ranges  0x0000000000000000        0xc /home/evln/proj/build-ia16.202501/prefix/bin/../lib/gcc/ia16-elf/6.3.0/../../../../ia16-elf/lib/regparmcall/libc.a(lib_a-strlwr.o)
 .debug_line    0x0000000000000000      0x184 /home/evln/proj/build-ia16.202501/prefix/bin/../lib/gcc/ia16-elf/6.3.0/../../../../ia16-elf/lib/regparmcall/libc.a(lib_a-strlwr.o)
 .debug_str     0x0000000000000000      0x59c /home/evln/proj/build-ia16.202501/prefix/bin/../lib/gcc/ia16-elf/6.3.0/../../../../ia16-elf/lib/regparmcall/libc.a(lib_a-strlwr.o)
 .comment       0x0000000000000000       0x12 /home/evln/proj/build-ia16.202501/prefix/bin/../lib/gcc/ia16-elf/6.3.0/../../../../ia16-elf/lib/regparmcall/libc.a(lib_a-strlwr.o)
 .debug_frame   0x0000000000000000       0x32 /home/evln/proj/build-ia16.202501/prefix/bin/../lib/gcc/ia16-elf/6.3.0/../../../../ia16-elf/lib/regparmcall/libc.a(lib_a-strncasecmp.o)
 .debug_info    0x0000000000000000      0x953 /home/evln/proj/build-ia16.202501/prefix/bin/../lib/gcc/ia16-elf/6.3.0/../../../../ia16-elf/lib/regparmcall/libc.a(lib_a-strncasecmp.o)
 .debug_abbrev  0x0000000000000000      0x190 /home/evln/proj/build-ia16.202501/prefix/bin/../lib/gcc/ia16-elf/6.3.0/../../../../ia16-elf/lib/regparmcall/libc.a(lib_a-strncasecmp.o)
 .debug_loc     0x0000000000000000      0x227 /home/evln/proj/build-ia16.202501/prefix/bin/../lib/gcc/ia16-elf/6.3.0/../../../../ia16-elf/lib/regparmcall/libc.a(lib_a-strncasecmp.o)
 .debug_aranges
                0x0000000000000000       0x14 /home/evln/proj/build-ia16.202501/prefix/bin/../lib/gcc/ia16-elf/6.3.0/../../../../ia16-elf/lib/regparmcall/libc.a(lib_a-strncasecmp.o)
 .debug_ranges  0x0000000000000000       0x2c /home/evln/proj/build-ia16.202501/prefix/bin/../lib/gcc/ia16-elf/6.3.0/../../../../ia16-elf/lib/regparmcall/libc.a(lib_a-strncasecmp.o)
 .debug_line    0x0000000000000000      0x1a4 /home/evln/proj/build-ia16.202501/prefix/bin/../lib/gcc/ia16-elf/6.3.0/../../../../ia16-elf/lib/regparmcall/libc.a(lib_a-strncasecmp.o)
 .debug_str     0x0000000000000000      0x5b7 /home/evln/proj/build-ia16.202501/prefix/bin/../lib/gcc/ia16-elf/6.3.0/../../../../ia16-elf/lib/regparmcall/libc.a(lib_a-strncasecmp.o)
 .comment       0x0000000000000000       0x12 /home/evln/proj/build-ia16.202501/prefix/bin/../lib/gcc/ia16-elf/6.3.0/../../../../ia16-elf/lib/regparmcall/libc.a(lib_a-strncasecmp.o)
 .debug_frame   0x0000000000000000       0x32 /home/evln/proj/build-ia16.202501/prefix/bin/../lib/gcc/ia16-elf/6.3.0/../../../../ia16-elf/lib/regparmcall/libc.a(lib_a-strpbrk.o)
 .debug_info    0x0000000000000000      0x896 /home/evln/proj/build-ia16.202501/prefix/bin/../lib/gcc/ia16-elf/6.3.0/../../../../ia16-elf/lib/regparmcall/libc.a(lib_a-strpbrk.o)
 .debug_abbrev  0x0000000000000000      0x168 /home/evln/proj/build-ia16.202501/prefix/bin/../lib/gcc/ia16-elf/6.3.0/../../../../ia16-elf/lib/regparmcall/libc.a(lib_a-strpbrk.o)
 .debug_loc     0x0000000000000000       0x76 /home/evln/proj/build-ia16.202501/prefix/bin/../lib/gcc/ia16-elf/6.3.0/../../../../ia16-elf/lib/regparmcall/libc.a(lib_a-strpbrk.o)
 .debug_aranges
                0x0000000000000000       0x14 /home/evln/proj/build-ia16.202501/prefix/bin/../lib/gcc/ia16-elf/6.3.0/../../../../ia16-elf/lib/regparmcall/libc.a(lib_a-strpbrk.o)
 .debug_line    0x0000000000000000      0x171 /home/evln/proj/build-ia16.202501/prefix/bin/../lib/gcc/ia16-elf/6.3.0/../../../../ia16-elf/lib/regparmcall/libc.a(lib_a-strpbrk.o)
 .debug_str     0x0000000000000000      0x588 /home/evln/proj/build-ia16.202501/prefix/bin/../lib/gcc/ia16-elf/6.3.0/../../../../ia16-elf/lib/regparmcall/libc.a(lib_a-strpbrk.o)
 .comment       0x0000000000000000       0x12 /home/evln/proj/build-ia16.202501/prefix/bin/../lib/gcc/ia16-elf/6.3.0/../../../../ia16-elf/lib/regparmcall/libc.a(lib_a-strpbrk.o)
 .debug_frame   0x0000000000000000       0x28 /home/evln/proj/build-ia16.202501/prefix/bin/../lib/gcc/ia16-elf/6.3.0/../../../../ia16-elf/lib/regparmcall/libc.a(lib_a-strrchr.o)
 .debug_info    0x0000000000000000      0x8cd /home/evln/proj/build-ia16.202501/prefix/bin/../lib/gcc/ia16-elf/6.3.0/../../../../ia16-elf/lib/regparmcall/libc.a(lib_a-strrchr.o)
 .debug_abbrev  0x0000000000000000      0x193 /home/evln/proj/build-ia16.202501/prefix/bin/../lib/gcc/ia16-elf/6.3.0/../../../../ia16-elf/lib/regparmcall/libc.a(lib_a-strrchr.o)
 .debug_loc     0x0000000000000000       0xda /home/evln/proj/build-ia16.202501/prefix/bin/../lib/gcc/ia16-elf/6.3.0/../../../../ia16-elf/lib/regparmcall/libc.a(lib_a-strrchr.o)
 .debug_aranges
                0x0000000000000000       0x14 /home/evln/proj/build-ia16.202501/prefix/bin/../lib/gcc/ia16-elf/6.3.0/../../../../ia16-elf/lib/regparmcall/libc.a(lib_a-strrchr.o)
 .debug_line    0x0000000000000000      0x166 /home/evln/proj/build-ia16.202501/prefix/bin/../lib/gcc/ia16-elf/6.3.0/../../../../ia16-elf/lib/regparmcall/libc.a(lib_a-strrchr.o)
 .debug_str     0x0000000000000000      0x594 /home/evln/proj/build-ia16.202501/prefix/bin/../lib/gcc/ia16-elf/6.3.0/../../../../ia16-elf/lib/regparmcall/libc.a(lib_a-strrchr.o)
 .comment       0x0000000000000000       0x12 /home/evln/proj/build-ia16.202501/prefix/bin/../lib/gcc/ia16-elf/6.3.0/../../../../ia16-elf/lib/regparmcall/libc.a(lib_a-strrchr.o)
 .debug_frame   0x0000000000000000       0x2c /home/evln/proj/build-ia16.202501/prefix/bin/../lib/gcc/ia16-elf/6.3.0/../../../../ia16-elf/lib/regparmcall/libc.a(lib_a-strspn.o)
 .debug_info    0x0000000000000000      0x8ae /home/evln/proj/build-ia16.202501/prefix/bin/../lib/gcc/ia16-elf/6.3.0/../../../../ia16-elf/lib/regparmcall/libc.a(lib_a-strspn.o)
 .debug_abbrev  0x0000000000000000      0x168 /home/evln/proj/build-ia16.202501/prefix/bin/../lib/gcc/ia16-elf/6.3.0/../../../../ia16-elf/lib/regparmcall/libc.a(lib_a-strspn.o)
 .debug_loc     0x0000000000000000       0x80 /home/evln/proj/build-ia16.202501/prefix/bin/../lib/gcc/ia16-elf/6.3.0/../../../../ia16-elf/lib/regparmcall/libc.a(lib_a-strspn.o)
 .debug_aranges
                0x0000000000000000       0x14 /home/evln/proj/build-ia16.202501/prefix/bin/../lib/gcc/ia16-elf/6.3.0/../../../../ia16-elf/lib/regparmcall/libc.a(lib_a-strspn.o)
 .debug_line    0x0000000000000000      0x174 /home/evln/proj/build-ia16.202501/prefix/bin/../lib/gcc/ia16-elf/6.3.0/../../../../ia16-elf/lib/regparmcall/libc.a(lib_a-strspn.o)
 .debug_str     0x0000000000000000      0x58d /home/evln/proj/build-ia16.202501/prefix/bin/../lib/gcc/ia16-elf/6.3.0/../../../../ia16-elf/lib/regparmcall/libc.a(lib_a-strspn.o)
 .comment       0x0000000000000000       0x12 /home/evln/proj/build-ia16.202501/prefix/bin/../lib/gcc/ia16-elf/6.3.0/../../../../ia16-elf/lib/regparmcall/libc.a(lib_a-strspn.o)
 .debug_frame   0x0000000000000000       0x30 /home/evln/proj/build-ia16.202501/prefix/bin/../lib/gcc/ia16-elf/6.3.0/../../../../ia16-elf/lib/regparmcall/libc.a(lib_a-strtok.o)
 .debug_info    0x0000000000000000      0x926 /home/evln/proj/build-ia16.202501/prefix/bin/../lib/gcc/ia16-elf/6.3.0/../../../../ia16-elf/lib/regparmcall/libc.a(lib_a-strtok.o)
 .debug_abbrev  0x0000000000000000      0x1d4 /home/evln/proj/build-ia16.202501/prefix/bin/../lib/gcc/ia16-elf/6.3.0/../../../../ia16-elf/lib/regparmcall/libc.a(lib_a-strtok.o)
 .debug_loc     0x0000000000000000       0x59 /home/evln/proj/build-ia16.202501/prefix/bin/../lib/gcc/ia16-elf/6.3.0/../../../../ia16-elf/lib/regparmcall/libc.a(lib_a-strtok.o)
 .debug_aranges
                0x0000000000000000       0x14 /home/evln/proj/build-ia16.202501/prefix/bin/../lib/gcc/ia16-elf/6.3.0/../../../../ia16-elf/lib/regparmcall/libc.a(lib_a-strtok.o)
 .debug_line    0x0000000000000000      0x168 /home/evln/proj/build-ia16.202501/prefix/bin/../lib/gcc/ia16-elf/6.3.0/../../../../ia16-elf/lib/regparmcall/libc.a(lib_a-strtok.o)
 .debug_str     0x0000000000000000      0x5a4 /home/evln/proj/build-ia16.202501/prefix/bin/../lib/gcc/ia16-elf/6.3.0/../../../../ia16-elf/lib/regparmcall/libc.a(lib_a-strtok.o)
 .comment       0x0000000000000000       0x12 /home/evln/proj/build-ia16.202501/prefix/bin/../lib/gcc/ia16-elf/6.3.0/../../../../ia16-elf/lib/regparmcall/libc.a(lib_a-strtok.o)
 .debug_frame   0x0000000000000000       0x78 /home/evln/proj/build-ia16.202501/prefix/bin/../lib/gcc/ia16-elf/6.3.0/../../../../ia16-elf/lib/regparmcall/libc.a(lib_a-strtok_r.o)
 .debug_info    0x0000000000000000      0x964 /home/evln/proj/build-ia16.202501/prefix/bin/../lib/gcc/ia16-elf/6.3.0/../../../../ia16-elf/lib/regparmcall/libc.a(lib_a-strtok_r.o)
 .debug_abbrev  0x0000000000000000      0x1d8 /home/evln/proj/build-ia16.202501/prefix/bin/../lib/gcc/ia16-elf/6.3.0/../../../../ia16-elf/lib/regparmcall/libc.a(lib_a-strtok_r.o)
 .debug_loc     0x0000000000000000      0x197 /home/evln/proj/build-ia16.202501/prefix/bin/../lib/gcc/ia16-elf/6.3.0/../../../../ia16-elf/lib/regparmcall/libc.a(lib_a-strtok_r.o)
 .debug_aranges
                0x0000000000000000       0x14 /home/evln/proj/build-ia16.202501/prefix/bin/../lib/gcc/ia16-elf/6.3.0/../../../../ia16-elf/lib/regparmcall/libc.a(lib_a-strtok_r.o)
 .debug_line    0x0000000000000000      0x194 /home/evln/proj/build-ia16.202501/prefix/bin/../lib/gcc/ia16-elf/6.3.0/../../../../ia16-elf/lib/regparmcall/libc.a(lib_a-strtok_r.o)
 .debug_str     0x0000000000000000      0x5bf /home/evln/proj/build-ia16.202501/prefix/bin/../lib/gcc/ia16-elf/6.3.0/../../../../ia16-elf/lib/regparmcall/libc.a(lib_a-strtok_r.o)
 .comment       0x0000000000000000       0x12 /home/evln/proj/build-ia16.202501/prefix/bin/../lib/gcc/ia16-elf/6.3.0/../../../../ia16-elf/lib/regparmcall/libc.a(lib_a-strtok_r.o)
 .debug_frame   0x0000000000000000       0x4c /home/evln/proj/build-ia16.202501/prefix/bin/../lib/gcc/ia16-elf/6.3.0/../../../../ia16-elf/lib/regparmcall/libc.a(lib_a-strtol.o)
 .debug_info    0x0000000000000000      0x9fd /home/evln/proj/build-ia16.202501/prefix/bin/../lib/gcc/ia16-elf/6.3.0/../../../../ia16-elf/lib/regparmcall/libc.a(lib_a-strtol.o)
 .debug_abbrev  0x0000000000000000      0x1c9 /home/evln/proj/build-ia16.202501/prefix/bin/../lib/gcc/ia16-elf/6.3.0/../../../../ia16-elf/lib/regparmcall/libc.a(lib_a-strtol.o)
 .debug_loc     0x0000000000000000      0x3ba /home/evln/proj/build-ia16.202501/prefix/bin/../lib/gcc/ia16-elf/6.3.0/../../../../ia16-elf/lib/regparmcall/libc.a(lib_a-strtol.o)
 .debug_aranges
                0x0000000000000000       0x14 /home/evln/proj/build-ia16.202501/prefix/bin/../lib/gcc/ia16-elf/6.3.0/../../../../ia16-elf/lib/regparmcall/libc.a(lib_a-strtol.o)
 .debug_line    0x0000000000000000      0x2c4 /home/evln/proj/build-ia16.202501/prefix/bin/../lib/gcc/ia16-elf/6.3.0/../../../../ia16-elf/lib/regparmcall/libc.a(lib_a-strtol.o)
 .debug_str     0x0000000000000000      0x5f7 /home/evln/proj/build-ia16.202501/prefix/bin/../lib/gcc/ia16-elf/6.3.0/../../../../ia16-elf/lib/regparmcall/libc.a(lib_a-strtol.o)
 .comment       0x0000000000000000       0x12 /home/evln/proj/build-ia16.202501/prefix/bin/../lib/gcc/ia16-elf/6.3.0/../../../../ia16-elf/lib/regparmcall/libc.a(lib_a-strtol.o)
 .debug_frame   0x0000000000000000       0x1e /home/evln/proj/build-ia16.202501/prefix/bin/../lib/gcc/ia16-elf/6.3.0/../../../../ia16-elf/lib/regparmcall/libc.a(lib_a-sysisatty.o)
 .debug_info    0x0000000000000000      0x8e3 /home/evln/proj/build-ia16.202501/prefix/bin/../lib/gcc/ia16-elf/6.3.0/../../../../ia16-elf/lib/regparmcall/libc.a(lib_a-sysisatty.o)
 .debug_abbrev  0x0000000000000000      0x188 /home/evln/proj/build-ia16.202501/prefix/bin/../lib/gcc/ia16-elf/6.3.0/../../../../ia16-elf/lib/regparmcall/libc.a(lib_a-sysisatty.o)
 .debug_loc     0x0000000000000000       0x26 /home/evln/proj/build-ia16.202501/prefix/bin/../lib/gcc/ia16-elf/6.3.0/../../../../ia16-elf/lib/regparmcall/libc.a(lib_a-sysisatty.o)
 .debug_aranges
                0x0000000000000000       0x14 /home/evln/proj/build-ia16.202501/prefix/bin/../lib/gcc/ia16-elf/6.3.0/../../../../ia16-elf/lib/regparmcall/libc.a(lib_a-sysisatty.o)
 .debug_line    0x0000000000000000      0x169 /home/evln/proj/build-ia16.202501/prefix/bin/../lib/gcc/ia16-elf/6.3.0/../../../../ia16-elf/lib/regparmcall/libc.a(lib_a-sysisatty.o)
 .debug_str     0x0000000000000000      0x5c4 /home/evln/proj/build-ia16.202501/prefix/bin/../lib/gcc/ia16-elf/6.3.0/../../../../ia16-elf/lib/regparmcall/libc.a(lib_a-sysisatty.o)
 .comment       0x0000000000000000       0x12 /home/evln/proj/build-ia16.202501/prefix/bin/../lib/gcc/ia16-elf/6.3.0/../../../../ia16-elf/lib/regparmcall/libc.a(lib_a-sysisatty.o)
 .debug_frame   0x0000000000000000       0x2c /home/evln/proj/build-ia16.202501/prefix/bin/../lib/gcc/ia16-elf/6.3.0/../../../../ia16-elf/lib/regparmcall/libc.a(lib_a-syslseek.o)
 .debug_info    0x0000000000000000      0x907 /home/evln/proj/build-ia16.202501/prefix/bin/../lib/gcc/ia16-elf/6.3.0/../../../../ia16-elf/lib/regparmcall/libc.a(lib_a-syslseek.o)
 .debug_abbrev  0x0000000000000000      0x1a1 /home/evln/proj/build-ia16.202501/prefix/bin/../lib/gcc/ia16-elf/6.3.0/../../../../ia16-elf/lib/regparmcall/libc.a(lib_a-syslseek.o)
 .debug_loc     0x0000000000000000       0x26 /home/evln/proj/build-ia16.202501/prefix/bin/../lib/gcc/ia16-elf/6.3.0/../../../../ia16-elf/lib/regparmcall/libc.a(lib_a-syslseek.o)
 .debug_aranges
                0x0000000000000000       0x14 /home/evln/proj/build-ia16.202501/prefix/bin/../lib/gcc/ia16-elf/6.3.0/../../../../ia16-elf/lib/regparmcall/libc.a(lib_a-syslseek.o)
 .debug_line    0x0000000000000000      0x176 /home/evln/proj/build-ia16.202501/prefix/bin/../lib/gcc/ia16-elf/6.3.0/../../../../ia16-elf/lib/regparmcall/libc.a(lib_a-syslseek.o)
 .debug_str     0x0000000000000000      0x5ce /home/evln/proj/build-ia16.202501/prefix/bin/../lib/gcc/ia16-elf/6.3.0/../../../../ia16-elf/lib/regparmcall/libc.a(lib_a-syslseek.o)
 .comment       0x0000000000000000       0x12 /home/evln/proj/build-ia16.202501/prefix/bin/../lib/gcc/ia16-elf/6.3.0/../../../../ia16-elf/lib/regparmcall/libc.a(lib_a-syslseek.o)
 .debug_frame   0x0000000000000000       0x1e /home/evln/proj/build-ia16.202501/prefix/bin/../lib/gcc/ia16-elf/6.3.0/../../../../ia16-elf/lib/regparmcall/libc.a(lib_a-sysunlink.o)
 .debug_info    0x0000000000000000      0x8e4 /home/evln/proj/build-ia16.202501/prefix/bin/../lib/gcc/ia16-elf/6.3.0/../../../../ia16-elf/lib/regparmcall/libc.a(lib_a-sysunlink.o)
 .debug_abbrev  0x0000000000000000      0x188 /home/evln/proj/build-ia16.202501/prefix/bin/../lib/gcc/ia16-elf/6.3.0/../../../../ia16-elf/lib/regparmcall/libc.a(lib_a-sysunlink.o)
 .debug_loc     0x0000000000000000       0x26 /home/evln/proj/build-ia16.202501/prefix/bin/../lib/gcc/ia16-elf/6.3.0/../../../../ia16-elf/lib/regparmcall/libc.a(lib_a-sysunlink.o)
 .debug_aranges
                0x0000000000000000       0x14 /home/evln/proj/build-ia16.202501/prefix/bin/../lib/gcc/ia16-elf/6.3.0/../../../../ia16-elf/lib/regparmcall/libc.a(lib_a-sysunlink.o)
 .debug_line    0x0000000000000000      0x169 /home/evln/proj/build-ia16.202501/prefix/bin/../lib/gcc/ia16-elf/6.3.0/../../../../ia16-elf/lib/regparmcall/libc.a(lib_a-sysunlink.o)
 .debug_str     0x0000000000000000      0x5c9 /home/evln/proj/build-ia16.202501/prefix/bin/../lib/gcc/ia16-elf/6.3.0/../../../../ia16-elf/lib/regparmcall/libc.a(lib_a-sysunlink.o)
 .comment       0x0000000000000000       0x12 /home/evln/proj/build-ia16.202501/prefix/bin/../lib/gcc/ia16-elf/6.3.0/../../../../ia16-elf/lib/regparmcall/libc.a(lib_a-sysunlink.o)
 .debug_frame   0x0000000000000000       0x2c /home/evln/proj/build-ia16.202501/prefix/bin/../lib/gcc/ia16-elf/6.3.0/../../../../ia16-elf/lib/regparmcall/libc.a(lib_a-syswrite.o)
 .debug_info    0x0000000000000000      0x91f /home/evln/proj/build-ia16.202501/prefix/bin/../lib/gcc/ia16-elf/6.3.0/../../../../ia16-elf/lib/regparmcall/libc.a(lib_a-syswrite.o)
 .debug_abbrev  0x0000000000000000      0x18a /home/evln/proj/build-ia16.202501/prefix/bin/../lib/gcc/ia16-elf/6.3.0/../../../../ia16-elf/lib/regparmcall/libc.a(lib_a-syswrite.o)
 .debug_loc     0x0000000000000000       0x6e /home/evln/proj/build-ia16.202501/prefix/bin/../lib/gcc/ia16-elf/6.3.0/../../../../ia16-elf/lib/regparmcall/libc.a(lib_a-syswrite.o)
 .debug_aranges
                0x0000000000000000       0x14 /home/evln/proj/build-ia16.202501/prefix/bin/../lib/gcc/ia16-elf/6.3.0/../../../../ia16-elf/lib/regparmcall/libc.a(lib_a-syswrite.o)
 .debug_line    0x0000000000000000      0x16b /home/evln/proj/build-ia16.202501/prefix/bin/../lib/gcc/ia16-elf/6.3.0/../../../../ia16-elf/lib/regparmcall/libc.a(lib_a-syswrite.o)
 .debug_str     0x0000000000000000      0x5c8 /home/evln/proj/build-ia16.202501/prefix/bin/../lib/gcc/ia16-elf/6.3.0/../../../../ia16-elf/lib/regparmcall/libc.a(lib_a-syswrite.o)
 .comment       0x0000000000000000       0x12 /home/evln/proj/build-ia16.202501/prefix/bin/../lib/gcc/ia16-elf/6.3.0/../../../../ia16-elf/lib/regparmcall/libc.a(lib_a-syswrite.o)
 .debug_frame   0x0000000000000000       0x26 /home/evln/proj/build-ia16.202501/prefix/bin/../lib/gcc/ia16-elf/6.3.0/../../../../ia16-elf/lib/regparmcall/libc.a(lib_a-toupper.o)
 .debug_info    0x0000000000000000       0xc6 /home/evln/proj/build-ia16.202501/prefix/bin/../lib/gcc/ia16-elf/6.3.0/../../../../ia16-elf/lib/regparmcall/libc.a(lib_a-toupper.o)
 .debug_abbrev  0x0000000000000000       0x82 /home/evln/proj/build-ia16.202501/prefix/bin/../lib/gcc/ia16-elf/6.3.0/../../../../ia16-elf/lib/regparmcall/libc.a(lib_a-toupper.o)
 .debug_loc     0x0000000000000000       0x1c /home/evln/proj/build-ia16.202501/prefix/bin/../lib/gcc/ia16-elf/6.3.0/../../../../ia16-elf/lib/regparmcall/libc.a(lib_a-toupper.o)
 .debug_aranges
                0x0000000000000000       0x14 /home/evln/proj/build-ia16.202501/prefix/bin/../lib/gcc/ia16-elf/6.3.0/../../../../ia16-elf/lib/regparmcall/libc.a(lib_a-toupper.o)
 .debug_line    0x0000000000000000       0xbf /home/evln/proj/build-ia16.202501/prefix/bin/../lib/gcc/ia16-elf/6.3.0/../../../../ia16-elf/lib/regparmcall/libc.a(lib_a-toupper.o)
 .debug_str     0x0000000000000000      0x1a2 /home/evln/proj/build-ia16.202501/prefix/bin/../lib/gcc/ia16-elf/6.3.0/../../../../ia16-elf/lib/regparmcall/libc.a(lib_a-toupper.o)
 .comment       0x0000000000000000       0x12 /home/evln/proj/build-ia16.202501/prefix/bin/../lib/gcc/ia16-elf/6.3.0/../../../../ia16-elf/lib/regparmcall/libc.a(lib_a-toupper.o)
 .debug_frame   0x0000000000000000       0x32 /home/evln/proj/build-ia16.202501/prefix/bin/../lib/gcc/ia16-elf/6.3.0/../../../../ia16-elf/lib/regparmcall/libc.a(lib_a-__atexit.o)
 .debug_info    0x0000000000000000      0x96a /home/evln/proj/build-ia16.202501/prefix/bin/../lib/gcc/ia16-elf/6.3.0/../../../../ia16-elf/lib/regparmcall/libc.a(lib_a-__atexit.o)
 .debug_abbrev  0x0000000000000000      0x202 /home/evln/proj/build-ia16.202501/prefix/bin/../lib/gcc/ia16-elf/6.3.0/../../../../ia16-elf/lib/regparmcall/libc.a(lib_a-__atexit.o)
 .debug_loc     0x0000000000000000       0xf8 /home/evln/proj/build-ia16.202501/prefix/bin/../lib/gcc/ia16-elf/6.3.0/../../../../ia16-elf/lib/regparmcall/libc.a(lib_a-__atexit.o)
 .debug_aranges
                0x0000000000000000       0x14 /home/evln/proj/build-ia16.202501/prefix/bin/../lib/gcc/ia16-elf/6.3.0/../../../../ia16-elf/lib/regparmcall/libc.a(lib_a-__atexit.o)
 .debug_line    0x0000000000000000      0x1fa /home/evln/proj/build-ia16.202501/prefix/bin/../lib/gcc/ia16-elf/6.3.0/../../../../ia16-elf/lib/regparmcall/libc.a(lib_a-__atexit.o)
 .debug_str     0x0000000000000000      0x60b /home/evln/proj/build-ia16.202501/prefix/bin/../lib/gcc/ia16-elf/6.3.0/../../../../ia16-elf/lib/regparmcall/libc.a(lib_a-__atexit.o)
 .comment       0x0000000000000000       0x12 /home/evln/proj/build-ia16.202501/prefix/bin/../lib/gcc/ia16-elf/6.3.0/../../../../ia16-elf/lib/regparmcall/libc.a(lib_a-__atexit.o)
 .debug_frame   0x0000000000000000       0x32 /home/evln/proj/build-ia16.202501/prefix/bin/../lib/gcc/ia16-elf/6.3.0/../../../../ia16-elf/lib/regparmcall/libc.a(lib_a-__call_atexit.o)
 .debug_info    0x0000000000000000      0x980 /home/evln/proj/build-ia16.202501/prefix/bin/../lib/gcc/ia16-elf/6.3.0/../../../../ia16-elf/lib/regparmcall/libc.a(lib_a-__call_atexit.o)
 .debug_abbrev  0x0000000000000000      0x1f2 /home/evln/proj/build-ia16.202501/prefix/bin/../lib/gcc/ia16-elf/6.3.0/../../../../ia16-elf/lib/regparmcall/libc.a(lib_a-__call_atexit.o)
 .debug_loc     0x0000000000000000      0x16e /home/evln/proj/build-ia16.202501/prefix/bin/../lib/gcc/ia16-elf/6.3.0/../../../../ia16-elf/lib/regparmcall/libc.a(lib_a-__call_atexit.o)
 .debug_aranges
                0x0000000000000000       0x14 /home/evln/proj/build-ia16.202501/prefix/bin/../lib/gcc/ia16-elf/6.3.0/../../../../ia16-elf/lib/regparmcall/libc.a(lib_a-__call_atexit.o)
 .debug_ranges  0x0000000000000000        0xc /home/evln/proj/build-ia16.202501/prefix/bin/../lib/gcc/ia16-elf/6.3.0/../../../../ia16-elf/lib/regparmcall/libc.a(lib_a-__call_atexit.o)
 .debug_line    0x0000000000000000      0x22b /home/evln/proj/build-ia16.202501/prefix/bin/../lib/gcc/ia16-elf/6.3.0/../../../../ia16-elf/lib/regparmcall/libc.a(lib_a-__call_atexit.o)
 .debug_str     0x0000000000000000      0x5d8 /home/evln/proj/build-ia16.202501/prefix/bin/../lib/gcc/ia16-elf/6.3.0/../../../../ia16-elf/lib/regparmcall/libc.a(lib_a-__call_atexit.o)
 .comment       0x0000000000000000       0x12 /home/evln/proj/build-ia16.202501/prefix/bin/../lib/gcc/ia16-elf/6.3.0/../../../../ia16-elf/lib/regparmcall/libc.a(lib_a-__call_atexit.o)
 .debug_frame   0x0000000000000000       0x32 /home/evln/proj/build-ia16.202501/prefix/bin/../lib/gcc/ia16-elf/6.3.0/../../../../ia16-elf/lib/regparmcall/libc.a(lib_a-nano-reallocr.o)
 .debug_info    0x0000000000000000      0xb2a /home/evln/proj/build-ia16.202501/prefix/bin/../lib/gcc/ia16-elf/6.3.0/../../../../ia16-elf/lib/regparmcall/libc.a(lib_a-nano-reallocr.o)
 .debug_abbrev  0x0000000000000000      0x1fd /home/evln/proj/build-ia16.202501/prefix/bin/../lib/gcc/ia16-elf/6.3.0/../../../../ia16-elf/lib/regparmcall/libc.a(lib_a-nano-reallocr.o)
 .debug_loc     0x0000000000000000      0x121 /home/evln/proj/build-ia16.202501/prefix/bin/../lib/gcc/ia16-elf/6.3.0/../../../../ia16-elf/lib/regparmcall/libc.a(lib_a-nano-reallocr.o)
 .debug_aranges
                0x0000000000000000       0x14 /home/evln/proj/build-ia16.202501/prefix/bin/../lib/gcc/ia16-elf/6.3.0/../../../../ia16-elf/lib/regparmcall/libc.a(lib_a-nano-reallocr.o)
 .debug_line    0x0000000000000000      0x263 /home/evln/proj/build-ia16.202501/prefix/bin/../lib/gcc/ia16-elf/6.3.0/../../../../ia16-elf/lib/regparmcall/libc.a(lib_a-nano-reallocr.o)
 .debug_str     0x0000000000000000      0x701 /home/evln/proj/build-ia16.202501/prefix/bin/../lib/gcc/ia16-elf/6.3.0/../../../../ia16-elf/lib/regparmcall/libc.a(lib_a-nano-reallocr.o)
 .comment       0x0000000000000000       0x12 /home/evln/proj/build-ia16.202501/prefix/bin/../lib/gcc/ia16-elf/6.3.0/../../../../ia16-elf/lib/regparmcall/libc.a(lib_a-nano-reallocr.o)
 .debug_frame   0x0000000000000000       0x26 /home/evln/proj/build-ia16.202501/prefix/bin/../lib/gcc/ia16-elf/6.3.0/../../../../ia16-elf/lib/regparmcall/libc.a(lib_a-nano-msizer.o)
 .debug_info    0x0000000000000000      0xa38 /home/evln/proj/build-ia16.202501/prefix/bin/../lib/gcc/ia16-elf/6.3.0/../../../../ia16-elf/lib/regparmcall/libc.a(lib_a-nano-msizer.o)
 .debug_abbrev  0x0000000000000000      0x18d /home/evln/proj/build-ia16.202501/prefix/bin/../lib/gcc/ia16-elf/6.3.0/../../../../ia16-elf/lib/regparmcall/libc.a(lib_a-nano-msizer.o)
 .debug_loc     0x0000000000000000       0x79 /home/evln/proj/build-ia16.202501/prefix/bin/../lib/gcc/ia16-elf/6.3.0/../../../../ia16-elf/lib/regparmcall/libc.a(lib_a-nano-msizer.o)
 .debug_aranges
                0x0000000000000000       0x14 /home/evln/proj/build-ia16.202501/prefix/bin/../lib/gcc/ia16-elf/6.3.0/../../../../ia16-elf/lib/regparmcall/libc.a(lib_a-nano-msizer.o)
 .debug_line    0x0000000000000000      0x237 /home/evln/proj/build-ia16.202501/prefix/bin/../lib/gcc/ia16-elf/6.3.0/../../../../ia16-elf/lib/regparmcall/libc.a(lib_a-nano-msizer.o)
 .debug_str     0x0000000000000000      0x6d7 /home/evln/proj/build-ia16.202501/prefix/bin/../lib/gcc/ia16-elf/6.3.0/../../../../ia16-elf/lib/regparmcall/libc.a(lib_a-nano-msizer.o)
 .comment       0x0000000000000000       0x12 /home/evln/proj/build-ia16.202501/prefix/bin/../lib/gcc/ia16-elf/6.3.0/../../../../ia16-elf/lib/regparmcall/libc.a(lib_a-nano-msizer.o)
 .debug_frame   0x0000000000000000       0x30 /home/evln/proj/build-ia16.202501/prefix/bin/../lib/gcc/ia16-elf/6.3.0/../../../../ia16-elf/lib/regparmcall/libdos-s.a(dos-sbrkr.o)
 .debug_info    0x0000000000000000      0x970 /home/evln/proj/build-ia16.202501/prefix/bin/../lib/gcc/ia16-elf/6.3.0/../../../../ia16-elf/lib/regparmcall/libdos-s.a(dos-sbrkr.o)
 .debug_abbrev  0x0000000000000000      0x1a2 /home/evln/proj/build-ia16.202501/prefix/bin/../lib/gcc/ia16-elf/6.3.0/../../../../ia16-elf/lib/regparmcall/libdos-s.a(dos-sbrkr.o)
 .debug_loc     0x0000000000000000       0x64 /home/evln/proj/build-ia16.202501/prefix/bin/../lib/gcc/ia16-elf/6.3.0/../../../../ia16-elf/lib/regparmcall/libdos-s.a(dos-sbrkr.o)
 .debug_aranges
                0x0000000000000000       0x14 /home/evln/proj/build-ia16.202501/prefix/bin/../lib/gcc/ia16-elf/6.3.0/../../../../ia16-elf/lib/regparmcall/libdos-s.a(dos-sbrkr.o)
 .debug_line    0x0000000000000000      0x22d /home/evln/proj/build-ia16.202501/prefix/bin/../lib/gcc/ia16-elf/6.3.0/../../../../ia16-elf/lib/regparmcall/libdos-s.a(dos-sbrkr.o)
 .debug_str     0x0000000000000000      0x613 /home/evln/proj/build-ia16.202501/prefix/bin/../lib/gcc/ia16-elf/6.3.0/../../../../ia16-elf/lib/regparmcall/libdos-s.a(dos-sbrkr.o)
 .comment       0x0000000000000000       0x12 /home/evln/proj/build-ia16.202501/prefix/bin/../lib/gcc/ia16-elf/6.3.0/../../../../ia16-elf/lib/regparmcall/libdos-s.a(dos-sbrkr.o)
 .debug_info    0x0000000000000000      0x8cd /home/evln/proj/build-ia16.202501/prefix/bin/../lib/gcc/ia16-elf/6.3.0/../../../../ia16-elf/lib/regparmcall/libdos-s.a(dos-heaplen.o)
 .debug_abbrev  0x0000000000000000      0x144 /home/evln/proj/build-ia16.202501/prefix/bin/../lib/gcc/ia16-elf/6.3.0/../../../../ia16-elf/lib/regparmcall/libdos-s.a(dos-heaplen.o)
 .debug_aranges
                0x0000000000000000       0x10 /home/evln/proj/build-ia16.202501/prefix/bin/../lib/gcc/ia16-elf/6.3.0/../../../../ia16-elf/lib/regparmcall/libdos-s.a(dos-heaplen.o)
 .debug_line    0x0000000000000000      0x1ab /home/evln/proj/build-ia16.202501/prefix/bin/../lib/gcc/ia16-elf/6.3.0/../../../../ia16-elf/lib/regparmcall/libdos-s.a(dos-heaplen.o)
 .debug_str     0x0000000000000000      0x5bb /home/evln/proj/build-ia16.202501/prefix/bin/../lib/gcc/ia16-elf/6.3.0/../../../../ia16-elf/lib/regparmcall/libdos-s.a(dos-heaplen.o)
 .comment       0x0000000000000000       0x12 /home/evln/proj/build-ia16.202501/prefix/bin/../lib/gcc/ia16-elf/6.3.0/../../../../ia16-elf/lib/regparmcall/libdos-s.a(dos-heaplen.o)
 .debug_frame   0x0000000000000000       0x4c /home/evln/proj/build-ia16.202501/prefix/bin/../lib/gcc/ia16-elf/6.3.0/../../../../ia16-elf/lib/regparmcall/libc.a(lib_a-abort.o)
 .debug_info    0x0000000000000000      0x334 /home/evln/proj/build-ia16.202501/prefix/bin/../lib/gcc/ia16-elf/6.3.0/../../../../ia16-elf/lib/regparmcall/libc.a(lib_a-abort.o)
 .debug_abbrev  0x0000000000000000      0x16a /home/evln/proj/build-ia16.202501/prefix/bin/../lib/gcc/ia16-elf/6.3.0/../../../../ia16-elf/lib/regparmcall/libc.a(lib_a-abort.o)
 .debug_loc     0x0000000000000000      0x10f /home/evln/proj/build-ia16.202501/prefix/bin/../lib/gcc/ia16-elf/6.3.0/../../../../ia16-elf/lib/regparmcall/libc.a(lib_a-abort.o)
 .debug_aranges
                0x0000000000000000       0x14 /home/evln/proj/build-ia16.202501/prefix/bin/../lib/gcc/ia16-elf/6.3.0/../../../../ia16-elf/lib/regparmcall/libc.a(lib_a-abort.o)
 .debug_ranges  0x0000000000000000        0xc /home/evln/proj/build-ia16.202501/prefix/bin/../lib/gcc/ia16-elf/6.3.0/../../../../ia16-elf/lib/regparmcall/libc.a(lib_a-abort.o)
 .debug_line    0x0000000000000000       0xdb /home/evln/proj/build-ia16.202501/prefix/bin/../lib/gcc/ia16-elf/6.3.0/../../../../ia16-elf/lib/regparmcall/libc.a(lib_a-abort.o)
 .debug_str     0x0000000000000000      0x225 /home/evln/proj/build-ia16.202501/prefix/bin/../lib/gcc/ia16-elf/6.3.0/../../../../ia16-elf/lib/regparmcall/libc.a(lib_a-abort.o)
 .comment       0x0000000000000000       0x12 /home/evln/proj/build-ia16.202501/prefix/bin/../lib/gcc/ia16-elf/6.3.0/../../../../ia16-elf/lib/regparmcall/libc.a(lib_a-abort.o)

Memory Configuration

Name             Origin             Length             Attributes
bseglma          0x0000000000000000 0x00000000000a0000 xw
hdrvma           0x0000000000000000 0x0000000000040020 xw
csegvma          0x0000000000000020 0x0000000000010000 xw
ft00segvma       0x0000000000000000 0x0000000000010000 xw
ft01segvma       0x0000000000000000 0x0000000000010000 xw
ft02segvma       0x0000000000000000 0x0000000000010000 xw
ft03segvma       0x0000000000000000 0x0000000000010000 xw
ft04segvma       0x0000000000000000 0x0000000000010000 xw
ft05segvma       0x0000000000000000 0x0000000000010000 xw
ft06segvma       0x0000000000000000 0x0000000000010000 xw
ft07segvma       0x0000000000000000 0x0000000000010000 xw
ft10segvma       0x0000000000000000 0x0000000000010000 xw
ft11segvma       0x0000000000000000 0x0000000000010000 xw
ft12segvma       0x0000000000000000 0x0000000000010000 xw
ft13segvma       0x0000000000000000 0x0000000000010000 xw
ft14segvma       0x0000000000000000 0x0000000000010000 xw
ft15segvma       0x0000000000000000 0x0000000000010000 xw
ft16segvma       0x0000000000000000 0x0000000000010000 xw
ft17segvma       0x0000000000000000 0x0000000000010000 xw
ft20segvma       0x0000000000000000 0x0000000000010000 xw
ft21segvma       0x0000000000000000 0x0000000000010000 xw
ft22segvma       0x0000000000000000 0x0000000000010000 xw
ft23segvma       0x0000000000000000 0x0000000000010000 xw
ft24segvma       0x0000000000000000 0x0000000000010000 xw
ft25segvma       0x0000000000000000 0x0000000000010000 xw
ft26segvma       0x0000000000000000 0x0000000000010000 xw
ft27segvma       0x0000000000000000 0x0000000000010000 xw
ft30segvma       0x0000000000000000 0x0000000000010000 xw
ft31segvma       0x0000000000000000 0x0000000000010000 xw
ft32segvma       0x0000000000000000 0x0000000000010000 xw
ft33segvma       0x0000000000000000 0x0000000000010000 xw
ft34segvma       0x0000000000000000 0x0000000000010000 xw
ft35segvma       0x0000000000000000 0x0000000000010000 xw
ft36segvma       0x0000000000000000 0x0000000000010000 xw
ft37segvma       0x0000000000000000 0x0000000000010000 xw
ft40segvma       0x0000000000000000 0x0000000000010000 xw
ft41segvma       0x0000000000000000 0x0000000000010000 xw
ft42segvma       0x0000000000000000 0x0000000000010000 xw
ft43segvma       0x0000000000000000 0x0000000000010000 xw
ft44segvma       0x0000000000000000 0x0000000000010000 xw
ft45segvma       0x0000000000000000 0x0000000000010000 xw
ft46segvma       0x0000000000000000 0x0000000000010000 xw
ft47segvma       0x0000000000000000 0x0000000000010000 xw
ft50segvma       0x0000000000000000 0x0000000000010000 xw
ft51segvma       0x0000000000000000 0x0000000000010000 xw
ft52segvma       0x0000000000000000 0x0000000000010000 xw
ft53segvma       0x0000000000000000 0x0000000000010000 xw
ft54segvma       0x0000000000000000 0x0000000000010000 xw
ft55segvma       0x0000000000000000 0x0000000000010000 xw
ft56segvma       0x0000000000000000 0x0000000000010000 xw
ft57segvma       0x0000000000000000 0x0000000000010000 xw
ft60segvma       0x0000000000000000 0x0000000000010000 xw
ft61segvma       0x0000000000000000 0x0000000000010000 xw
ft62segvma       0x0000000000000000 0x0000000000010000 xw
ft63segvma       0x0000000000000000 0x0000000000010000 xw
ft64segvma       0x0000000000000000 0x0000000000010000 xw
ft65segvma       0x0000000000000000 0x0000000000010000 xw
ft66segvma       0x0000000000000000 0x0000000000010000 xw
ft67segvma       0x0000000000000000 0x0000000000010000 xw
ft70segvma       0x0000000000000000 0x0000000000010000 xw
ft71segvma       0x0000000000000000 0x0000000000010000 xw
ft72segvma       0x0000000000000000 0x0000000000010000 xw
ft73segvma       0x0000000000000000 0x0000000000010000 xw
ft74segvma       0x0000000000000000 0x0000000000010000 xw
ft75segvma       0x0000000000000000 0x0000000000010000 xw
ft76segvma       0x0000000000000000 0x0000000000010000 xw
ft77segvma       0x0000000000000000 0x0000000000010000 xw
ftXXsegvma       0x0000000000000000 0x0000000000010000 xw
fr00segvma       0x0000000000000000 0x0000000000010000 xw
fr01segvma       0x0000000000000000 0x0000000000010000 xw
fr02segvma       0x0000000000000000 0x0000000000010000 xw
fr03segvma       0x0000000000000000 0x0000000000010000 xw
fr04segvma       0x0000000000000000 0x0000000000010000 xw
fr05segvma       0x0000000000000000 0x0000000000010000 xw
fr06segvma       0x0000000000000000 0x0000000000010000 xw
fr07segvma       0x0000000000000000 0x0000000000010000 xw
fr10segvma       0x0000000000000000 0x0000000000010000 xw
fr11segvma       0x0000000000000000 0x0000000000010000 xw
fr12segvma       0x0000000000000000 0x0000000000010000 xw
fr13segvma       0x0000000000000000 0x0000000000010000 xw
fr14segvma       0x0000000000000000 0x0000000000010000 xw
fr15segvma       0x0000000000000000 0x0000000000010000 xw
fr16segvma       0x0000000000000000 0x0000000000010000 xw
fr17segvma       0x0000000000000000 0x0000000000010000 xw
fr20segvma       0x0000000000000000 0x0000000000010000 xw
fr21segvma       0x0000000000000000 0x0000000000010000 xw
fr22segvma       0x0000000000000000 0x0000000000010000 xw
fr23segvma       0x0000000000000000 0x0000000000010000 xw
fr24segvma       0x0000000000000000 0x0000000000010000 xw
fr25segvma       0x0000000000000000 0x0000000000010000 xw
fr26segvma       0x0000000000000000 0x0000000000010000 xw
fr27segvma       0x0000000000000000 0x0000000000010000 xw
fr30segvma       0x0000000000000000 0x0000000000010000 xw
fr31segvma       0x0000000000000000 0x0000000000010000 xw
fr32segvma       0x0000000000000000 0x0000000000010000 xw
fr33segvma       0x0000000000000000 0x0000000000010000 xw
fr34segvma       0x0000000000000000 0x0000000000010000 xw
fr35segvma       0x0000000000000000 0x0000000000010000 xw
fr36segvma       0x0000000000000000 0x0000000000010000 xw
fr37segvma       0x0000000000000000 0x0000000000010000 xw
fr40segvma       0x0000000000000000 0x0000000000010000 xw
fr41segvma       0x0000000000000000 0x0000000000010000 xw
fr42segvma       0x0000000000000000 0x0000000000010000 xw
fr43segvma       0x0000000000000000 0x0000000000010000 xw
fr44segvma       0x0000000000000000 0x0000000000010000 xw
fr45segvma       0x0000000000000000 0x0000000000010000 xw
fr46segvma       0x0000000000000000 0x0000000000010000 xw
fr47segvma       0x0000000000000000 0x0000000000010000 xw
fr50segvma       0x0000000000000000 0x0000000000010000 xw
fr51segvma       0x0000000000000000 0x0000000000010000 xw
fr52segvma       0x0000000000000000 0x0000000000010000 xw
fr53segvma       0x0000000000000000 0x0000000000010000 xw
fr54segvma       0x0000000000000000 0x0000000000010000 xw
fr55segvma       0x0000000000000000 0x0000000000010000 xw
fr56segvma       0x0000000000000000 0x0000000000010000 xw
fr57segvma       0x0000000000000000 0x0000000000010000 xw
fr60segvma       0x0000000000000000 0x0000000000010000 xw
fr61segvma       0x0000000000000000 0x0000000000010000 xw
fr62segvma       0x0000000000000000 0x0000000000010000 xw
fr63segvma       0x0000000000000000 0x0000000000010000 xw
fr64segvma       0x0000000000000000 0x0000000000010000 xw
fr65segvma       0x0000000000000000 0x0000000000010000 xw
fr66segvma       0x0000000000000000 0x0000000000010000 xw
fr67segvma       0x0000000000000000 0x0000000000010000 xw
fr70segvma       0x0000000000000000 0x0000000000010000 xw
fr71segvma       0x0000000000000000 0x0000000000010000 xw
fr72segvma       0x0000000000000000 0x0000000000010000 xw
fr73segvma       0x0000000000000000 0x0000000000010000 xw
fr74segvma       0x0000000000000000 0x0000000000010000 xw
fr75segvma       0x0000000000000000 0x0000000000010000 xw
fr76segvma       0x0000000000000000 0x0000000000010000 xw
fr77segvma       0x0000000000000000 0x0000000000010000 xw
frXXsegvma       0x0000000000000000 0x0000000000010000 xw
fd00segvma       0x0000000000000000 0x0000000000010000 xw
fd01segvma       0x0000000000000000 0x0000000000010000 xw
fd02segvma       0x0000000000000000 0x0000000000010000 xw
fd03segvma       0x0000000000000000 0x0000000000010000 xw
fd04segvma       0x0000000000000000 0x0000000000010000 xw
fd05segvma       0x0000000000000000 0x0000000000010000 xw
fd06segvma       0x0000000000000000 0x0000000000010000 xw
fd07segvma       0x0000000000000000 0x0000000000010000 xw
fd10segvma       0x0000000000000000 0x0000000000010000 xw
fd11segvma       0x0000000000000000 0x0000000000010000 xw
fd12segvma       0x0000000000000000 0x0000000000010000 xw
fd13segvma       0x0000000000000000 0x0000000000010000 xw
fd14segvma       0x0000000000000000 0x0000000000010000 xw
fd15segvma       0x0000000000000000 0x0000000000010000 xw
fd16segvma       0x0000000000000000 0x0000000000010000 xw
fd17segvma       0x0000000000000000 0x0000000000010000 xw
fd20segvma       0x0000000000000000 0x0000000000010000 xw
fd21segvma       0x0000000000000000 0x0000000000010000 xw
fd22segvma       0x0000000000000000 0x0000000000010000 xw
fd23segvma       0x0000000000000000 0x0000000000010000 xw
fd24segvma       0x0000000000000000 0x0000000000010000 xw
fd25segvma       0x0000000000000000 0x0000000000010000 xw
fd26segvma       0x0000000000000000 0x0000000000010000 xw
fd27segvma       0x0000000000000000 0x0000000000010000 xw
fd30segvma       0x0000000000000000 0x0000000000010000 xw
fd31segvma       0x0000000000000000 0x0000000000010000 xw
fd32segvma       0x0000000000000000 0x0000000000010000 xw
fd33segvma       0x0000000000000000 0x0000000000010000 xw
fd34segvma       0x0000000000000000 0x0000000000010000 xw
fd35segvma       0x0000000000000000 0x0000000000010000 xw
fd36segvma       0x0000000000000000 0x0000000000010000 xw
fd37segvma       0x0000000000000000 0x0000000000010000 xw
fd40segvma       0x0000000000000000 0x0000000000010000 xw
fd41segvma       0x0000000000000000 0x0000000000010000 xw
fd42segvma       0x0000000000000000 0x0000000000010000 xw
fd43segvma       0x0000000000000000 0x0000000000010000 xw
fd44segvma       0x0000000000000000 0x0000000000010000 xw
fd45segvma       0x0000000000000000 0x0000000000010000 xw
fd46segvma       0x0000000000000000 0x0000000000010000 xw
fd47segvma       0x0000000000000000 0x0000000000010000 xw
fd50segvma       0x0000000000000000 0x0000000000010000 xw
fd51segvma       0x0000000000000000 0x0000000000010000 xw
fd52segvma       0x0000000000000000 0x0000000000010000 xw
fd53segvma       0x0000000000000000 0x0000000000010000 xw
fd54segvma       0x0000000000000000 0x0000000000010000 xw
fd55segvma       0x0000000000000000 0x0000000000010000 xw
fd56segvma       0x0000000000000000 0x0000000000010000 xw
fd57segvma       0x0000000000000000 0x0000000000010000 xw
fd60segvma       0x0000000000000000 0x0000000000010000 xw
fd61segvma       0x0000000000000000 0x0000000000010000 xw
fd62segvma       0x0000000000000000 0x0000000000010000 xw
fd63segvma       0x0000000000000000 0x0000000000010000 xw
fd64segvma       0x0000000000000000 0x0000000000010000 xw
fd65segvma       0x0000000000000000 0x0000000000010000 xw
fd66segvma       0x0000000000000000 0x0000000000010000 xw
fd67segvma       0x0000000000000000 0x0000000000010000 xw
fd70segvma       0x0000000000000000 0x0000000000010000 xw
fd71segvma       0x0000000000000000 0x0000000000010000 xw
fd72segvma       0x0000000000000000 0x0000000000010000 xw
fd73segvma       0x0000000000000000 0x0000000000010000 xw
fd74segvma       0x0000000000000000 0x0000000000010000 xw
fd75segvma       0x0000000000000000 0x0000000000010000 xw
fd76segvma       0x0000000000000000 0x0000000000010000 xw
fd77segvma       0x0000000000000000 0x0000000000010000 xw
fdXXsegvma       0x0000000000000000 0x0000000000010000 xw
dsegvma          0x0000000000000020 0x0000000000010000 xw
*default*        0x0000000000000000 0xffffffffffffffff

Linker script and memory map

LOAD cb_catch.obj
LOAD termhook.obj
LOAD xms_crit.obj
LOAD xms_brk.obj
LOAD xms_2e.obj
LOAD cswap.obj
LOAD cswapc.obj
LOAD batch.obj
LOAD cmdtable.obj
LOAD command.obj
LOAD expalias.obj
LOAD init.obj
LOAD kswap.obj
LOAD loadhigh.obj
LOAD module.obj
LOAD redir.obj
LOAD ver.obj
LOAD command.ld
                0x000000000000fffe                _TEXTSEG = ((((LOADADDR (.text) / 0x10) - __msdos_mz_hdr_paras) - (ADDR (.text) / 0x10)) + 0x10000)
LOAD ../cmd/cmds.lib
LOAD ../lib/freecom.lib
LOAD ../strings/strings.lib
LOAD ../suppl/suppl_s.lib
LOAD /home/evln/proj/build-ia16.202501/prefix/bin/../lib/gcc/ia16-elf/6.3.0/../../../../ia16-elf/lib/regparmcall/libi86.a
LOAD /home/evln/proj/build-ia16.202501/prefix/bin/../lib/gcc/ia16-elf/6.3.0/../../../../ia16-elf/lib/regparmcall/libastdio.a
LOAD /home/evln/proj/build-ia16.202501/prefix/bin/../lib/gcc/ia16-elf/6.3.0/../../../../ia16-elf/lib/regparmcall/gprtf-fw.a
LOAD /home/evln/proj/build-ia16.202501/prefix/bin/../lib/gcc/ia16-elf/6.3.0/../../../../ia16-elf/lib/regparmcall/gscnf-fw.a
LOAD /home/evln/proj/build-ia16.202501/prefix/bin/../lib/gcc/ia16-elf/6.3.0/../../../../ia16-elf/lib/regparmcall/tprtf-fw.a
LOAD /home/evln/proj/build-ia16.202501/prefix/bin/../lib/gcc/ia16-elf/6.3.0/../../../../ia16-elf/lib/regparmcall/tscnf-fw.a
LOAD /home/evln/proj/build-ia16.202501/prefix/bin/../lib/gcc/ia16-elf/6.3.0/../../../../ia16-elf/lib/regparmcall/iprtf-fw.a
LOAD /home/evln/proj/build-ia16.202501/prefix/bin/../lib/gcc/ia16-elf/6.3.0/../../../../ia16-elf/lib/regparmcall/iscnf-fw.a
LOAD /home/evln/proj/build-ia16.202501/prefix/bin/../lib/gcc/ia16-elf/6.3.0/../../../../ia16-elf/lib/regparmcall/libfstdio.a
LOAD /home/evln/proj/build-ia16.202501/prefix/bin/../lib/gcc/ia16-elf/6.3.0/../../../../ia16-elf/lib/regparmcall/tprtf-fw.a
LOAD /home/evln/proj/build-ia16.202501/prefix/bin/../lib/gcc/ia16-elf/6.3.0/../../../../ia16-elf/lib/regparmcall/tscnf-fw.a
LOAD /home/evln/proj/build-ia16.202501/prefix/bin/../lib/gcc/ia16-elf/6.3.0/../../../../ia16-elf/lib/regparmcall/gprtf-fw.a
LOAD /home/evln/proj/build-ia16.202501/prefix/bin/../lib/gcc/ia16-elf/6.3.0/../../../../ia16-elf/lib/regparmcall/gscnf-fw.a
LOAD /home/evln/proj/build-ia16.202501/prefix/bin/../lib/gcc/ia16-elf/6.3.0/regparmcall/crtbegin.o
LOAD /home/evln/proj/build-ia16.202501/prefix/bin/../lib/gcc/ia16-elf/6.3.0/regparmcall/crtend.o
LOAD /home/evln/proj/build-ia16.202501/prefix/bin/../lib/gcc/ia16-elf/6.3.0/../../../../ia16-elf/lib/regparmcall/dos-s-c0.o
START GROUP
LOAD /home/evln/proj/build-ia16.202501/prefix/bin/../lib/gcc/ia16-elf/6.3.0/../../../../ia16-elf/lib/regparmcall/libc.a
LOAD /home/evln/proj/build-ia16.202501/prefix/bin/../lib/gcc/ia16-elf/6.3.0/regparmcall/libgcc.a
LOAD /home/evln/proj/build-ia16.202501/prefix/bin/../lib/gcc/ia16-elf/6.3.0/../../../../ia16-elf/lib/regparmcall/libdos-s.a
LOAD /home/evln/proj/build-ia16.202501/prefix/bin/../lib/gcc/ia16-elf/6.3.0/../../../../ia16-elf/lib/regparmcall/libm.a
END GROUP

.head
 *(.head)
 *(.head.*)

.msdos_mz_hdr   0x0000000000000000       0xb0
                0x0000000000000000                __msdos_mz_hdr_start = .
                0x0000000000000000        0x2 SHORT 0x5a4d
                0x0000000000000002        0x2 SHORT 0x1b0 ((LOADADDR (.data) + SIZEOF (.data)) % 0x200)
                0x0000000000000004        0x2 SHORT 0x79 (((LOADADDR (.data) + SIZEOF (.data)) + 0x1ff) / 0x200)
                0x0000000000000006        0x2 SHORT 0x24 __msdos_mz_rels
                0x0000000000000008        0x2 SHORT 0xb __msdos_mz_hdr_paras
                0x000000000000000a        0x2 SHORT 0xf05 (((0x10000 - SIZEOF (.data)) - ADDR (.data)) / 0x10)
                0x000000000000000c        0x2 SHORT 0xf05 DEFINED (__msdos_handle_v1)?0xffff:(((0x10000 - SIZEOF (.data)) - ADDR (.data)) / 0x10)
                0x000000000000000e        0x2 SHORT 0x10e15 ((((LOADADDR (.data) / 0x10) - __msdos_mz_hdr_paras) - (ADDR (.data) / 0x10)) + 0x10000)
                0x0000000000000010        0x2 SHORT 0x0
                0x0000000000000012        0x2 SHORT 0x0
                0x0000000000000014        0x2 SHORT 0x20 _start
                0x0000000000000016        0x2 SHORT 0xfffe ((((LOADADDR (.text) / 0x10) - __msdos_mz_hdr_paras) - (ADDR (.text) / 0x10)) + 0x10000)
                0x0000000000000018        0x2 SHORT 0x1c (__msdos_mz_rel_start - __msdos_mz_hdr_start)
                0x000000000000001a        0x2 SHORT 0x0
 *(.msdos_mz_hdr .msdos_mz_hdr.*)
                0x000000000000001c                __msdos_mz_rel_start = .
 *(.msdos_mz_reloc .msdos_mz_reloc.*)
 .msdos_mz_reloc
                0x000000000000001c        0x8 cswap.obj
 .msdos_mz_reloc.0
                0x0000000000000024       0x10 cswapc.obj
 .msdos_mz_reloc.0
                0x0000000000000034       0x14 command.obj
 .msdos_mz_reloc.0
                0x0000000000000048       0x38 init.obj
 .msdos_mz_reloc.0
                0x0000000000000080        0x4 ../cmd/cmds.lib(if.obj)
 .msdos_mz_reloc.0
                0x0000000000000084        0xc ../lib/freecom.lib(cbreak.obj)
 .msdos_mz_reloc.0
                0x0000000000000090        0x4 ../lib/freecom.lib(cgetch.obj)
 .msdos_mz_reloc.0
                0x0000000000000094       0x10 ../lib/freecom.lib(exec.obj)
 .msdos_mz_reloc.0
                0x00000000000000a4        0x4 ../lib/freecom.lib(exec1.obj)
 .msdos_mz_reloc.0
                0x00000000000000a8        0x4 /home/evln/proj/build-ia16.202501/prefix/bin/../lib/gcc/ia16-elf/6.3.0/../../../../ia16-elf/lib/regparmcall/libdos-s.a(dos-near-data-segment.o)
                0x00000000000000ac                __msdos_mz_rel_end = .
                0x0000000000000024                __msdos_mz_rels = ((. - __msdos_mz_rel_start) / 0x4)
                0x00000000000000ac                . = DEFINED (__msdos_handle_v1)?ALIGN (0x200):.
                0x000000000000000b                __msdos_mz_hdr_paras = (((. - __msdos_mz_hdr_start) + 0xf) / 0x10)
                0x00000000000000b0                . = ALIGN (0x10)
 *fill*         0x00000000000000ac        0x4 
                0x0000000000000001                ASSERT ((((__msdos_mz_rel_end - __msdos_mz_rel_start) % 0x4) == 0x0), Error: MZ relocations are not 4-byte aligned)
                0x0000000000000001                ASSERT ((__msdos_mz_rels <= 0xffff), Error: too many MZ relocations)

.text           0x0000000000000020     0xe170 load address 0x00000000000000b0
                0x0000000000000020                __stext = .
 *(.startupA)
 .startupA      0x0000000000000020        0x0 /home/evln/proj/build-ia16.202501/prefix/bin/../lib/gcc/ia16-elf/6.3.0/../../../../ia16-elf/lib/regparmcall/dos-s-c0.o
                0x0000000000000020                _start
 *(.startupB)
 *(.startupC)
 .startupC      0x0000000000000020        0x8 /home/evln/proj/build-ia16.202501/prefix/bin/../lib/gcc/ia16-elf/6.3.0/../../../../ia16-elf/lib/regparmcall/dos-s-c0.o
 *(.msdos_init)
 *(.msdos_init.*)
 *(.msdos_initA)
 *(.msdos_initA.*)
 *(.startupD)
 .startupD      0x0000000000000028        0xf /home/evln/proj/build-ia16.202501/prefix/bin/../lib/gcc/ia16-elf/6.3.0/../../../../ia16-elf/lib/regparmcall/dos-s-c0.o
 *(.msdos_initB)
 *(.msdos_initB.*)
 *(.startupE)
 .startupE      0x0000000000000037       0xab /home/evln/proj/build-ia16.202501/prefix/bin/../lib/gcc/ia16-elf/6.3.0/../../../../ia16-elf/lib/regparmcall/dos-s-c0.o
 *(.preinit)
 *(.preinit.*)
 *(.init)
 .init          0x00000000000000e2        0x3 /home/evln/proj/build-ia16.202501/prefix/bin/../lib/gcc/ia16-elf/6.3.0/regparmcall/crtbegin.o
 .init          0x00000000000000e5        0x3 /home/evln/proj/build-ia16.202501/prefix/bin/../lib/gcc/ia16-elf/6.3.0/regparmcall/crtend.o
 *(.startupF)
 .startupF      0x00000000000000e8       0x76 /home/evln/proj/build-ia16.202501/prefix/bin/../lib/gcc/ia16-elf/6.3.0/../../../../ia16-elf/lib/regparmcall/dos-s-c0.o
 *(.exitA)
 .exitA         0x000000000000015e        0x1 /home/evln/proj/build-ia16.202501/prefix/bin/../lib/gcc/ia16-elf/6.3.0/../../../../ia16-elf/lib/regparmcall/dos-s-c0.o
                0x000000000000015e                _exit
 *(.fini)
 .fini          0x000000000000015f        0x3 /home/evln/proj/build-ia16.202501/prefix/bin/../lib/gcc/ia16-elf/6.3.0/regparmcall/crtbegin.o
 *(.exitB)
 .exitB         0x0000000000000162        0x5 /home/evln/proj/build-ia16.202501/prefix/bin/../lib/gcc/ia16-elf/6.3.0/../../../../ia16-elf/lib/regparmcall/dos-s-c0.o
                0x0000000000000163                __msdos_crt_exit
 *(.text)
 *fill*         0x0000000000000167        0x9 
 .text          0x0000000000000170        0xb cb_catch.obj
                0x0000000000000170                CBreakCounter
                0x0000000000000172                cbreak_handler
 *fill*         0x000000000000017b        0x5 
 .text          0x0000000000000180       0xa6 termhook.obj
                0x0000000000000180                termAddr
                0x0000000000000184                myPID
                0x0000000000000186                origPPID
                0x0000000000000188                terminateFreeCOMHook
 *fill*         0x0000000000000226        0xa 
 .text          0x0000000000000230      0x481 xms_crit.obj
                0x0000000000000230                autofail_err_handler
                0x0000000000000233                lowlevel_err_handler
                0x00000000000003ea                criter_repeat_checkarea
 *fill*         0x00000000000006b1        0xf 
 .text          0x00000000000006c0        0x2 xms_brk.obj
                0x00000000000006c0                lowlevel_cbreak_handler
 *fill*         0x00000000000006c2        0xe 
 .text          0x00000000000006d0        0x4 xms_2e.obj
                0x00000000000006d0                lowlevel_int_2e_handler
 *fill*         0x00000000000006d4        0xc 
 .text          0x00000000000006e0      0x315 cswap.obj
                0x00000000000006e0                dosFCB1
                0x0000000000000705                dosFCB2
                0x000000000000072a                dosCMDNAME
                0x00000000000008aa                dosParamDosExec
                0x00000000000008aa                localStack
                0x00000000000008c0                XMSdriverAdress
                0x00000000000008c4                SwapTransientSize
                0x00000000000008c6                XMSrestore
                0x00000000000008d6                canexit
                0x00000000000008d8                mySS
                0x00000000000008da                mySP
                0x0000000000000984                xms_kill
                0x0000000000000993                SWAPresidentEnd
                0x0000000000000993                XMSrequest
                0x0000000000000998                XMSexec
 .text          0x00000000000009f5      0x222 cswapc.obj
                0x0000000000000a0d                XMSisactive
                0x0000000000000a1a                XMSinit
                0x0000000000000bac                XMSexit
                0x0000000000000bc9                XMSswapmessagesIn
 .text          0x0000000000000c17      0x5b4 batch.obj
                0x0000000000000c6b                find_arg_bc
                0x0000000000000cb3                activeBatchContext
                0x0000000000000cc8                setBatchParams
                0x0000000000000ce7                exit_batch
                0x0000000000000d25                newBatchContext
                0x0000000000000d56                batch
                0x0000000000000def                readbatchline
 .text          0x00000000000011cb        0x0 cmdtable.obj
 .text          0x00000000000011cb      0x9e5 command.obj
                0x00000000000011cb                stack_check_init
                0x00000000000011ef                stack_check
                0x000000000000123b                dup
                0x0000000000001241                dup2
                0x000000000000124b                switchar
                0x000000000000126e                isdrive
                0x000000000000128e                execute
                0x000000000000163a                parsecommandline
                0x000000000000188d                expandEnvVars
                0x0000000000001a01                process_input
                0x0000000000001b95                my2e_parsecommandline
 .text          0x0000000000001bb0      0x13b expalias.obj
                0x0000000000001bb0                aliasexpand
 .text          0x0000000000001ceb      0x6a0 init.obj
                0x0000000000001ceb                exitfct
                0x0000000000001ead                initialize
 .text          0x000000000000238b        0x0 kswap.obj
 .text          0x000000000000238b      0x74c loadhigh.obj
                0x0000000000002aa7                cmd_loadhigh
                0x0000000000002acd                cmd_loadfix
 .text          0x0000000000002ad7        0x0 module.obj
 .text          0x0000000000002ad7      0x141 redir.obj
                0x0000000000002ad7                get_redirection
 .text          0x0000000000002c18      0x1c9 ver.obj
                0x0000000000002c65                cmd_ver
 .text          0x0000000000002de1       0x80 ../cmd/cmds.lib(alias.obj)
                0x0000000000002de1                cmd_alias
 .text          0x0000000000002e61        0x6 ../cmd/cmds.lib(beep.obj)
                0x0000000000002e61                cmd_beep
 .text          0x0000000000002e67       0x3d ../cmd/cmds.lib(break.obj)
                0x0000000000002e67                cmd_break
 .text          0x0000000000002ea4       0xc7 ../cmd/cmds.lib(call.obj)
                0x0000000000002ee4                cmd_call
 .text          0x0000000000002f6b        0xa ../cmd/cmds.lib(cdd.obj)
                0x0000000000002f6b                cmd_cdd
 .text          0x0000000000002f75       0xce ../cmd/cmds.lib(chcp.obj)
                0x0000000000002f75                cmd_chcp
 .text          0x0000000000003043        0x9 ../cmd/cmds.lib(chdir.obj)
                0x0000000000003043                cmd_chdir
 .text          0x000000000000304c       0xb8 ../cmd/cmds.lib(cls.obj)
                0x000000000000304c                cmd_cls
 .text          0x0000000000003104      0xb6b ../cmd/cmds.lib(copy.obj)
                0x0000000000003913                cmd_copy
 .text          0x0000000000003c6f       0xc0 ../cmd/cmds.lib(ctty.obj)
                0x0000000000003c6f                cmd_ctty
 .text          0x0000000000003d2f       0xff ../cmd/cmds.lib(date.obj)
                0x0000000000003d5c                cmd_date
 .text          0x0000000000003e2e      0x238 ../cmd/cmds.lib(del.obj)
                0x0000000000003e63                cmd_del
 .text          0x0000000000004066     0x1355 ../cmd/cmds.lib(dir.obj)
                0x0000000000005271                cmd_dir
                0x0000000000005360                cmd_vol
 .text          0x00000000000053bb        0x9 ../cmd/cmds.lib(dirs.obj)
                0x00000000000053bb                cmd_dirs
 .text          0x00000000000053c4        0x9 ../cmd/cmds.lib(doskey.obj)
                0x00000000000053c4                cmd_doskey
 .text          0x00000000000053cd       0x77 ../cmd/cmds.lib(echo.obj)
                0x00000000000053cd                cmd_echo
 .text          0x0000000000005444        0x9 ../cmd/cmds.lib(exit.obj)
                0x0000000000005444                internal_exit
 .text          0x000000000000544d      0x2ee ../cmd/cmds.lib(for.obj)
                0x0000000000005682                cmd_for
                0x00000000000056e4                cmd_for_hackery
 .text          0x000000000000573b       0x57 ../cmd/cmds.lib(goto.obj)
                0x000000000000573b                cmd_goto
 .text          0x0000000000005792       0x40 ../cmd/cmds.lib(history.obj)
                0x0000000000005792                cmd_history
 .text          0x00000000000057d2      0x218 ../cmd/cmds.lib(if.obj)
                0x00000000000057d2                cmd_if
 .text          0x00000000000059ea       0x96 ../cmd/cmds.lib(lfnfor.obj)
                0x00000000000059ea                cmd_lfnfor
 .text          0x0000000000005a80       0xd8 ../cmd/cmds.lib(memory.obj)
                0x0000000000005ab8                cmd_memory
 .text          0x0000000000005b58       0x78 ../cmd/cmds.lib(mkdir.obj)
                0x0000000000005bb9                recursive_mkdir
                0x0000000000005bc6                cmd_mkdir
 .text          0x0000000000005bd0       0x4c ../cmd/cmds.lib(path.obj)
                0x0000000000005bd0                cmd_path
 .text          0x0000000000005c1c       0x2c ../cmd/cmds.lib(pause.obj)
                0x0000000000005c1c                cmd_pause
 .text          0x0000000000005c48       0x3d ../cmd/cmds.lib(popd.obj)
                0x0000000000005c48                cmd_popd
 .text          0x0000000000005c85       0x17 ../cmd/cmds.lib(prompt.obj)
                0x0000000000005c85                cmd_prompt
 .text          0x0000000000005c9c       0x37 ../cmd/cmds.lib(pushd.obj)
                0x0000000000005c9c                cmd_pushd
 .text          0x0000000000005cd3        0x3 ../cmd/cmds.lib(rem.obj)
                0x0000000000005cd3                cmd_rem
 .text          0x0000000000005cd6      0x26f ../cmd/cmds.lib(ren.obj)
                0x0000000000005cd6                myfnsplit
                0x0000000000005dab                myfnmerge
                0x0000000000005e0c                cmd_rename
 .text          0x0000000000005f45      0x1ce ../cmd/cmds.lib(rmdir.obj)
                0x0000000000005f45                rmdir_withfiles
                0x000000000000607e                recursive_rmdir
                0x0000000000006109                cmd_rmdir
 .text          0x0000000000006113      0x275 ../cmd/cmds.lib(set.obj)
                0x000000000000618b                cmd_set
 .text          0x0000000000006388       0x30 ../cmd/cmds.lib(shift.obj)
                0x0000000000006388                cmd_shift
 .text          0x00000000000063b8       0xe7 ../cmd/cmds.lib(time.obj)
                0x00000000000063e5                cmd_time
 .text          0x000000000000649f       0x2a ../cmd/cmds.lib(truename.obj)
                0x000000000000649f                cmd_truename
 .text          0x00000000000064c9      0x112 ../cmd/cmds.lib(type.obj)
                0x00000000000064c9                cmd_type
 .text          0x00000000000065db       0x43 ../cmd/cmds.lib(verify.obj)
                0x00000000000065db                cmd_verify
 .text          0x000000000000661e       0x65 ../cmd/cmds.lib(which.obj)
                0x000000000000661e                cmd_which
 .text          0x0000000000006683       0x1e ../lib/freecom.lib(absfile.obj)
                0x0000000000006683                abspath
 .text          0x00000000000066a1       0x56 ../lib/freecom.lib(app_get.obj)
                0x00000000000066a1                appendDisable
 .text          0x00000000000066f7       0x1f ../lib/freecom.lib(app_set.obj)
                0x00000000000066f7                appendRestore
 .text          0x0000000000006716       0x25 ../lib/freecom.lib(beep_n.obj)
                0x0000000000006716                beep
 .text          0x000000000000673b       0x1d ../lib/freecom.lib(brk_get.obj)
                0x000000000000673b                getbreak
 .text          0x0000000000006758       0x1b ../lib/freecom.lib(brk_set.obj)
                0x0000000000006758                setbreak
 .text          0x0000000000006773      0x16a ../lib/freecom.lib(cbreak.obj)
                0x00000000000067b6                getCurrentConDev
                0x00000000000067ba                setCurrentConDev
                0x00000000000067de                chkCBreak
 .text          0x00000000000068dd      0x15d ../lib/freecom.lib(cd_dir.obj)
                0x00000000000068dd                cd_dir
 .text          0x0000000000006a3a       0x4a ../lib/freecom.lib(cgetch.obj)
                0x0000000000006a3a                cgetchar
 .text          0x0000000000006a84      0x179 ../lib/freecom.lib(chgctxt.obj)
                0x0000000000006a84                chgCtxt
 .text          0x0000000000006bfd       0x1e ../lib/freecom.lib(chgdrv.obj)
                0x0000000000006bfd                changeDrive
 .text          0x0000000000006c1b       0x32 ../lib/freecom.lib(chgenv.obj)
                0x0000000000006c1b                chgEnv
 .text          0x0000000000006c4d       0x21 ../lib/freecom.lib(chgenvc.obj)
                0x0000000000006c4d                chgEnvCase
 .text          0x0000000000006c6e       0x11 ../lib/freecom.lib(chgenvr.obj)
                0x0000000000006c6e                chgEnvRemove
 .text          0x0000000000006c7f      0x94f ../lib/freecom.lib(cmdinput.obj)
                0x0000000000006d18                mywherex
                0x0000000000006d30                mywherey
                0x0000000000006dc1                outc
                0x0000000000006de0                outs
                0x0000000000006deb                readcommandEnhanced
 .text          0x00000000000075ce       0x22 ../lib/freecom.lib(critrchk.obj)
                0x00000000000075ce                registerCriterRepeatCheckAddr
 .text          0x00000000000075f0        0x0 ../lib/freecom.lib(ctxt.obj)
 .text          0x00000000000075f0       0x54 ../lib/freecom.lib(ctxt_clr.obj)
                0x000000000000761e                ctxtClear
 .text          0x0000000000007644       0x91 ../lib/freecom.lib(ctxt_get.obj)
                0x0000000000007644                ctxtGet
 .text          0x00000000000076d5        0x0 ../lib/freecom.lib(ctxt_inf.obj)
 .text          0x00000000000076d5       0x63 ../lib/freecom.lib(ctxt_mk.obj)
                0x00000000000076d5                ctxtCreate
 .text          0x0000000000007738       0x2a ../lib/freecom.lib(ctxt_mkb.obj)
                0x0000000000007738                ctxtCreateMemBlock
 .text          0x0000000000007762       0x1b ../lib/freecom.lib(ctxt_mkn.obj)
                0x0000000000007762                ctxtMkItemName
 .text          0x000000000000777d       0x62 ../lib/freecom.lib(ctxt_pop.obj)
                0x000000000000777d                ctxtPop
 .text          0x00000000000077df       0x54 ../lib/freecom.lib(ctxt_psh.obj)
                0x00000000000077df                ctxtPush
 .text          0x0000000000007833       0x6a ../lib/freecom.lib(ctxt_rnu.obj)
                0x000000000000787c                ctxtRenumberItems
 .text          0x000000000000789d       0x58 ../lib/freecom.lib(ctxt_set.obj)
                0x000000000000789d                ctxtSet
 .text          0x00000000000078f5       0x68 ../lib/freecom.lib(ctxt_vw.obj)
                0x000000000000791f                ctxtView
 .text          0x000000000000795d       0xb2 ../lib/freecom.lib(curdatel.obj)
                0x000000000000795d                curDateLong
 .text          0x0000000000007a0f       0x36 ../lib/freecom.lib(curtime.obj)
                0x0000000000007a0f                curTime
 .text          0x0000000000007a45       0x2a ../lib/freecom.lib(cwd.obj)
                0x0000000000007a45                cwd
 .text          0x0000000000007a6f       0x35 ../lib/freecom.lib(dateget.obj)
                0x0000000000007a6f                _dos_getdate
 .text          0x0000000000007aa4       0x37 ../lib/freecom.lib(dateset.obj)
                0x0000000000007aa4                _dos_setdate
 .text          0x0000000000007adb       0x56 ../lib/freecom.lib(devopen.obj)
                0x0000000000007adb                devopen
 .text          0x0000000000007b31       0x1d ../lib/freecom.lib(dfn_err.obj)
                0x0000000000007b31                display_errno_fnam_error
 .text          0x0000000000007b4e       0x1f ../lib/freecom.lib(dispcnt.obj)
                0x0000000000007b4e                dispCount
 .text          0x0000000000007b6d       0x2e ../lib/freecom.lib(drvnum.obj)
                0x0000000000007b6d                drvNum
 .text          0x0000000000007b9b      0x14a ../lib/freecom.lib(exec.obj)
                0x0000000000007b9b                exec
 .text          0x0000000000007ce5       0x86 ../lib/freecom.lib(exec1.obj)
                0x0000000000007ce5                setErrorLevel
 .text          0x0000000000007d6b      0x12a ../lib/freecom.lib(farread.obj)
                0x0000000000007d6b                farread
                0x0000000000007da2                farwrite
                0x0000000000007dd9                sfn_open
                0x0000000000007e06                dos_close
                0x0000000000007e29                dos_read
                0x0000000000007e30                dos_write
                0x0000000000007e37                sfn_creat
                0x0000000000007e66                sfn_creatnew
 .text          0x0000000000007e95      0x2d0 ../lib/freecom.lib(filecomp.obj)
                0x0000000000008145                complete_filename
                0x0000000000008152                show_completion_matches
 .text          0x0000000000008165       0x28 ../lib/freecom.lib(fdattr.obj)
                0x0000000000008165                fdattr
 .text          0x000000000000818d       0x29 ../lib/freecom.lib(fdsattr.obj)
                0x000000000000818d                fdsetattr
 .text          0x00000000000081b6       0xf8 ../lib/freecom.lib(fillcomp.obj)
                0x0000000000008218                fillFnam
 .text          0x00000000000082ae      0x1cd ../lib/freecom.lib(find.obj)
                0x00000000000083aa                skip_word
                0x00000000000083b1                skipdm
                0x00000000000083b7                skipnonoptdm
                0x0000000000008420                skipnonopt_word
 .text          0x000000000000847b       0x1e ../lib/freecom.lib(freep.obj)
                0x000000000000847b                freep
 .text          0x0000000000008499       0x25 ../lib/freecom.lib(gallstr.obj)
                0x0000000000008499                dosGetAllocStrategy
 .text          0x00000000000084be       0x22 ../lib/freecom.lib(get1mcb.obj)
                0x00000000000084be                GetFirstMCB
 .text          0x00000000000084e0       0x17 ../lib/freecom.lib(getenv.obj)
                0x00000000000084e0                getEnv
 .text          0x00000000000084f7       0x3c ../lib/freecom.lib(goxy.obj)
                0x00000000000084f7                goxy
 .text          0x0000000000008533      0x15a ../lib/freecom.lib(grabfcom.obj)
                0x0000000000008533                grabComFilename
 .text          0x000000000000868d       0x25 ../lib/freecom.lib(gumblink.obj)
                0x000000000000868d                dosGetUMBLinkState
 .text          0x00000000000086b2       0x5b ../lib/freecom.lib(hdlrctxt.obj)
                0x00000000000086cd                breakVarAssign
 .text          0x000000000000870d       0x4e ../lib/freecom.lib(hist_get.obj)
                0x000000000000870d                histGet
 .text          0x000000000000875b       0x1a ../lib/freecom.lib(hist_set.obj)
                0x000000000000875b                histSet
 .text          0x0000000000008775       0x2a ../lib/freecom.lib(is_empty.obj)
                0x0000000000008775                is_empty
 .text          0x000000000000879f       0x4d ../lib/freecom.lib(is_fnamc.obj)
                0x000000000000879f                is_fnchar
 .text          0x00000000000087ec       0x18 ../lib/freecom.lib(is_fnstr.obj)
                0x00000000000087ec                is_fnstr
 .text          0x0000000000008804       0x25 ../lib/freecom.lib(is_pchr.obj)
                0x0000000000008804                is_pathdelim
 .text          0x0000000000008829        0xb ../lib/freecom.lib(isadev.obj)
                0x0000000000008829                isadev
 .text          0x0000000000008834       0x20 ../lib/freecom.lib(lastdget.obj)
                0x0000000000008834                lastDirGet
 .text          0x0000000000008854       0x20 ../lib/freecom.lib(lastdset.obj)
                0x0000000000008854                lastDirSet
 .text          0x0000000000008874       0x86 ../lib/freecom.lib(leadopt.obj)
                0x0000000000008874                leadOptions
 .text          0x00000000000088fa      0x390 ../lib/freecom.lib(lfnfuncs.obj)
                0x00000000000088fa                getshortfilename
                0x000000000000897d                lfn_creat
                0x00000000000089eb                lfnrename
                0x0000000000008a5f                lfnfindfirst
                0x0000000000008b2b                lfnfindnext
                0x0000000000008be1                lfnfindclose
                0x0000000000008c2f                lfnmkdir
                0x0000000000008c7c                lfnrmdir
                0x0000000000008c83                lfnchdir
 *fill*         0x0000000000008c8a        0x6 
 .text          0x0000000000008c90       0x36 ../lib/freecom.lib(lowexec.obj)
                0x0000000000008c90                lowLevelExec
 .text          0x0000000000008cc6       0x37 ../lib/freecom.lib(ltrimcl.obj)
                0x0000000000008cc6                ltrimcl
 .text          0x0000000000008cfd       0x3e ../lib/freecom.lib(match.obj)
                0x0000000000008cfd                match_
 .text          0x0000000000008d3b      0x1fe ../lib/freecom.lib(messages.obj)
                0x0000000000008d3b                unloadMsgs
                0x0000000000008e5b                msgSegment
 .text          0x0000000000008f39       0xad ../lib/freecom.lib(mk_rddir.obj)
                0x0000000000008f73                mk_rd_dir
 .text          0x0000000000008fe6       0x60 ../lib/freecom.lib(msg_dps.obj)
                0x0000000000008fe6                displayString
                0x0000000000009016                displayError
 .text          0x0000000000009046       0x5e ../lib/freecom.lib(msg_fstr.obj)
                0x0000000000009046                getString
 .text          0x00000000000090a4       0x2e ../lib/freecom.lib(msg_gpt.obj)
                0x00000000000090a4                getPromptString
 .text          0x00000000000090d2       0x19 ../lib/freecom.lib(msg_mkey.obj)
                0x00000000000090d2                mapMetakey
 .text          0x00000000000090eb       0x57 ../lib/freecom.lib(msg_prmp.obj)
                0x00000000000090eb                userprompt
 .text          0x0000000000009142      0x136 ../lib/freecom.lib(mux_ae.obj)
                0x0000000000009142                runExtension
 .text          0x0000000000009278       0x28 ../lib/freecom.lib(myperror.obj)
                0x0000000000009278                myperror
 .text          0x00000000000092a0        0xe ../lib/freecom.lib(nls.obj)
                0x00000000000092a0                refreshNLS
 .text          0x00000000000092ae       0x5f ../lib/freecom.lib(nls_date.obj)
                0x00000000000092ae                nls_makedate
 .text          0x000000000000930d      0x120 ../lib/freecom.lib(nls_time.obj)
                0x000000000000930d                nls_maketime
 .text          0x000000000000942d       0xc3 ../lib/freecom.lib(num_fmt.obj)
                0x000000000000942d                convert
 .text          0x00000000000094f0       0x4d ../lib/freecom.lib(onoff.obj)
                0x00000000000094f0                onoffStr
 .text          0x000000000000953d       0x54 ../lib/freecom.lib(openf.obj)
                0x000000000000953d                isDeviceName
 .text          0x0000000000009591       0x40 ../lib/freecom.lib(optsb.obj)
                0x0000000000009591                optScanBool_
 .text          0x00000000000095d1       0x60 ../lib/freecom.lib(optsi.obj)
                0x00000000000095d1                optScanInteger_
 .text          0x0000000000009631       0x33 ../lib/freecom.lib(optss.obj)
                0x0000000000009631                optScanString_
 .text          0x0000000000009664      0x189 ../lib/freecom.lib(pr_date.obj)
                0x0000000000009664                parsedate
 .text          0x00000000000097ed       0x19 ../lib/freecom.lib(pr_prmpt.obj)
                0x00000000000097ed                printprompt
 .text          0x0000000000009806      0x151 ../lib/freecom.lib(pr_time.obj)
                0x0000000000009806                parsetime
 .text          0x0000000000009957      0x464 ../lib/freecom.lib(prf.obj)
                0x00000000000099a2                vsprintf
                0x00000000000099c0                sprintf
                0x0000000000009d57                vfprintf
                0x0000000000009d7a                vprintf
                0x0000000000009d84                printf
                0x0000000000009d9c                puts
                0x0000000000009da7                fprintf
 .text          0x0000000000009dbb      0x1f8 ../lib/freecom.lib(prprompt.obj)
                0x0000000000009dbb                displayPrompt
 .text          0x0000000000009fb3       0x20 ../lib/freecom.lib(readcmd.obj)
                0x0000000000009fb3                set_readcommandType
                0x0000000000009fc3                readcommand
 .text          0x0000000000009fd3       0x38 ../lib/freecom.lib(realnum.obj)
                0x0000000000009fd3                realNum
 .text          0x000000000000a00b       0x27 ../lib/freecom.lib(res.obj)
                0x000000000000a00b                enumResources
 .text          0x000000000000a032      0x118 ../lib/freecom.lib(res_r.obj)
                0x000000000000a032                enumFileResources
 .text          0x000000000000a14a       0x4f ../lib/freecom.lib(res_vald.obj)
                0x000000000000a158                validResFile
 .text          0x000000000000a199       0x32 ../lib/freecom.lib(resfile.obj)
                0x000000000000a199                comResFile
 .text          0x000000000000a1cb       0x10 ../lib/freecom.lib(rmtmpfil.obj)
                0x000000000000a1cb                killtmpfn
 .text          0x000000000000a1db       0x47 ../lib/freecom.lib(rtrimcl.obj)
                0x000000000000a1db                rtrimcl
 .text          0x000000000000a222       0x3b ../lib/freecom.lib(rtrimsp.obj)
                0x000000000000a222                rtrimsp
 .text          0x000000000000a25d       0x1b ../lib/freecom.lib(salloc.obj)
                0x000000000000a25d                dosSetAllocStrategy
 .text          0x000000000000a278       0x3e ../lib/freecom.lib(samefile.obj)
                0x000000000000a278                samefile
 .text          0x000000000000a2b6       0xbd ../lib/freecom.lib(scancmd.obj)
                0x000000000000a2b6                scanCmdline
 .text          0x000000000000a373      0x11a ../lib/freecom.lib(scanopt.obj)
                0x000000000000a373                scanOption
 .text          0x000000000000a48d       0x61 ../lib/freecom.lib(session.obj)
                0x000000000000a48d                saveSession
                0x000000000000a4c2                restoreSession
 .text          0x000000000000a4ee       0x98 ../lib/freecom.lib(showcmds.obj)
                0x000000000000a4ee                showcmds
 .text          0x000000000000a586      0x179 ../lib/freecom.lib(skqwd.obj)
                0x000000000000a586                skipqword
 .text          0x000000000000a6ff       0x11 ../lib/freecom.lib(spfnam.obj)
                0x000000000000a6ff                skipfnam
 .text          0x000000000000a710       0xc8 ../lib/freecom.lib(split.obj)
                0x000000000000a7cb                split
                0x000000000000a7d1                split_batchargs
 .text          0x000000000000a7d8       0x1b ../lib/freecom.lib(sumblink.obj)
                0x000000000000a7d8                dosSetUMBLinkState
 .text          0x000000000000a7f3       0x36 ../lib/freecom.lib(timeget.obj)
                0x000000000000a7f3                _dos_gettime
 .text          0x000000000000a829       0x35 ../lib/freecom.lib(timeset.obj)
                0x000000000000a829                _dos_settime
 .text          0x000000000000a85e       0xb6 ../lib/freecom.lib(tmpnam.obj)
                0x000000000000a873                tmpfn
 .text          0x000000000000a914        0xc ../lib/freecom.lib(trimsp.obj)
                0x000000000000a914                trimsp
 .text          0x000000000000a920       0x18 ../lib/freecom.lib(truepath.obj)
                0x000000000000a920                truepath
 .text          0x000000000000a938       0x23 ../lib/freecom.lib(truncate.obj)
                0x000000000000a938                truncate
 .text          0x000000000000a95b       0x1e ../lib/freecom.lib(txtlend.obj)
                0x000000000000a95b                textlineEnd
 .text          0x000000000000a979       0x98 ../lib/freecom.lib(unquote.obj)
                0x000000000000a979                unquote
 .text          0x000000000000aa11       0x2f ../lib/freecom.lib(vcgetch.obj)
                0x000000000000aa11                vcgetchar
 .text          0x000000000000aa40      0x1a4 ../lib/freecom.lib(where.obj)
                0x000000000000aa40                find_which
 .text          0x000000000000abe4       0x45 ../lib/freecom.lib(delay.obj)
                0x000000000000abe4                delay
 .text          0x000000000000ac29        0xb ../lib/freecom.lib(err2.obj)
                0x000000000000ac29                error_invalid_lswitch
 .text          0x000000000000ac34        0xb ../lib/freecom.lib(err3.obj)
                0x000000000000ac34                error_too_many_parameters
 .text          0x000000000000ac3f        0x7 ../lib/freecom.lib(err5.obj)
                0x000000000000ac3f                error_file_not_found
 .text          0x000000000000ac46        0xb ../lib/freecom.lib(err6.obj)
                0x000000000000ac46                error_sfile_not_found
 .text          0x000000000000ac51        0x7 ../lib/freecom.lib(err7.obj)
                0x000000000000ac51                error_req_param_missing
 .text          0x000000000000ac58        0xb ../lib/freecom.lib(err8.obj)
                0x000000000000ac58                error_bad_command
 .text          0x000000000000ac63        0x7 ../lib/freecom.lib(err10.obj)
                0x000000000000ac63                error_out_of_memory
 .text          0x000000000000ac6a       0x12 ../lib/freecom.lib(err11.obj)
                0x000000000000ac6a                error_syntax
 .text          0x000000000000ac7c        0xb ../lib/freecom.lib(err13.obj)
                0x000000000000ac7c                error_selfcopy
 .text          0x000000000000ac87        0xd ../lib/freecom.lib(err14.obj)
                0x000000000000ac87                error_long_batchline
 .text          0x000000000000ac94        0xb ../lib/freecom.lib(err15.obj)
                0x000000000000ac94                error_bfile_vanished
 .text          0x000000000000ac9f        0xc ../lib/freecom.lib(err16.obj)
                0x000000000000ac9f                error_bfile_no_such_label
 .text          0x000000000000acab        0x7 ../lib/freecom.lib(err17.obj)
                0x000000000000acab                error_invalid_time
 .text          0x000000000000acb2        0xb ../lib/freecom.lib(err18.obj)
                0x000000000000acb2                error_env_var
 .text          0x000000000000acbd        0xb ../lib/freecom.lib(err19.obj)
                0x000000000000acbd                error_env_var_not_found
 .text          0x000000000000acc8        0xb ../lib/freecom.lib(err20.obj)
                0x000000000000acc8                error_filename_too_long
 .text          0x000000000000acd3        0x7 ../lib/freecom.lib(err21.obj)
                0x000000000000acd3                error_command_too_long
 .text          0x000000000000acda        0x7 ../lib/freecom.lib(err22.obj)
                0x000000000000acda                error_line_too_long
 .text          0x000000000000ace1        0x7 ../lib/freecom.lib(err23.obj)
                0x000000000000ace1                error_tempfile
 .text          0x000000000000ace8        0xb ../lib/freecom.lib(err25.obj)
                0x000000000000ace8                error_illformed_option
 .text          0x000000000000acf3        0xb ../lib/freecom.lib(err26.obj)
                0x000000000000acf3                error_opt_arg
 .text          0x000000000000acfe        0xb ../lib/freecom.lib(err27.obj)
                0x000000000000acfe                error_opt_noarg
 .text          0x000000000000ad09        0x7 ../lib/freecom.lib(err28.obj)
                0x000000000000ad09                error_leading_plus
 .text          0x000000000000ad10        0x7 ../lib/freecom.lib(err29.obj)
                0x000000000000ad10                error_trailing_plus
 .text          0x000000000000ad17        0xb ../lib/freecom.lib(err30.obj)
                0x000000000000ad17                error_open_file
 .text          0x000000000000ad22        0xb ../lib/freecom.lib(err31.obj)
                0x000000000000ad22                error_read_file
 .text          0x000000000000ad2d        0xb ../lib/freecom.lib(err32.obj)
                0x000000000000ad2d                error_write_file
 .text          0x000000000000ad38        0xd ../lib/freecom.lib(err33.obj)
                0x000000000000ad38                error_write_file_disc_full
 .text          0x000000000000ad45        0x7 ../lib/freecom.lib(err34.obj)
                0x000000000000ad45                error_copy
 .text          0x000000000000ad4c        0x7 ../lib/freecom.lib(err35.obj)
                0x000000000000ad4c                error_nothing_to_do
 .text          0x000000000000ad53        0xb ../lib/freecom.lib(err36.obj)
                0x000000000000ad53                error_invalid_number
 .text          0x000000000000ad5e        0xb ../lib/freecom.lib(err37.obj)
                0x000000000000ad5e                error_init_fully_qualified
 .text          0x000000000000ad69        0x7 ../lib/freecom.lib(err38.obj)
                0x000000000000ad69                error_corrupt_command_line
 .text          0x000000000000ad70        0x7 ../lib/freecom.lib(err39.obj)
                0x000000000000ad70                error_quoted_c_k
 .text          0x000000000000ad77        0x7 ../lib/freecom.lib(err41.obj)
                0x000000000000ad77                error_l_notimplemented
 .text          0x000000000000ad7e        0x7 ../lib/freecom.lib(err42.obj)
                0x000000000000ad7e                error_u_notimplemented
 .text          0x000000000000ad85        0xb ../lib/freecom.lib(err45.obj)
                0x000000000000ad85                error_no_rw_device
 .text          0x000000000000ad90        0xb ../lib/freecom.lib(err46.obj)
                0x000000000000ad90                error_ctty_dup
 .text          0x000000000000ad9b       0x11 ../lib/freecom.lib(err47.obj)
                0x000000000000ad9b                error_no_cwd
 .text          0x000000000000adac        0x7 ../lib/freecom.lib(err50.obj)
                0x000000000000adac                error_if_exist
 .text          0x000000000000adb3        0x7 ../lib/freecom.lib(err51.obj)
                0x000000000000adb3                error_if_errorlevel
 .text          0x000000000000adba        0x7 ../lib/freecom.lib(err53.obj)
                0x000000000000adba                error_if_command
 .text          0x000000000000adc1        0x7 ../lib/freecom.lib(err54.obj)
                0x000000000000adc1                error_alias_out_of_memory
 .text          0x000000000000adc8        0xc ../lib/freecom.lib(err58.obj)
                0x000000000000adc8                error_dirfct_failed
 .text          0x000000000000add4        0xb ../lib/freecom.lib(err59.obj)
                0x000000000000add4                error_no_alias_name
 .text          0x000000000000addf        0xb ../lib/freecom.lib(err60.obj)
                0x000000000000addf                error_history_size
 .text          0x000000000000adea        0x7 ../lib/freecom.lib(err61.obj)
                0x000000000000adea                error_context_out_of_memory
 .text          0x000000000000adf1        0x7 ../lib/freecom.lib(err63.obj)
                0x000000000000adf1                error_out_of_dos_memory
 .text          0x000000000000adf8        0xd ../lib/freecom.lib(err64.obj)
                0x000000000000adf8                error_context_length
 .text          0x000000000000ae05        0x7 ../lib/freecom.lib(err65.obj)
                0x000000000000ae05                error_context_add_status
 .text          0x000000000000ae0c        0xb ../lib/freecom.lib(err67.obj)
                0x000000000000ae0c                error_redirect_from_file
 .text          0x000000000000ae17        0xb ../lib/freecom.lib(err68.obj)
                0x000000000000ae17                error_redirect_to_file
 .text          0x000000000000ae22        0x7 ../lib/freecom.lib(err69.obj)
                0x000000000000ae22                error_bad_mcb_chain
 .text          0x000000000000ae29        0xb ../lib/freecom.lib(err70.obj)
                0x000000000000ae29                error_unknown
 .text          0x000000000000ae34        0xe ../lib/freecom.lib(err71.obj)
                0x000000000000ae34                error_invalid_drive
 .text          0x000000000000ae42        0x7 ../lib/freecom.lib(err72.obj)
                0x000000000000ae42                error_no_env
 .text          0x000000000000ae49        0x7 ../lib/freecom.lib(err73.obj)
                0x000000000000ae49                error_on_off
 .text          0x000000000000ae50        0x7 ../lib/freecom.lib(err74.obj)
                0x000000000000ae50                error_invalid_date
 .text          0x000000000000ae57        0x7 ../lib/freecom.lib(err75.obj)
                0x000000000000ae57                error_for_bad_var
 .text          0x000000000000ae5e        0x7 ../lib/freecom.lib(err76.obj)
                0x000000000000ae5e                error_for_in
 .text          0x000000000000ae65        0x7 ../lib/freecom.lib(err77.obj)
                0x000000000000ae65                error_for_parens
 .text          0x000000000000ae6c        0x7 ../lib/freecom.lib(err78.obj)
                0x000000000000ae6c                error_for_do
 .text          0x000000000000ae73        0x7 ../lib/freecom.lib(err79.obj)
                0x000000000000ae73                error_for_no_command
 .text          0x000000000000ae7a        0x7 ../lib/freecom.lib(err80.obj)
                0x000000000000ae7a                error_goto_label
 .text          0x000000000000ae81        0x7 ../lib/freecom.lib(err81.obj)
                0x000000000000ae81                error_get_codepage
 .text          0x000000000000ae88        0x7 ../lib/freecom.lib(err82.obj)
                0x000000000000ae88                error_set_codepage
 .text          0x000000000000ae8f        0x7 ../lib/freecom.lib(err83.obj)
                0x000000000000ae8f                error_copy_plus_destination
 .text          0x000000000000ae96        0xb ../lib/freecom.lib(err84.obj)
                0x000000000000ae96                error_invalid_parameter
 .text          0x000000000000aea1        0xb ../lib/freecom.lib(err85.obj)
                0x000000000000aea1                error_fcom_is_device
 .text          0x000000000000aeac        0xb ../lib/freecom.lib(err86.obj)
                0x000000000000aeac                error_fcom_invalid
 .text          0x000000000000aeb7        0x7 ../lib/freecom.lib(err87.obj)
                0x000000000000aeb7                error_exe_corrupt
 .text          0x000000000000aebe       0x18 ../lib/freecom.lib(almemblk.obj)
                0x000000000000aebe                allocMemBlk
 .text          0x000000000000aed6       0x25 ../lib/freecom.lib(beep_l.obj)
                0x000000000000aed6                beep_low
 .text          0x000000000000aefb       0x23 ../lib/freecom.lib(cbs.obj)
                0x000000000000aefb                cutBackslash
 .text          0x000000000000af1e       0x21 ../lib/freecom.lib(comfile.obj)
                0x000000000000af1e                comFile
 .text          0x000000000000af3f       0x2a ../lib/freecom.lib(ctxt_as.obj)
                0x000000000000af3f                ctxtAddStatus
 .text          0x000000000000af69       0x54 ../lib/freecom.lib(dispexit.obj)
                0x000000000000af69                displayExitcode
 .text          0x000000000000afbd       0x65 ../lib/freecom.lib(inputdos.obj)
                0x000000000000afbd                readcommandDOS
 .text          0x000000000000b022       0x20 ../lib/freecom.lib(ltrimsp.obj)
                0x000000000000b022                ltrimsp
 .text          0x000000000000b042       0x96 ../lib/freecom.lib(mktmpfil.obj)
                0x000000000000b042                mktempfile
 .text          0x000000000000b0d8       0x62 ../lib/freecom.lib(msg_dflt.obj)
                0x000000000000b0d8                defaultMessage
 .text          0x000000000000b13a       0x22 ../lib/freecom.lib(msg_get.obj)
                0x000000000000b13a                getMessage
 .text          0x000000000000b15c       0xe0 ../lib/freecom.lib(parsenum.obj)
                0x000000000000b15c                parsenum
 .text          0x000000000000b23c        0x0 ../strings/strings.lib(str0011.obj)
 .text          0x000000000000b23c        0x0 ../strings/strings.lib(str0018.obj)
 .text          0x000000000000b23c        0x0 ../strings/strings.lib(str003c.obj)
 .text          0x000000000000b23c        0x0 ../strings/strings.lib(str00b1.obj)
 .text          0x000000000000b23c        0x0 ../strings/strings.lib(str00b2.obj)
 .text          0x000000000000b23c        0x0 ../strings/strings.lib(str00f4.obj)
 .text          0x000000000000b23c        0x0 ../strings/strings.lib(str00f5.obj)
 .text          0x000000000000b23c        0x0 ../strings/strings.lib(str00f6.obj)
 .text          0x000000000000b23c       0x12 ../suppl/suppl_s.lib(byte2par.obj)
                0x000000000000b23c                BLK_byte2para
 .text          0x000000000000b24e      0x275 ../suppl/suppl_s.lib(cntry.obj)
                0x000000000000b284                nlsWriteFallback
                0x000000000000b2d5                nlsNewInfo
                0x000000000000b4b3                nlsInfo
 .text          0x000000000000b4c3       0x31 ../suppl/suppl_s.lib(dfnfnam.obj)
                0x000000000000b4c3                dfnfilename
 .text          0x000000000000b4f4       0x9d ../suppl/suppl_s.lib(dfnfullp.obj)
                0x000000000000b4f4                dfnfullpath
 .text          0x000000000000b591      0x101 ../suppl/suppl_s.lib(dfnmerge.obj)
                0x000000000000b591                dfnmerge
 .text          0x000000000000b692       0x4a ../suppl/suppl_s.lib(dfnpath.obj)
                0x000000000000b692                dfnpath
 .text          0x000000000000b6dc       0xa5 ../suppl/suppl_s.lib(dfnstat.obj)
                0x000000000000b6dc                dfnstat
 .text          0x000000000000b781       0x76 ../suppl/suppl_s.lib(dfntruen.obj)
                0x000000000000b781                dfntruename
 .text          0x000000000000b7f7      0x12b ../suppl/suppl_s.lib(dosalloc.obj)
                0x000000000000b7f7                DOSalloc
 .text          0x000000000000b922       0x1d ../suppl/suppl_s.lib(dosfree.obj)
                0x000000000000b922                DOSfree
 .text          0x000000000000b93f       0x2c ../suppl/suppl_s.lib(dossize.obj)
                0x000000000000b93f                DOSresize
 .text          0x000000000000b96b       0x1d ../suppl/suppl_s.lib(dstrfupr.obj)
                0x000000000000b96b                StrFUpr
 .text          0x000000000000b988       0x1c ../suppl/suppl_s.lib(dstrtrim.obj)
                0x000000000000b988                StrTrim
 .text          0x000000000000b9a4       0x1d ../suppl/suppl_s.lib(dstrupr.obj)
                0x000000000000b9a4                StrUpr
 .text          0x000000000000b9c1       0x15 ../suppl/suppl_s.lib(enoallc.obj)
                0x000000000000b9c1                eno_malloc
 .text          0x000000000000b9d6       0x15 ../suppl/suppl_s.lib(enoreal.obj)
                0x000000000000b9d6                eno_realloc
 .text          0x000000000000b9eb        0x1 ../suppl/suppl_s.lib(enosetos.obj)
                0x000000000000b9eb                eno_setOSerror
 .text          0x000000000000b9ec       0x72 ../suppl/suppl_s.lib(env_chg.obj)
                0x000000000000b9ec                env_change
 .text          0x000000000000ba5e       0x79 ../suppl/suppl_s.lib(env_dvar.obj)
                0x000000000000ba5e                env_dupvar
                0x000000000000bad0                dupvar
 .text          0x000000000000bad7       0x70 ../suppl/suppl_s.lib(env_find.obj)
                0x000000000000bad7                env_findVar
 .text          0x000000000000bb47       0x7d ../suppl/suppl_s.lib(env_fora.obj)
                0x000000000000bb47                env_forAll
 .text          0x000000000000bbc4       0x40 ../suppl/suppl_s.lib(env_free.obj)
                0x000000000000bbc4                env_endOfVars
                0x000000000000bbe3                env_firstFree
                0x000000000000bbf2                env_freeCount
 .text          0x000000000000bc04      0x105 ../suppl/suppl_s.lib(env_insv.obj)
                0x000000000000bc04                env_insVarOffset
                0x000000000000bccc                env_appVar
 .text          0x000000000000bd09        0x9 ../suppl/suppl_s.lib(env_len.obj)
                0x000000000000bd09                env_varlen
 .text          0x000000000000bd12       0xf2 ../suppl/suppl_s.lib(env_mtch.obj)
                0x000000000000bd12                env_matchVar
 .text          0x000000000000be04       0x76 ../suppl/suppl_s.lib(env_new.obj)
                0x000000000000be04                env_create
 .text          0x000000000000be7a       0x4a ../suppl/suppl_s.lib(env_nost.obj)
                0x000000000000be7a                env_nullStrings
 .text          0x000000000000bec4      0x11c ../suppl/suppl_s.lib(env_ovrw.obj)
                0x000000000000bec4                env_ovrVarOffset
 .text          0x000000000000bfe0      0x14c ../suppl/suppl_s.lib(env_repl.obj)
                0x000000000000bfe0                env_replace
 .text          0x000000000000c12c       0x27 ../suppl/suppl_s.lib(env_rlsg.obj)
                0x000000000000c12c                env_relocateSegment
 .text          0x000000000000c153       0x61 ../suppl/suppl_s.lib(env_scnt.obj)
                0x000000000000c153                env_strcounter
 .text          0x000000000000c1b4      0x110 ../suppl/suppl_s.lib(env_size.obj)
                0x000000000000c1b4                env_setsize
                0x000000000000c267                env_resize
 .text          0x000000000000c2c4       0x79 ../suppl/suppl_s.lib(env_strg.obj)
                0x000000000000c2c4                env_string
 .text          0x000000000000c33d       0x2b ../suppl/suppl_s.lib(env_sub.obj)
                0x000000000000c33d                env_subVarOffset
 .text          0x000000000000c368        0x0 ../suppl/suppl_s.lib(env_var1.obj)
 .text          0x000000000000c368        0x0 ../suppl/suppl_s.lib(env_var2.obj)
 .text          0x000000000000c368       0x2a ../suppl/suppl_s.lib(fstrdup.obj)
                0x000000000000c368                _fdupstr
 .text          0x000000000000c392       0x14 ../suppl/suppl_s.lib(mcb_is.obj)
                0x000000000000c39c                isMCB
 .text          0x000000000000c3a6       0x1f ../suppl/suppl_s.lib(mcb_leng.obj)
                0x000000000000c3a6                mcb_length
 .text          0x000000000000c3c5       0x1a ../suppl/suppl_s.lib(mcb_nxt.obj)
                0x000000000000c3c5                nxtMCB
 .text          0x000000000000c3df       0xae ../suppl/suppl_s.lib(mcb_walk.obj)
                0x000000000000c3df                mcb_walk
 .text          0x000000000000c48d       0x5f ../suppl/suppl_s.lib(toupperx.obj)
                0x000000000000c48d                toFUpper
                0x000000000000c4bd                toUpper
 .text          0x000000000000c4ec       0x6b ../suppl/suppl_s.lib(filefind.obj)
                0x000000000000c4ec                findfirst
                0x000000000000c527                findnext
 .text          0x000000000000c557       0x16 ../suppl/suppl_s.lib(invokedo.obj)
                0x000000000000c557                invokeDOS
 *fill*         0x000000000000c56d        0x3 
 .text          0x000000000000c570       0x64 ../suppl/suppl_s.lib(intr.obj)
                0x000000000000c570                _intrf
                0x000000000000c570                intrf
 .text          0x000000000000c5d4        0x7 ../suppl/suppl_s.lib(addu.obj)
                0x000000000000c5d4                addu
 .text          0x000000000000c5db       0x33 ../suppl/suppl_s.lib(dfndeli2.obj)
                0x000000000000c5db                dfndelim2
 .text          0x000000000000c60e       0x20 ../suppl/suppl_s.lib(dfndelim.obj)
                0x000000000000c60e                dfndelim
 .text          0x000000000000c62e      0x17d ../suppl/suppl_s.lib(dfnexpan.obj)
                0x000000000000c62e                dfnexpand
 .text          0x000000000000c7ab      0x15c ../suppl/suppl_s.lib(dfnsplit.obj)
                0x000000000000c7ab                dfnsplit
 .text          0x000000000000c907       0x75 ../suppl/suppl_s.lib(dfnsquee.obj)
                0x000000000000c907                dfnsqueeze
 .text          0x000000000000c97c       0x7d ../suppl/suppl_s.lib(dmemcmpf.obj)
                0x000000000000c97c                _fMemiCmp
 .text          0x000000000000c9f9       0x19 ../suppl/suppl_s.lib(dstrchar.obj)
                0x000000000000c9f9                StrChar
 .text          0x000000000000ca12       0x3f ../suppl/suppl_s.lib(dstrleft.obj)
                0x000000000000ca12                StrLeft
 .text          0x000000000000ca51       0x10 ../suppl/suppl_s.lib(dstrrepl.obj)
                0x000000000000ca51                StrRepl_
 .text          0x000000000000ca61       0x1d ../suppl/suppl_s.lib(enosdup.obj)
                0x000000000000ca61                eno_strdup
 .text          0x000000000000ca7e       0x3d ../suppl/suppl_s.lib(env_del.obj)
                0x000000000000ca7e                env_delete
 .text          0x000000000000cabb       0x2d ../suppl/suppl_s.lib(mcb_1st.obj)
                0x000000000000cabb                mcb_first
 .text          0x000000000000cae8       0x1f /home/evln/proj/build-ia16.202501/prefix/bin/../lib/gcc/ia16-elf/6.3.0/../../../../ia16-elf/lib/regparmcall/libi86.a(fmemchr.o)
                0x000000000000cae8                _fmemchr
 .text          0x000000000000cb07       0x37 /home/evln/proj/build-ia16.202501/prefix/bin/../lib/gcc/ia16-elf/6.3.0/../../../../ia16-elf/lib/regparmcall/libi86.a(fmemcmp.o)
                0x000000000000cb07                _fmemcmp
 .text          0x000000000000cb3e       0x1f /home/evln/proj/build-ia16.202501/prefix/bin/../lib/gcc/ia16-elf/6.3.0/../../../../ia16-elf/lib/regparmcall/libi86.a(fmemcpy.o)
                0x000000000000cb3e                _fmemcpy
                0x000000000000cb3e                __libi86_fmemmove_forward
 .text          0x000000000000cb5d      0x165 /home/evln/proj/build-ia16.202501/prefix/bin/../lib/gcc/ia16-elf/6.3.0/../../../../ia16-elf/lib/regparmcall/libi86.a(fmemmove.o)
                0x000000000000cb5d                _fmemmove
 .text          0x000000000000ccc2       0x1d /home/evln/proj/build-ia16.202501/prefix/bin/../lib/gcc/ia16-elf/6.3.0/../../../../ia16-elf/lib/regparmcall/libi86.a(fstrcpy.o)
                0x000000000000ccc2                _fstrcpy
 .text          0x000000000000ccdf       0x18 /home/evln/proj/build-ia16.202501/prefix/bin/../lib/gcc/ia16-elf/6.3.0/../../../../ia16-elf/lib/regparmcall/libi86.a(fstrlen.o)
                0x000000000000ccdf                _fstrlen
 .text          0x000000000000ccf7       0x2b /home/evln/proj/build-ia16.202501/prefix/bin/../lib/gcc/ia16-elf/6.3.0/../../../../ia16-elf/lib/regparmcall/libi86.a(libi86-fmemmove-backward.o)
                0x000000000000ccf7                __libi86_fmemmove_backward
 .text          0x000000000000cd22       0xc4 /home/evln/proj/build-ia16.202501/prefix/bin/../lib/gcc/ia16-elf/6.3.0/../../../../ia16-elf/lib/regparmcall/libi86.a(getdcwd.o)
                0x000000000000cd6a                _getdcwd
 .text          0x000000000000cde6        0x8 /home/evln/proj/build-ia16.202501/prefix/bin/../lib/gcc/ia16-elf/6.3.0/../../../../ia16-elf/lib/regparmcall/libi86.a(getdrive.o)
                0x000000000000cde6                _getdrive
 .text          0x000000000000cdee       0x38 /home/evln/proj/build-ia16.202501/prefix/bin/../lib/gcc/ia16-elf/6.3.0/regparmcall/crtbegin.o
 .text          0x000000000000ce26       0x1b /home/evln/proj/build-ia16.202501/prefix/bin/../lib/gcc/ia16-elf/6.3.0/regparmcall/crtend.o
 .text          0x000000000000ce41        0x0 /home/evln/proj/build-ia16.202501/prefix/bin/../lib/gcc/ia16-elf/6.3.0/../../../../ia16-elf/lib/regparmcall/dos-s-c0.o
 .text          0x000000000000ce41        0xa /home/evln/proj/build-ia16.202501/prefix/bin/../lib/gcc/ia16-elf/6.3.0/../../../../ia16-elf/lib/regparmcall/libc.a(lib_a-atexit.o)
                0x000000000000ce41                atexit
 .text          0x000000000000ce4b       0x12 /home/evln/proj/build-ia16.202501/prefix/bin/../lib/gcc/ia16-elf/6.3.0/../../../../ia16-elf/lib/regparmcall/libc.a(lib_a-atol.o)
                0x000000000000ce4b                atol
                0x000000000000ce53                _atol_r
 .text          0x000000000000ce5d        0x7 /home/evln/proj/build-ia16.202501/prefix/bin/../lib/gcc/ia16-elf/6.3.0/../../../../ia16-elf/lib/regparmcall/libc.a(lib_a-ctype_.o)
                0x000000000000ce5d                __set_ctype
 .text          0x000000000000ce64        0x4 /home/evln/proj/build-ia16.202501/prefix/bin/../lib/gcc/ia16-elf/6.3.0/../../../../ia16-elf/lib/regparmcall/libc.a(lib_a-errno.o)
                0x000000000000ce64                __errno
 .text          0x000000000000ce68       0x1a /home/evln/proj/build-ia16.202501/prefix/bin/../lib/gcc/ia16-elf/6.3.0/../../../../ia16-elf/lib/regparmcall/libc.a(lib_a-exit.o)
                0x000000000000ce68                exit
 .text          0x000000000000ce82        0x0 /home/evln/proj/build-ia16.202501/prefix/bin/../lib/gcc/ia16-elf/6.3.0/../../../../ia16-elf/lib/regparmcall/libc.a(lib_a-impure.o)
 .text          0x000000000000ce82        0xe /home/evln/proj/build-ia16.202501/prefix/bin/../lib/gcc/ia16-elf/6.3.0/../../../../ia16-elf/lib/regparmcall/libc.a(lib_a-malloc.o)
                0x000000000000ce82                malloc
                0x000000000000ce89                free
 .text          0x000000000000ce90       0x19 /home/evln/proj/build-ia16.202501/prefix/bin/../lib/gcc/ia16-elf/6.3.0/../../../../ia16-elf/lib/regparmcall/libc.a(lib_a-memchr.o)
                0x000000000000ce90                memchr
 .text          0x000000000000cea9       0x53 /home/evln/proj/build-ia16.202501/prefix/bin/../lib/gcc/ia16-elf/6.3.0/../../../../ia16-elf/lib/regparmcall/libc.a(lib_a-memcmp.o)
                0x000000000000cea9                memcmp
 .text          0x000000000000cefc       0x17 /home/evln/proj/build-ia16.202501/prefix/bin/../lib/gcc/ia16-elf/6.3.0/../../../../ia16-elf/lib/regparmcall/libc.a(lib_a-memcpy.o)
                0x000000000000cefc                memcpy
 .text          0x000000000000cf13       0x4d /home/evln/proj/build-ia16.202501/prefix/bin/../lib/gcc/ia16-elf/6.3.0/../../../../ia16-elf/lib/regparmcall/libc.a(lib_a-memmove.o)
                0x000000000000cf13                memmove
 .text          0x000000000000cf60       0x1b /home/evln/proj/build-ia16.202501/prefix/bin/../lib/gcc/ia16-elf/6.3.0/../../../../ia16-elf/lib/regparmcall/libc.a(lib_a-memset.o)
                0x000000000000cf60                memset
 .text          0x000000000000cf7b       0xc6 /home/evln/proj/build-ia16.202501/prefix/bin/../lib/gcc/ia16-elf/6.3.0/../../../../ia16-elf/lib/regparmcall/libc.a(lib_a-nano-freer.o)
                0x000000000000cf7b                _free_r
 .text          0x000000000000d041      0x13b /home/evln/proj/build-ia16.202501/prefix/bin/../lib/gcc/ia16-elf/6.3.0/../../../../ia16-elf/lib/regparmcall/libc.a(lib_a-nano-mallocr.o)
                0x000000000000d041                _malloc_r
 .text          0x000000000000d17c      0x484 /home/evln/proj/build-ia16.202501/prefix/bin/../lib/gcc/ia16-elf/6.3.0/../../../../ia16-elf/lib/regparmcall/libc.a(lib_a-qsort.o)
                0x000000000000d252                qsort
 .text          0x000000000000d600        0x9 /home/evln/proj/build-ia16.202501/prefix/bin/../lib/gcc/ia16-elf/6.3.0/../../../../ia16-elf/lib/regparmcall/libc.a(lib_a-realloc.o)
                0x000000000000d600                realloc
 .text          0x000000000000d609       0x10 /home/evln/proj/build-ia16.202501/prefix/bin/../lib/gcc/ia16-elf/6.3.0/../../../../ia16-elf/lib/regparmcall/libc.a(lib_a-remove.o)
                0x000000000000d609                _remove_r
                0x000000000000d613                remove
 .text          0x000000000000d619       0x5f /home/evln/proj/build-ia16.202501/prefix/bin/../lib/gcc/ia16-elf/6.3.0/../../../../ia16-elf/lib/regparmcall/libc.a(lib_a-setjmp.o)
                0x000000000000d619                setjmp
                0x000000000000d64d                longjmp
 .text          0x000000000000d678       0x18 /home/evln/proj/build-ia16.202501/prefix/bin/../lib/gcc/ia16-elf/6.3.0/../../../../ia16-elf/lib/regparmcall/libc.a(lib_a-stpcpy.o)
                0x000000000000d678                stpcpy
 .text          0x000000000000d690       0x6f /home/evln/proj/build-ia16.202501/prefix/bin/../lib/gcc/ia16-elf/6.3.0/../../../../ia16-elf/lib/regparmcall/libc.a(lib_a-strcasecmp.o)
                0x000000000000d690                strcasecmp
 .text          0x000000000000d6ff       0x1c /home/evln/proj/build-ia16.202501/prefix/bin/../lib/gcc/ia16-elf/6.3.0/../../../../ia16-elf/lib/regparmcall/libc.a(lib_a-strcat.o)
                0x000000000000d6ff                strcat
 .text          0x000000000000d71b       0x17 /home/evln/proj/build-ia16.202501/prefix/bin/../lib/gcc/ia16-elf/6.3.0/../../../../ia16-elf/lib/regparmcall/libc.a(lib_a-strchr.o)
                0x000000000000d71b                strchr
 .text          0x000000000000d732       0x1a /home/evln/proj/build-ia16.202501/prefix/bin/../lib/gcc/ia16-elf/6.3.0/../../../../ia16-elf/lib/regparmcall/libc.a(lib_a-strcmp.o)
                0x000000000000d732                strcmp
 .text          0x000000000000d74c       0x19 /home/evln/proj/build-ia16.202501/prefix/bin/../lib/gcc/ia16-elf/6.3.0/../../../../ia16-elf/lib/regparmcall/libc.a(lib_a-strcpy.o)
                0x000000000000d74c                strcpy
 .text          0x000000000000d765        0x7 /home/evln/proj/build-ia16.202501/prefix/bin/../lib/gcc/ia16-elf/6.3.0/../../../../ia16-elf/lib/regparmcall/libc.a(lib_a-strdup.o)
                0x000000000000d765                strdup
 .text          0x000000000000d76c       0x2c /home/evln/proj/build-ia16.202501/prefix/bin/../lib/gcc/ia16-elf/6.3.0/../../../../ia16-elf/lib/regparmcall/libc.a(lib_a-strdup_r.o)
                0x000000000000d76c                _strdup_r
 .text          0x000000000000d798       0x19 /home/evln/proj/build-ia16.202501/prefix/bin/../lib/gcc/ia16-elf/6.3.0/../../../../ia16-elf/lib/regparmcall/libc.a(lib_a-strlen.o)
                0x000000000000d798                strlen
 .text          0x000000000000d7b1       0x30 /home/evln/proj/build-ia16.202501/prefix/bin/../lib/gcc/ia16-elf/6.3.0/../../../../ia16-elf/lib/regparmcall/libc.a(lib_a-strlwr.o)
                0x000000000000d7b1                strlwr
 .text          0x000000000000d7e1       0x76 /home/evln/proj/build-ia16.202501/prefix/bin/../lib/gcc/ia16-elf/6.3.0/../../../../ia16-elf/lib/regparmcall/libc.a(lib_a-strncasecmp.o)
                0x000000000000d7e1                strncasecmp
 .text          0x000000000000d857       0x25 /home/evln/proj/build-ia16.202501/prefix/bin/../lib/gcc/ia16-elf/6.3.0/../../../../ia16-elf/lib/regparmcall/libc.a(lib_a-strncpy.o)
                0x000000000000d857                strncpy
 .text          0x000000000000d87c       0x2f /home/evln/proj/build-ia16.202501/prefix/bin/../lib/gcc/ia16-elf/6.3.0/../../../../ia16-elf/lib/regparmcall/libc.a(lib_a-strpbrk.o)
                0x000000000000d87c                strpbrk
 .text          0x000000000000d8ab       0x27 /home/evln/proj/build-ia16.202501/prefix/bin/../lib/gcc/ia16-elf/6.3.0/../../../../ia16-elf/lib/regparmcall/libc.a(lib_a-strrchr.o)
                0x000000000000d8ab                strrchr
 .text          0x000000000000d8d2       0x2b /home/evln/proj/build-ia16.202501/prefix/bin/../lib/gcc/ia16-elf/6.3.0/../../../../ia16-elf/lib/regparmcall/libc.a(lib_a-strspn.o)
                0x000000000000d8d2                strspn
 .text          0x000000000000d8fd       0x8f /home/evln/proj/build-ia16.202501/prefix/bin/../lib/gcc/ia16-elf/6.3.0/../../../../ia16-elf/lib/regparmcall/libc.a(lib_a-strtok.o)
                0x000000000000d8fd                strtok
 .text          0x000000000000d98c       0x8d /home/evln/proj/build-ia16.202501/prefix/bin/../lib/gcc/ia16-elf/6.3.0/../../../../ia16-elf/lib/regparmcall/libc.a(lib_a-strtok_r.o)
                0x000000000000d98c                __strtok_r
                0x000000000000da11                strtok_r
 .text          0x000000000000da19      0x244 /home/evln/proj/build-ia16.202501/prefix/bin/../lib/gcc/ia16-elf/6.3.0/../../../../ia16-elf/lib/regparmcall/libc.a(lib_a-strtol.o)
                0x000000000000da19                _strtol_r
                0x000000000000dc52                strtol
 .text          0x000000000000dc5d        0x7 /home/evln/proj/build-ia16.202501/prefix/bin/../lib/gcc/ia16-elf/6.3.0/../../../../ia16-elf/lib/regparmcall/libc.a(lib_a-sysisatty.o)
                0x000000000000dc5d                isatty
 .text          0x000000000000dc64       0x15 /home/evln/proj/build-ia16.202501/prefix/bin/../lib/gcc/ia16-elf/6.3.0/../../../../ia16-elf/lib/regparmcall/libc.a(lib_a-syslseek.o)
                0x000000000000dc64                lseek
 .text          0x000000000000dc79        0x7 /home/evln/proj/build-ia16.202501/prefix/bin/../lib/gcc/ia16-elf/6.3.0/../../../../ia16-elf/lib/regparmcall/libc.a(lib_a-sysunlink.o)
                0x000000000000dc79                unlink
 .text          0x000000000000dc80        0xb /home/evln/proj/build-ia16.202501/prefix/bin/../lib/gcc/ia16-elf/6.3.0/../../../../ia16-elf/lib/regparmcall/libc.a(lib_a-syswrite.o)
                0x000000000000dc80                write
 .text          0x000000000000dc8b       0x17 /home/evln/proj/build-ia16.202501/prefix/bin/../lib/gcc/ia16-elf/6.3.0/../../../../ia16-elf/lib/regparmcall/libc.a(lib_a-toupper.o)
                0x000000000000dc8b                toupper
 .text          0x000000000000dca2      0x108 /home/evln/proj/build-ia16.202501/prefix/bin/../lib/gcc/ia16-elf/6.3.0/../../../../ia16-elf/lib/regparmcall/libc.a(lib_a-__atexit.o)
                0x000000000000dca2                __register_exitproc
 .text          0x000000000000ddaa      0x12f /home/evln/proj/build-ia16.202501/prefix/bin/../lib/gcc/ia16-elf/6.3.0/../../../../ia16-elf/lib/regparmcall/libc.a(lib_a-__call_atexit.o)
                0x000000000000ddaa                __call_exitprocs
 .text          0x000000000000ded9       0x5d /home/evln/proj/build-ia16.202501/prefix/bin/../lib/gcc/ia16-elf/6.3.0/../../../../ia16-elf/lib/regparmcall/libc.a(lib_a-nano-reallocr.o)
                0x000000000000ded9                _realloc_r
 .text          0x000000000000df36       0x1a /home/evln/proj/build-ia16.202501/prefix/bin/../lib/gcc/ia16-elf/6.3.0/../../../../ia16-elf/lib/regparmcall/libc.a(lib_a-nano-msizer.o)
                0x000000000000df36                _malloc_usable_size_r
 .text          0x000000000000df50        0xb /home/evln/proj/build-ia16.202501/prefix/bin/../lib/gcc/ia16-elf/6.3.0/regparmcall/libgcc.a(udivsi3.o)
                0x000000000000df50                __udivsi3
 .text          0x000000000000df5b       0x10 /home/evln/proj/build-ia16.202501/prefix/bin/../lib/gcc/ia16-elf/6.3.0/regparmcall/libgcc.a(umodsi3.o)
                0x000000000000df5b                __umodsi3
 .text          0x000000000000df6b       0x4f /home/evln/proj/build-ia16.202501/prefix/bin/../lib/gcc/ia16-elf/6.3.0/regparmcall/libgcc.a(ia16-ldivmodu.o)
                0x000000000000df6b                __ia16_ldivmodu
 .text          0x000000000000dfba       0x1c /home/evln/proj/build-ia16.202501/prefix/bin/../lib/gcc/ia16-elf/6.3.0/../../../../ia16-elf/lib/regparmcall/libdos-s.a(dos-isattyr.o)
                0x000000000000dfba                _isatty_r
 .text          0x000000000000dfd6       0x1d /home/evln/proj/build-ia16.202501/prefix/bin/../lib/gcc/ia16-elf/6.3.0/../../../../ia16-elf/lib/regparmcall/libdos-s.a(dos-lseekr.o)
                0x000000000000dfd6                _lseek_r
 .text          0x000000000000dff3       0x4a /home/evln/proj/build-ia16.202501/prefix/bin/../lib/gcc/ia16-elf/6.3.0/../../../../ia16-elf/lib/regparmcall/libdos-s.a(dos-sbrkr.o)
                0x000000000000dff3                _sbrk_r
 .text          0x000000000000e03d       0x11 /home/evln/proj/build-ia16.202501/prefix/bin/../lib/gcc/ia16-elf/6.3.0/../../../../ia16-elf/lib/regparmcall/libdos-s.a(dos-unlinkr.o)
                0x000000000000e03d                _unlink_r
 .text          0x000000000000e04e       0x1f /home/evln/proj/build-ia16.202501/prefix/bin/../lib/gcc/ia16-elf/6.3.0/../../../../ia16-elf/lib/regparmcall/libdos-s.a(dos-writer.o)
                0x000000000000e04e                _write_r
 .text          0x000000000000e06d       0x2d /home/evln/proj/build-ia16.202501/prefix/bin/../lib/gcc/ia16-elf/6.3.0/../../../../ia16-elf/lib/regparmcall/libdos-s.a(dos-msmmabort.o)
                0x000000000000e06d                abort
 .text          0x000000000000e09a        0x0 /home/evln/proj/build-ia16.202501/prefix/bin/../lib/gcc/ia16-elf/6.3.0/../../../../ia16-elf/lib/regparmcall/libdos-s.a(dos-heaplen.o)
 .text          0x000000000000e09a        0x2 /home/evln/proj/build-ia16.202501/prefix/bin/../lib/gcc/ia16-elf/6.3.0/../../../../ia16-elf/lib/regparmcall/libdos-s.a(dos-near-data-segment.o)
                0x000000000000e09a                __ia16_near_data_segment
 .text          0x000000000000e09c       0xb1 /home/evln/proj/build-ia16.202501/prefix/bin/../lib/gcc/ia16-elf/6.3.0/../../../../ia16-elf/lib/regparmcall/libc.a(lib_a-abort.o)
                0x000000000000e10d                __ia16_abort_impl
 *(.text.*)
 .text.startup  0x000000000000e14d       0x41 command.obj
                0x000000000000e14d                main
                0x000000000000e18e                __etext = .
                0x000000000000e190                . = ALIGN (0x10)
 *fill*         0x000000000000e18e        0x2 
                0x000000000000e190                __etext_padded = .
                0x0000000000000001                ASSERT ((. <= 0x10000), Error: too large for a small or medium model .exe file.)
                0x000000000000e16e                __ltext = (__etext - __stext)
                0x000000000000e170                __ltext_padded = (__etext_padded - __stext)

.fartext.00$    0x0000000000000000        0x0 load address 0x000000000000e220
 *(.fartext.*00 .fartext.*00$)
                0x0000000000000000                . = ALIGN (0x10)

.fartext.01$    0x0000000000000000        0x0 load address 0x000000000000e220
 *(.fartext.*01 .fartext.*01$)
                0x0000000000000000                . = ALIGN (0x10)

.fartext.02$    0x0000000000000000        0x0 load address 0x000000000000e220
 *(.fartext.*02 .fartext.*02$)
                0x0000000000000000                . = ALIGN (0x10)

.fartext.03$    0x0000000000000000        0x0 load address 0x000000000000e220
 *(.fartext.*03 .fartext.*03$)
                0x0000000000000000                . = ALIGN (0x10)

.fartext.04$    0x0000000000000000        0x0 load address 0x000000000000e220
 *(.fartext.*04 .fartext.*04$)
                0x0000000000000000                . = ALIGN (0x10)

.fartext.05$    0x0000000000000000        0x0 load address 0x000000000000e220
 *(.fartext.*05 .fartext.*05$)
                0x0000000000000000                . = ALIGN (0x10)

.fartext.06$    0x0000000000000000        0x0 load address 0x000000000000e220
 *(.fartext.*06 .fartext.*06$)
                0x0000000000000000                . = ALIGN (0x10)

.fartext.07$    0x0000000000000000        0x0 load address 0x000000000000e220
 *(.fartext.*07 .fartext.*07$)
                0x0000000000000000                . = ALIGN (0x10)

.fartext.10$    0x0000000000000000        0x0 load address 0x000000000000e220
 *(.fartext.*10 .fartext.*10$)
                0x0000000000000000                . = ALIGN (0x10)

.fartext.11$    0x0000000000000000        0x0 load address 0x000000000000e220
 *(.fartext.*11 .fartext.*11$)
                0x0000000000000000                . = ALIGN (0x10)

.fartext.12$    0x0000000000000000        0x0 load address 0x000000000000e220
 *(.fartext.*12 .fartext.*12$)
                0x0000000000000000                . = ALIGN (0x10)

.fartext.13$    0x0000000000000000        0x0 load address 0x000000000000e220
 *(.fartext.*13 .fartext.*13$)
                0x0000000000000000                . = ALIGN (0x10)

.fartext.14$    0x0000000000000000        0x0 load address 0x000000000000e220
 *(.fartext.*14 .fartext.*14$)
                0x0000000000000000                . = ALIGN (0x10)

.fartext.15$    0x0000000000000000        0x0 load address 0x000000000000e220
 *(.fartext.*15 .fartext.*15$)
                0x0000000000000000                . = ALIGN (0x10)

.fartext.16$    0x0000000000000000        0x0 load address 0x000000000000e220
 *(.fartext.*16 .fartext.*16$)
                0x0000000000000000                . = ALIGN (0x10)

.fartext.17$    0x0000000000000000        0x0 load address 0x000000000000e220
 *(.fartext.*17 .fartext.*17$)
                0x0000000000000000                . = ALIGN (0x10)

.fartext.20$    0x0000000000000000        0x0 load address 0x000000000000e220
 *(.fartext.*20 .fartext.*20$)
                0x0000000000000000                . = ALIGN (0x10)

.fartext.21$    0x0000000000000000        0x0 load address 0x000000000000e220
 *(.fartext.*21 .fartext.*21$)
                0x0000000000000000                . = ALIGN (0x10)

.fartext.22$    0x0000000000000000        0x0 load address 0x000000000000e220
 *(.fartext.*22 .fartext.*22$)
                0x0000000000000000                . = ALIGN (0x10)

.fartext.23$    0x0000000000000000        0x0 load address 0x000000000000e220
 *(.fartext.*23 .fartext.*23$)
                0x0000000000000000                . = ALIGN (0x10)

.fartext.24$    0x0000000000000000        0x0 load address 0x000000000000e220
 *(.fartext.*24 .fartext.*24$)
                0x0000000000000000                . = ALIGN (0x10)

.fartext.25$    0x0000000000000000        0x0 load address 0x000000000000e220
 *(.fartext.*25 .fartext.*25$)
                0x0000000000000000                . = ALIGN (0x10)

.fartext.26$    0x0000000000000000        0x0 load address 0x000000000000e220
 *(.fartext.*26 .fartext.*26$)
                0x0000000000000000                . = ALIGN (0x10)

.fartext.27$    0x0000000000000000        0x0 load address 0x000000000000e220
 *(.fartext.*27 .fartext.*27$)
                0x0000000000000000                . = ALIGN (0x10)

.fartext.30$    0x0000000000000000        0x0 load address 0x000000000000e220
 *(.fartext.*30 .fartext.*30$)
                0x0000000000000000                . = ALIGN (0x10)

.fartext.31$    0x0000000000000000        0x0 load address 0x000000000000e220
 *(.fartext.*31 .fartext.*31$)
                0x0000000000000000                . = ALIGN (0x10)

.fartext.32$    0x0000000000000000        0x0 load address 0x000000000000e220
 *(.fartext.*32 .fartext.*32$)
                0x0000000000000000                . = ALIGN (0x10)

.fartext.33$    0x0000000000000000        0x0 load address 0x000000000000e220
 *(.fartext.*33 .fartext.*33$)
                0x0000000000000000                . = ALIGN (0x10)

.fartext.34$    0x0000000000000000        0x0 load address 0x000000000000e220
 *(.fartext.*34 .fartext.*34$)
                0x0000000000000000                . = ALIGN (0x10)

.fartext.35$    0x0000000000000000        0x0 load address 0x000000000000e220
 *(.fartext.*35 .fartext.*35$)
                0x0000000000000000                . = ALIGN (0x10)

.fartext.36$    0x0000000000000000        0x0 load address 0x000000000000e220
 *(.fartext.*36 .fartext.*36$)
                0x0000000000000000                . = ALIGN (0x10)

.fartext.37$    0x0000000000000000        0x0 load address 0x000000000000e220
 *(.fartext.*37 .fartext.*37$)
                0x0000000000000000                . = ALIGN (0x10)

.fartext.40$    0x0000000000000000        0x0 load address 0x000000000000e220
 *(.fartext.*40 .fartext.*40$)
                0x0000000000000000                . = ALIGN (0x10)

.fartext.41$    0x0000000000000000        0x0 load address 0x000000000000e220
 *(.fartext.*41 .fartext.*41$)
                0x0000000000000000                . = ALIGN (0x10)

.fartext.42$    0x0000000000000000        0x0 load address 0x000000000000e220
 *(.fartext.*42 .fartext.*42$)
                0x0000000000000000                . = ALIGN (0x10)

.fartext.43$    0x0000000000000000        0x0 load address 0x000000000000e220
 *(.fartext.*43 .fartext.*43$)
                0x0000000000000000                . = ALIGN (0x10)

.fartext.44$    0x0000000000000000        0x0 load address 0x000000000000e220
 *(.fartext.*44 .fartext.*44$)
                0x0000000000000000                . = ALIGN (0x10)

.fartext.45$    0x0000000000000000        0x0 load address 0x000000000000e220
 *(.fartext.*45 .fartext.*45$)
                0x0000000000000000                . = ALIGN (0x10)

.fartext.46$    0x0000000000000000        0x0 load address 0x000000000000e220
 *(.fartext.*46 .fartext.*46$)
                0x0000000000000000                . = ALIGN (0x10)

.fartext.47$    0x0000000000000000        0x0 load address 0x000000000000e220
 *(.fartext.*47 .fartext.*47$)
                0x0000000000000000                . = ALIGN (0x10)

.fartext.50$    0x0000000000000000        0x0 load address 0x000000000000e220
 *(.fartext.*50 .fartext.*50$)
                0x0000000000000000                . = ALIGN (0x10)

.fartext.51$    0x0000000000000000        0x0 load address 0x000000000000e220
 *(.fartext.*51 .fartext.*51$)
                0x0000000000000000                . = ALIGN (0x10)

.fartext.52$    0x0000000000000000        0x0 load address 0x000000000000e220
 *(.fartext.*52 .fartext.*52$)
                0x0000000000000000                . = ALIGN (0x10)

.fartext.53$    0x0000000000000000        0x0 load address 0x000000000000e220
 *(.fartext.*53 .fartext.*53$)
                0x0000000000000000                . = ALIGN (0x10)

.fartext.54$    0x0000000000000000        0x0 load address 0x000000000000e220
 *(.fartext.*54 .fartext.*54$)
                0x0000000000000000                . = ALIGN (0x10)

.fartext.55$    0x0000000000000000        0x0 load address 0x000000000000e220
 *(.fartext.*55 .fartext.*55$)
                0x0000000000000000                . = ALIGN (0x10)

.fartext.56$    0x0000000000000000        0x0 load address 0x000000000000e220
 *(.fartext.*56 .fartext.*56$)
                0x0000000000000000                . = ALIGN (0x10)

.fartext.57$    0x0000000000000000        0x0 load address 0x000000000000e220
 *(.fartext.*57 .fartext.*57$)
                0x0000000000000000                . = ALIGN (0x10)

.fartext.60$    0x0000000000000000        0x0 load address 0x000000000000e220
 *(.fartext.*60 .fartext.*60$)
                0x0000000000000000                . = ALIGN (0x10)

.fartext.61$    0x0000000000000000        0x0 load address 0x000000000000e220
 *(.fartext.*61 .fartext.*61$)
                0x0000000000000000                . = ALIGN (0x10)

.fartext.62$    0x0000000000000000        0x0 load address 0x000000000000e220
 *(.fartext.*62 .fartext.*62$)
                0x0000000000000000                . = ALIGN (0x10)

.fartext.63$    0x0000000000000000        0x0 load address 0x000000000000e220
 *(.fartext.*63 .fartext.*63$)
                0x0000000000000000                . = ALIGN (0x10)

.fartext.64$    0x0000000000000000        0x0 load address 0x000000000000e220
 *(.fartext.*64 .fartext.*64$)
                0x0000000000000000                . = ALIGN (0x10)

.fartext.65$    0x0000000000000000        0x0 load address 0x000000000000e220
 *(.fartext.*65 .fartext.*65$)
                0x0000000000000000                . = ALIGN (0x10)

.fartext.66$    0x0000000000000000        0x0 load address 0x000000000000e220
 *(.fartext.*66 .fartext.*66$)
                0x0000000000000000                . = ALIGN (0x10)

.fartext.67$    0x0000000000000000        0x0 load address 0x000000000000e220
 *(.fartext.*67 .fartext.*67$)
                0x0000000000000000                . = ALIGN (0x10)

.fartext.70$    0x0000000000000000        0x0 load address 0x000000000000e220
 *(.fartext.*70 .fartext.*70$)
                0x0000000000000000                . = ALIGN (0x10)

.fartext.71$    0x0000000000000000        0x0 load address 0x000000000000e220
 *(.fartext.*71 .fartext.*71$)
                0x0000000000000000                . = ALIGN (0x10)

.fartext.72$    0x0000000000000000        0x0 load address 0x000000000000e220
 *(.fartext.*72 .fartext.*72$)
                0x0000000000000000                . = ALIGN (0x10)

.fartext.73$    0x0000000000000000        0x0 load address 0x000000000000e220
 *(.fartext.*73 .fartext.*73$)
                0x0000000000000000                . = ALIGN (0x10)

.fartext.74$    0x0000000000000000        0x0 load address 0x000000000000e220
 *(.fartext.*74 .fartext.*74$)
                0x0000000000000000                . = ALIGN (0x10)

.fartext.75$    0x0000000000000000        0x0 load address 0x000000000000e220
 *(.fartext.*75 .fartext.*75$)
                0x0000000000000000                . = ALIGN (0x10)

.fartext.76$    0x0000000000000000        0x0 load address 0x000000000000e220
 *(.fartext.*76 .fartext.*76$)
                0x0000000000000000                . = ALIGN (0x10)

.fartext.77$    0x0000000000000000        0x0 load address 0x000000000000e220
 *(.fartext.*77 .fartext.*77$)
                0x0000000000000000                . = ALIGN (0x10)

.fartext.XX$    0x0000000000000000        0x0 load address 0x000000000000e220
 *(.fartext .fartext$ .fartext.*)
                0x0000000000000000                . = ALIGN (0x10)

.farrodata.00$  0x0000000000000000        0x0 load address 0x000000000000e220
 *(.farrodata.*00 .farrodata.*00$)
                0x0000000000000000                . = ALIGN (0x10)

.farrodata.01$  0x0000000000000000        0x0 load address 0x000000000000e220
 *(.farrodata.*01 .farrodata.*01$)
                0x0000000000000000                . = ALIGN (0x10)

.farrodata.02$  0x0000000000000000        0x0 load address 0x000000000000e220
 *(.farrodata.*02 .farrodata.*02$)
                0x0000000000000000                . = ALIGN (0x10)

.farrodata.03$  0x0000000000000000        0x0 load address 0x000000000000e220
 *(.farrodata.*03 .farrodata.*03$)
                0x0000000000000000                . = ALIGN (0x10)

.farrodata.04$  0x0000000000000000        0x0 load address 0x000000000000e220
 *(.farrodata.*04 .farrodata.*04$)
                0x0000000000000000                . = ALIGN (0x10)

.farrodata.05$  0x0000000000000000        0x0 load address 0x000000000000e220
 *(.farrodata.*05 .farrodata.*05$)
                0x0000000000000000                . = ALIGN (0x10)

.farrodata.06$  0x0000000000000000        0x0 load address 0x000000000000e220
 *(.farrodata.*06 .farrodata.*06$)
                0x0000000000000000                . = ALIGN (0x10)

.farrodata.07$  0x0000000000000000        0x0 load address 0x000000000000e220
 *(.farrodata.*07 .farrodata.*07$)
                0x0000000000000000                . = ALIGN (0x10)

.farrodata.10$  0x0000000000000000        0x0 load address 0x000000000000e220
 *(.farrodata.*10 .farrodata.*10$)
                0x0000000000000000                . = ALIGN (0x10)

.farrodata.11$  0x0000000000000000        0x0 load address 0x000000000000e220
 *(.farrodata.*11 .farrodata.*11$)
                0x0000000000000000                . = ALIGN (0x10)

.farrodata.12$  0x0000000000000000        0x0 load address 0x000000000000e220
 *(.farrodata.*12 .farrodata.*12$)
                0x0000000000000000                . = ALIGN (0x10)

.farrodata.13$  0x0000000000000000        0x0 load address 0x000000000000e220
 *(.farrodata.*13 .farrodata.*13$)
                0x0000000000000000                . = ALIGN (0x10)

.farrodata.14$  0x0000000000000000        0x0 load address 0x000000000000e220
 *(.farrodata.*14 .farrodata.*14$)
                0x0000000000000000                . = ALIGN (0x10)

.farrodata.15$  0x0000000000000000        0x0 load address 0x000000000000e220
 *(.farrodata.*15 .farrodata.*15$)
                0x0000000000000000                . = ALIGN (0x10)

.farrodata.16$  0x0000000000000000        0x0 load address 0x000000000000e220
 *(.farrodata.*16 .farrodata.*16$)
                0x0000000000000000                . = ALIGN (0x10)

.farrodata.17$  0x0000000000000000        0x0 load address 0x000000000000e220
 *(.farrodata.*17 .farrodata.*17$)
                0x0000000000000000                . = ALIGN (0x10)

.farrodata.20$  0x0000000000000000        0x0 load address 0x000000000000e220
 *(.farrodata.*20 .farrodata.*20$)
                0x0000000000000000                . = ALIGN (0x10)

.farrodata.21$  0x0000000000000000        0x0 load address 0x000000000000e220
 *(.farrodata.*21 .farrodata.*21$)
                0x0000000000000000                . = ALIGN (0x10)

.farrodata.22$  0x0000000000000000        0x0 load address 0x000000000000e220
 *(.farrodata.*22 .farrodata.*22$)
                0x0000000000000000                . = ALIGN (0x10)

.farrodata.23$  0x0000000000000000        0x0 load address 0x000000000000e220
 *(.farrodata.*23 .farrodata.*23$)
                0x0000000000000000                . = ALIGN (0x10)

.farrodata.24$  0x0000000000000000        0x0 load address 0x000000000000e220
 *(.farrodata.*24 .farrodata.*24$)
                0x0000000000000000                . = ALIGN (0x10)

.farrodata.25$  0x0000000000000000        0x0 load address 0x000000000000e220
 *(.farrodata.*25 .farrodata.*25$)
                0x0000000000000000                . = ALIGN (0x10)

.farrodata.26$  0x0000000000000000        0x0 load address 0x000000000000e220
 *(.farrodata.*26 .farrodata.*26$)
                0x0000000000000000                . = ALIGN (0x10)

.farrodata.27$  0x0000000000000000        0x0 load address 0x000000000000e220
 *(.farrodata.*27 .farrodata.*27$)
                0x0000000000000000                . = ALIGN (0x10)

.farrodata.30$  0x0000000000000000        0x0 load address 0x000000000000e220
 *(.farrodata.*30 .farrodata.*30$)
                0x0000000000000000                . = ALIGN (0x10)

.farrodata.31$  0x0000000000000000        0x0 load address 0x000000000000e220
 *(.farrodata.*31 .farrodata.*31$)
                0x0000000000000000                . = ALIGN (0x10)

.farrodata.32$  0x0000000000000000        0x0 load address 0x000000000000e220
 *(.farrodata.*32 .farrodata.*32$)
                0x0000000000000000                . = ALIGN (0x10)

.farrodata.33$  0x0000000000000000        0x0 load address 0x000000000000e220
 *(.farrodata.*33 .farrodata.*33$)
                0x0000000000000000                . = ALIGN (0x10)

.farrodata.34$  0x0000000000000000        0x0 load address 0x000000000000e220
 *(.farrodata.*34 .farrodata.*34$)
                0x0000000000000000                . = ALIGN (0x10)

.farrodata.35$  0x0000000000000000        0x0 load address 0x000000000000e220
 *(.farrodata.*35 .farrodata.*35$)
                0x0000000000000000                . = ALIGN (0x10)

.farrodata.36$  0x0000000000000000        0x0 load address 0x000000000000e220
 *(.farrodata.*36 .farrodata.*36$)
                0x0000000000000000                . = ALIGN (0x10)

.farrodata.37$  0x0000000000000000        0x0 load address 0x000000000000e220
 *(.farrodata.*37 .farrodata.*37$)
                0x0000000000000000                . = ALIGN (0x10)

.farrodata.40$  0x0000000000000000        0x0 load address 0x000000000000e220
 *(.farrodata.*40 .farrodata.*40$)
                0x0000000000000000                . = ALIGN (0x10)

.farrodata.41$  0x0000000000000000        0x0 load address 0x000000000000e220
 *(.farrodata.*41 .farrodata.*41$)
                0x0000000000000000                . = ALIGN (0x10)

.farrodata.42$  0x0000000000000000        0x0 load address 0x000000000000e220
 *(.farrodata.*42 .farrodata.*42$)
                0x0000000000000000                . = ALIGN (0x10)

.farrodata.43$  0x0000000000000000        0x0 load address 0x000000000000e220
 *(.farrodata.*43 .farrodata.*43$)
                0x0000000000000000                . = ALIGN (0x10)

.farrodata.44$  0x0000000000000000        0x0 load address 0x000000000000e220
 *(.farrodata.*44 .farrodata.*44$)
                0x0000000000000000                . = ALIGN (0x10)

.farrodata.45$  0x0000000000000000        0x0 load address 0x000000000000e220
 *(.farrodata.*45 .farrodata.*45$)
                0x0000000000000000                . = ALIGN (0x10)

.farrodata.46$  0x0000000000000000        0x0 load address 0x000000000000e220
 *(.farrodata.*46 .farrodata.*46$)
                0x0000000000000000                . = ALIGN (0x10)

.farrodata.47$  0x0000000000000000        0x0 load address 0x000000000000e220
 *(.farrodata.*47 .farrodata.*47$)
                0x0000000000000000                . = ALIGN (0x10)

.farrodata.50$  0x0000000000000000        0x0 load address 0x000000000000e220
 *(.farrodata.*50 .farrodata.*50$)
                0x0000000000000000                . = ALIGN (0x10)

.farrodata.51$  0x0000000000000000        0x0 load address 0x000000000000e220
 *(.farrodata.*51 .farrodata.*51$)
                0x0000000000000000                . = ALIGN (0x10)

.farrodata.52$  0x0000000000000000        0x0 load address 0x000000000000e220
 *(.farrodata.*52 .farrodata.*52$)
                0x0000000000000000                . = ALIGN (0x10)

.farrodata.53$  0x0000000000000000        0x0 load address 0x000000000000e220
 *(.farrodata.*53 .farrodata.*53$)
                0x0000000000000000                . = ALIGN (0x10)

.farrodata.54$  0x0000000000000000        0x0 load address 0x000000000000e220
 *(.farrodata.*54 .farrodata.*54$)
                0x0000000000000000                . = ALIGN (0x10)

.farrodata.55$  0x0000000000000000        0x0 load address 0x000000000000e220
 *(.farrodata.*55 .farrodata.*55$)
                0x0000000000000000                . = ALIGN (0x10)

.farrodata.56$  0x0000000000000000        0x0 load address 0x000000000000e220
 *(.farrodata.*56 .farrodata.*56$)
                0x0000000000000000                . = ALIGN (0x10)

.farrodata.57$  0x0000000000000000        0x0 load address 0x000000000000e220
 *(.farrodata.*57 .farrodata.*57$)
                0x0000000000000000                . = ALIGN (0x10)

.farrodata.60$  0x0000000000000000        0x0 load address 0x000000000000e220
 *(.farrodata.*60 .farrodata.*60$)
                0x0000000000000000                . = ALIGN (0x10)

.farrodata.61$  0x0000000000000000        0x0 load address 0x000000000000e220
 *(.farrodata.*61 .farrodata.*61$)
                0x0000000000000000                . = ALIGN (0x10)

.farrodata.62$  0x0000000000000000        0x0 load address 0x000000000000e220
 *(.farrodata.*62 .farrodata.*62$)
                0x0000000000000000                . = ALIGN (0x10)

.farrodata.63$  0x0000000000000000        0x0 load address 0x000000000000e220
 *(.farrodata.*63 .farrodata.*63$)
                0x0000000000000000                . = ALIGN (0x10)

.farrodata.64$  0x0000000000000000        0x0 load address 0x000000000000e220
 *(.farrodata.*64 .farrodata.*64$)
                0x0000000000000000                . = ALIGN (0x10)

.farrodata.65$  0x0000000000000000        0x0 load address 0x000000000000e220
 *(.farrodata.*65 .farrodata.*65$)
                0x0000000000000000                . = ALIGN (0x10)

.farrodata.66$  0x0000000000000000        0x0 load address 0x000000000000e220
 *(.farrodata.*66 .farrodata.*66$)
                0x0000000000000000                . = ALIGN (0x10)

.farrodata.67$  0x0000000000000000        0x0 load address 0x000000000000e220
 *(.farrodata.*67 .farrodata.*67$)
                0x0000000000000000                . = ALIGN (0x10)

.farrodata.70$  0x0000000000000000        0x0 load address 0x000000000000e220
 *(.farrodata.*70 .farrodata.*70$)
                0x0000000000000000                . = ALIGN (0x10)

.farrodata.71$  0x0000000000000000        0x0 load address 0x000000000000e220
 *(.farrodata.*71 .farrodata.*71$)
                0x0000000000000000                . = ALIGN (0x10)

.farrodata.72$  0x0000000000000000        0x0 load address 0x000000000000e220
 *(.farrodata.*72 .farrodata.*72$)
                0x0000000000000000                . = ALIGN (0x10)

.farrodata.73$  0x0000000000000000        0x0 load address 0x000000000000e220
 *(.farrodata.*73 .farrodata.*73$)
                0x0000000000000000                . = ALIGN (0x10)

.farrodata.74$  0x0000000000000000        0x0 load address 0x000000000000e220
 *(.farrodata.*74 .farrodata.*74$)
                0x0000000000000000                . = ALIGN (0x10)

.farrodata.75$  0x0000000000000000        0x0 load address 0x000000000000e220
 *(.farrodata.*75 .farrodata.*75$)
                0x0000000000000000                . = ALIGN (0x10)

.farrodata.76$  0x0000000000000000        0x0 load address 0x000000000000e220
 *(.farrodata.*76 .farrodata.*76$)
                0x0000000000000000                . = ALIGN (0x10)

.farrodata.77$  0x0000000000000000        0x0 load address 0x000000000000e220
 *(.farrodata.*77 .farrodata.*77$)
                0x0000000000000000                . = ALIGN (0x10)

.farrodata.XX$  0x0000000000000000        0x0 load address 0x000000000000e220
 *(.farrodata .farrodata$ .farrodata.*)
                0x0000000000000000                . = ALIGN (0x10)

.fardata.00$    0x0000000000000000        0x0 load address 0x000000000000e220
 *(.fardata.*00 .fardata.*00$)
                0x0000000000000000                . = ALIGN (0x10)

.fardata.01$    0x0000000000000000        0x0 load address 0x000000000000e220
 *(.fardata.*01 .fardata.*01$)
                0x0000000000000000                . = ALIGN (0x10)

.fardata.02$    0x0000000000000000        0x0 load address 0x000000000000e220
 *(.fardata.*02 .fardata.*02$)
                0x0000000000000000                . = ALIGN (0x10)

.fardata.03$    0x0000000000000000        0x0 load address 0x000000000000e220
 *(.fardata.*03 .fardata.*03$)
                0x0000000000000000                . = ALIGN (0x10)

.fardata.04$    0x0000000000000000        0x0 load address 0x000000000000e220
 *(.fardata.*04 .fardata.*04$)
                0x0000000000000000                . = ALIGN (0x10)

.fardata.05$    0x0000000000000000        0x0 load address 0x000000000000e220
 *(.fardata.*05 .fardata.*05$)
                0x0000000000000000                . = ALIGN (0x10)

.fardata.06$    0x0000000000000000        0x0 load address 0x000000000000e220
 *(.fardata.*06 .fardata.*06$)
                0x0000000000000000                . = ALIGN (0x10)

.fardata.07$    0x0000000000000000        0x0 load address 0x000000000000e220
 *(.fardata.*07 .fardata.*07$)
                0x0000000000000000                . = ALIGN (0x10)

.fardata.10$    0x0000000000000000        0x0 load address 0x000000000000e220
 *(.fardata.*10 .fardata.*10$)
                0x0000000000000000                . = ALIGN (0x10)

.fardata.11$    0x0000000000000000        0x0 load address 0x000000000000e220
 *(.fardata.*11 .fardata.*11$)
                0x0000000000000000                . = ALIGN (0x10)

.fardata.12$    0x0000000000000000        0x0 load address 0x000000000000e220
 *(.fardata.*12 .fardata.*12$)
                0x0000000000000000                . = ALIGN (0x10)

.fardata.13$    0x0000000000000000        0x0 load address 0x000000000000e220
 *(.fardata.*13 .fardata.*13$)
                0x0000000000000000                . = ALIGN (0x10)

.fardata.14$    0x0000000000000000        0x0 load address 0x000000000000e220
 *(.fardata.*14 .fardata.*14$)
                0x0000000000000000                . = ALIGN (0x10)

.fardata.15$    0x0000000000000000        0x0 load address 0x000000000000e220
 *(.fardata.*15 .fardata.*15$)
                0x0000000000000000                . = ALIGN (0x10)

.fardata.16$    0x0000000000000000        0x0 load address 0x000000000000e220
 *(.fardata.*16 .fardata.*16$)
                0x0000000000000000                . = ALIGN (0x10)

.fardata.17$    0x0000000000000000        0x0 load address 0x000000000000e220
 *(.fardata.*17 .fardata.*17$)
                0x0000000000000000                . = ALIGN (0x10)

.fardata.20$    0x0000000000000000        0x0 load address 0x000000000000e220
 *(.fardata.*20 .fardata.*20$)
                0x0000000000000000                . = ALIGN (0x10)

.fardata.21$    0x0000000000000000        0x0 load address 0x000000000000e220
 *(.fardata.*21 .fardata.*21$)
                0x0000000000000000                . = ALIGN (0x10)

.fardata.22$    0x0000000000000000        0x0 load address 0x000000000000e220
 *(.fardata.*22 .fardata.*22$)
                0x0000000000000000                . = ALIGN (0x10)

.fardata.23$    0x0000000000000000        0x0 load address 0x000000000000e220
 *(.fardata.*23 .fardata.*23$)
                0x0000000000000000                . = ALIGN (0x10)

.fardata.24$    0x0000000000000000        0x0 load address 0x000000000000e220
 *(.fardata.*24 .fardata.*24$)
                0x0000000000000000                . = ALIGN (0x10)

.fardata.25$    0x0000000000000000        0x0 load address 0x000000000000e220
 *(.fardata.*25 .fardata.*25$)
                0x0000000000000000                . = ALIGN (0x10)

.fardata.26$    0x0000000000000000        0x0 load address 0x000000000000e220
 *(.fardata.*26 .fardata.*26$)
                0x0000000000000000                . = ALIGN (0x10)

.fardata.27$    0x0000000000000000        0x0 load address 0x000000000000e220
 *(.fardata.*27 .fardata.*27$)
                0x0000000000000000                . = ALIGN (0x10)

.fardata.30$    0x0000000000000000        0x0 load address 0x000000000000e220
 *(.fardata.*30 .fardata.*30$)
                0x0000000000000000                . = ALIGN (0x10)

.fardata.31$    0x0000000000000000        0x0 load address 0x000000000000e220
 *(.fardata.*31 .fardata.*31$)
                0x0000000000000000                . = ALIGN (0x10)

.fardata.32$    0x0000000000000000        0x0 load address 0x000000000000e220
 *(.fardata.*32 .fardata.*32$)
                0x0000000000000000                . = ALIGN (0x10)

.fardata.33$    0x0000000000000000        0x0 load address 0x000000000000e220
 *(.fardata.*33 .fardata.*33$)
                0x0000000000000000                . = ALIGN (0x10)

.fardata.34$    0x0000000000000000        0x0 load address 0x000000000000e220
 *(.fardata.*34 .fardata.*34$)
                0x0000000000000000                . = ALIGN (0x10)

.fardata.35$    0x0000000000000000        0x0 load address 0x000000000000e220
 *(.fardata.*35 .fardata.*35$)
                0x0000000000000000                . = ALIGN (0x10)

.fardata.36$    0x0000000000000000        0x0 load address 0x000000000000e220
 *(.fardata.*36 .fardata.*36$)
                0x0000000000000000                . = ALIGN (0x10)

.fardata.37$    0x0000000000000000        0x0 load address 0x000000000000e220
 *(.fardata.*37 .fardata.*37$)
                0x0000000000000000                . = ALIGN (0x10)

.fardata.40$    0x0000000000000000        0x0 load address 0x000000000000e220
 *(.fardata.*40 .fardata.*40$)
                0x0000000000000000                . = ALIGN (0x10)

.fardata.41$    0x0000000000000000        0x0 load address 0x000000000000e220
 *(.fardata.*41 .fardata.*41$)
                0x0000000000000000                . = ALIGN (0x10)

.fardata.42$    0x0000000000000000        0x0 load address 0x000000000000e220
 *(.fardata.*42 .fardata.*42$)
                0x0000000000000000                . = ALIGN (0x10)

.fardata.43$    0x0000000000000000        0x0 load address 0x000000000000e220
 *(.fardata.*43 .fardata.*43$)
                0x0000000000000000                . = ALIGN (0x10)

.fardata.44$    0x0000000000000000        0x0 load address 0x000000000000e220
 *(.fardata.*44 .fardata.*44$)
                0x0000000000000000                . = ALIGN (0x10)

.fardata.45$    0x0000000000000000        0x0 load address 0x000000000000e220
 *(.fardata.*45 .fardata.*45$)
                0x0000000000000000                . = ALIGN (0x10)

.fardata.46$    0x0000000000000000        0x0 load address 0x000000000000e220
 *(.fardata.*46 .fardata.*46$)
                0x0000000000000000                . = ALIGN (0x10)

.fardata.47$    0x0000000000000000        0x0 load address 0x000000000000e220
 *(.fardata.*47 .fardata.*47$)
                0x0000000000000000                . = ALIGN (0x10)

.fardata.50$    0x0000000000000000        0x0 load address 0x000000000000e220
 *(.fardata.*50 .fardata.*50$)
                0x0000000000000000                . = ALIGN (0x10)

.fardata.51$    0x0000000000000000        0x0 load address 0x000000000000e220
 *(.fardata.*51 .fardata.*51$)
                0x0000000000000000                . = ALIGN (0x10)

.fardata.52$    0x0000000000000000        0x0 load address 0x000000000000e220
 *(.fardata.*52 .fardata.*52$)
                0x0000000000000000                . = ALIGN (0x10)

.fardata.53$    0x0000000000000000        0x0 load address 0x000000000000e220
 *(.fardata.*53 .fardata.*53$)
                0x0000000000000000                . = ALIGN (0x10)

.fardata.54$    0x0000000000000000        0x0 load address 0x000000000000e220
 *(.fardata.*54 .fardata.*54$)
                0x0000000000000000                . = ALIGN (0x10)

.fardata.55$    0x0000000000000000        0x0 load address 0x000000000000e220
 *(.fardata.*55 .fardata.*55$)
                0x0000000000000000                . = ALIGN (0x10)

.fardata.56$    0x0000000000000000        0x0 load address 0x000000000000e220
 *(.fardata.*56 .fardata.*56$)
                0x0000000000000000                . = ALIGN (0x10)

.fardata.57$    0x0000000000000000        0x0 load address 0x000000000000e220
 *(.fardata.*57 .fardata.*57$)
                0x0000000000000000                . = ALIGN (0x10)

.fardata.60$    0x0000000000000000        0x0 load address 0x000000000000e220
 *(.fardata.*60 .fardata.*60$)
                0x0000000000000000                . = ALIGN (0x10)

.fardata.61$    0x0000000000000000        0x0 load address 0x000000000000e220
 *(.fardata.*61 .fardata.*61$)
                0x0000000000000000                . = ALIGN (0x10)

.fardata.62$    0x0000000000000000        0x0 load address 0x000000000000e220
 *(.fardata.*62 .fardata.*62$)
                0x0000000000000000                . = ALIGN (0x10)

.fardata.63$    0x0000000000000000        0x0 load address 0x000000000000e220
 *(.fardata.*63 .fardata.*63$)
                0x0000000000000000                . = ALIGN (0x10)

.fardata.64$    0x0000000000000000        0x0 load address 0x000000000000e220
 *(.fardata.*64 .fardata.*64$)
                0x0000000000000000                . = ALIGN (0x10)

.fardata.65$    0x0000000000000000        0x0 load address 0x000000000000e220
 *(.fardata.*65 .fardata.*65$)
                0x0000000000000000                . = ALIGN (0x10)

.fardata.66$    0x0000000000000000        0x0 load address 0x000000000000e220
 *(.fardata.*66 .fardata.*66$)
                0x0000000000000000                . = ALIGN (0x10)

.fardata.67$    0x0000000000000000        0x0 load address 0x000000000000e220
 *(.fardata.*67 .fardata.*67$)
                0x0000000000000000                . = ALIGN (0x10)

.fardata.70$    0x0000000000000000        0x0 load address 0x000000000000e220
 *(.fardata.*70 .fardata.*70$)
                0x0000000000000000                . = ALIGN (0x10)

.fardata.71$    0x0000000000000000        0x0 load address 0x000000000000e220
 *(.fardata.*71 .fardata.*71$)
                0x0000000000000000                . = ALIGN (0x10)

.fardata.72$    0x0000000000000000        0x0 load address 0x000000000000e220
 *(.fardata.*72 .fardata.*72$)
                0x0000000000000000                . = ALIGN (0x10)

.fardata.73$    0x0000000000000000        0x0 load address 0x000000000000e220
 *(.fardata.*73 .fardata.*73$)
                0x0000000000000000                . = ALIGN (0x10)

.fardata.74$    0x0000000000000000        0x0 load address 0x000000000000e220
 *(.fardata.*74 .fardata.*74$)
                0x0000000000000000                . = ALIGN (0x10)

.fardata.75$    0x0000000000000000        0x0 load address 0x000000000000e220
 *(.fardata.*75 .fardata.*75$)
                0x0000000000000000                . = ALIGN (0x10)

.fardata.76$    0x0000000000000000        0x0 load address 0x000000000000e220
 *(.fardata.*76 .fardata.*76$)
                0x0000000000000000                . = ALIGN (0x10)

.fardata.77$    0x0000000000000000        0x0 load address 0x000000000000e220
 *(.fardata.*77 .fardata.*77$)
                0x0000000000000000                . = ALIGN (0x10)

.fardata.XX$    0x0000000000000000        0x0 load address 0x000000000000e220
 *(.fardata .fardata$ .fardata.*)
                0x0000000000000000                . = ALIGN (0x10)

.data           0x0000000000000020      0xf90 load address 0x000000000000e220
                0x0000000000000020                __sdata = .
 *crtbegin*.o(.ctors)
 .ctors         0x0000000000000020        0x2 /home/evln/proj/build-ia16.202501/prefix/bin/../lib/gcc/ia16-elf/6.3.0/regparmcall/crtbegin.o
 *(EXCLUDE_FILE(*crtend*.o) .ctors)
 *(SORT_BY_NAME(.ctors.*))
 *(.ctors)
 .ctors         0x0000000000000022        0x2 /home/evln/proj/build-ia16.202501/prefix/bin/../lib/gcc/ia16-elf/6.3.0/regparmcall/crtend.o
 *crtbegin*.o(.dtors)
 .dtors         0x0000000000000024        0x2 /home/evln/proj/build-ia16.202501/prefix/bin/../lib/gcc/ia16-elf/6.3.0/regparmcall/crtbegin.o
 *(EXCLUDE_FILE(*crtend*.o) .dtors)
 *(SORT_BY_NAME(.dtors.*))
 *(.dtors)
 .dtors         0x0000000000000026        0x2 /home/evln/proj/build-ia16.202501/prefix/bin/../lib/gcc/ia16-elf/6.3.0/regparmcall/crtend.o
                0x0000000000000026                __DTOR_END__
 *(.msdos_init_rodata)
 *(.msdos_init_rodata.*)
 *(.rodata)
 .rodata        0x0000000000000028        0x4 loadhigh.obj
 .rodata        0x000000000000002c       0x34 ver.obj
                0x000000000000002c                shellname
                0x0000000000000049                shellver
 .rodata        0x0000000000000060        0xc ../cmd/cmds.lib(for.obj)
 .rodata        0x000000000000006c        0xc ../lib/freecom.lib(cbreak.obj)
 .rodata        0x0000000000000078       0x1a ../lib/freecom.lib(pr_date.obj)
 .rodata        0x0000000000000092       0x14 ../lib/freecom.lib(msg_dflt.obj)
 .rodata        0x00000000000000a6       0x16 ../strings/strings.lib(str0011.obj)
                0x00000000000000a6                TEXT_ERROR_OUT_OF_MEMORY
 .rodata        0x00000000000000bc       0x3a ../strings/strings.lib(str0018.obj)
                0x00000000000000bc                TEXT_ERROR_SET_ENV_VAR
 .rodata        0x00000000000000f6       0x1a ../strings/strings.lib(str003c.obj)
                0x00000000000000f6                TEXT_ERROR_OPEN_FILE
 .rodata        0x0000000000000110       0xe6 ../strings/strings.lib(str00b1.obj)
                0x0000000000000110                TEXT_MSG_REBOOT_NOW
 .rodata        0x00000000000001f6       0x89 ../strings/strings.lib(str00b2.obj)
                0x00000000000001f6                TEXT_MSG_FREECOM_NOT_FOUND
 .rodata        0x000000000000027f       0x41 ../strings/strings.lib(str00f4.obj)
                0x000000000000027f                TEXT_ERROR_FCOM_INVALID
 .rodata        0x00000000000002c0       0xfe ../strings/strings.lib(str00f5.obj)
                0x00000000000002c0                TEXT_ERROR_LOADING_STRINGS
 .rodata        0x00000000000003be       0x12 ../strings/strings.lib(str00f6.obj)
                0x00000000000003be                TEXT_TERMINATING
 .rodata        0x00000000000003d0      0x281 /home/evln/proj/build-ia16.202501/prefix/bin/../lib/gcc/ia16-elf/6.3.0/../../../../ia16-elf/lib/regparmcall/libc.a(lib_a-ctype_.o)
                0x00000000000003d0                _ctype_
 *fill*         0x0000000000000651        0x1 
 .rodata        0x0000000000000652        0x2 /home/evln/proj/build-ia16.202501/prefix/bin/../lib/gcc/ia16-elf/6.3.0/../../../../ia16-elf/lib/regparmcall/libc.a(lib_a-impure.o)
                0x0000000000000652                _global_impure_ptr
 .rodata        0x0000000000000654       0x4f /home/evln/proj/build-ia16.202501/prefix/bin/../lib/gcc/ia16-elf/6.3.0/../../../../ia16-elf/lib/regparmcall/libc.a(lib_a-nano-freer.o)
 .rodata        0x00000000000006a3       0x2a /home/evln/proj/build-ia16.202501/prefix/bin/../lib/gcc/ia16-elf/6.3.0/../../../../ia16-elf/lib/regparmcall/libc.a(lib_a-nano-mallocr.o)
 .rodata        0x00000000000006cd       0x43 /home/evln/proj/build-ia16.202501/prefix/bin/../lib/gcc/ia16-elf/6.3.0/../../../../ia16-elf/lib/regparmcall/libc.a(lib_a-abort.o)
 *(.rodata.*)
 .rodata.str1.1
                0x0000000000000710        0x4 batch.obj
 .rodata.str1.1
                0x0000000000000714      0x10d cmdtable.obj
 .rodata.str1.1
                0x0000000000000821       0x82 command.obj
 .rodata.str1.1
                0x00000000000008a3       0x2f init.obj
 .rodata.str1.1
                0x00000000000008d2       0x11 loadhigh.obj
 .rodata.str1.1
                0x00000000000008e3        0x4 redir.obj
 .rodata.str1.1
                0x00000000000008e7       0x1c ver.obj
 .rodata.str1.1
                0x0000000000000903        0x7 ../cmd/cmds.lib(break.obj)
 .rodata.str1.1
                0x000000000000090a        0x4 ../cmd/cmds.lib(cdd.obj)
 .rodata.str1.1
                0x000000000000090e        0x6 ../cmd/cmds.lib(chdir.obj)
 .rodata.str1.1
                0x0000000000000914        0x5 ../cmd/cmds.lib(cls.obj)
 .rodata.str1.1
                0x0000000000000919       0x25 ../cmd/cmds.lib(copy.obj)
 .rodata.str1.1
                0x000000000000093e        0x3 ../cmd/cmds.lib(ctty.obj)
 .rodata.str1.1
                0x0000000000000941        0x4 ../cmd/cmds.lib(del.obj)
 .rodata.str1.1
                0x0000000000000945       0x63 ../cmd/cmds.lib(dir.obj)
 .rodata.str1.1
                0x00000000000009a8        0x7 ../cmd/cmds.lib(echo.obj)
 .rodata.str1.1
                0x00000000000009af        0xe ../cmd/cmds.lib(for.obj)
 .rodata.str1.1
                0x00000000000009bd       0x42 ../cmd/cmds.lib(history.obj)
 .rodata.str1.1
                0x00000000000009ff       0x1f ../cmd/cmds.lib(if.obj)
 .rodata.str1.1
                0x0000000000000a1e       0x10 ../cmd/cmds.lib(lfnfor.obj)
 .rodata.str1.1
                0x0000000000000a2e        0x6 ../cmd/cmds.lib(mkdir.obj)
 .rodata.str1.1
                0x0000000000000a34        0x5 ../cmd/cmds.lib(path.obj)
 .rodata.str1.1
                0x0000000000000a39        0x7 ../cmd/cmds.lib(prompt.obj)
 .rodata.str1.1
                0x0000000000000a40        0x9 ../cmd/cmds.lib(ren.obj)
 .rodata.str1.1
                0x0000000000000a49        0xf ../cmd/cmds.lib(rmdir.obj)
 .rodata.str1.1
                0x0000000000000a58       0x3d ../cmd/cmds.lib(set.obj)
 .rodata.str1.1
                0x0000000000000a95        0x5 ../cmd/cmds.lib(shift.obj)
 .rodata.str1.1
                0x0000000000000a9a        0x2 ../cmd/cmds.lib(truename.obj)
 .rodata.str1.1
                0x0000000000000a9c        0x3 ../cmd/cmds.lib(type.obj)
 .rodata.str1.1
                0x0000000000000a9f        0x7 ../cmd/cmds.lib(verify.obj)
 .rodata.str1.1
                0x0000000000000aa6        0xf ../lib/freecom.lib(cbreak.obj)
 .rodata.str1.1
                0x0000000000000ab5        0x2 ../lib/freecom.lib(cd_dir.obj)
 .rodata.str1.1
                0x0000000000000ab7        0xa ../lib/freecom.lib(cmdinput.obj)
 .rodata.str1.1
                0x0000000000000ac1        0x7 ../lib/freecom.lib(ctxt_mkn.obj)
 .rodata.str1.1
                0x0000000000000ac8        0x5 ../lib/freecom.lib(ctxt_vw.obj)
 .rodata.str1.1
                0x0000000000000acd        0x7 ../lib/freecom.lib(curdatel.obj)
 .rodata.str1.1
                0x0000000000000ad4        0x2 ../lib/freecom.lib(exec.obj)
 .rodata.str1.1
                0x0000000000000ad6       0x15 ../lib/freecom.lib(filecomp.obj)
 .rodata.str1.1
                0x0000000000000aeb        0x1 ../lib/freecom.lib(fillcomp.obj)
 .rodata.str1.1
                0x0000000000000aec        0x6 ../lib/freecom.lib(find.obj)
 .rodata.str1.1
                0x0000000000000af2       0x16 ../lib/freecom.lib(grabfcom.obj)
 .rodata.str1.1
                0x0000000000000b08        0x5 ../lib/freecom.lib(hdlrctxt.obj)
 .rodata.str1.1
                0x0000000000000b0d        0x1 ../lib/freecom.lib(leadopt.obj)
 .rodata.str1.1
                0x0000000000000b0e        0x4 ../lib/freecom.lib(ltrimcl.obj)
 .rodata.str1.1
                0x0000000000000b12       0x3c ../lib/freecom.lib(messages.obj)
 .rodata.str1.1
                0x0000000000000b4e        0x2 ../lib/freecom.lib(mux_ae.obj)
 .rodata.str1.1
                0x0000000000000b50       0x11 ../lib/freecom.lib(nls_date.obj)
 .rodata.str1.1
                0x0000000000000b61       0x18 ../lib/freecom.lib(nls_time.obj)
 .rodata.str1.1
                0x0000000000000b79        0x7 ../lib/freecom.lib(onoff.obj)
 .rodata.str1.1
                0x0000000000000b80        0x4 ../lib/freecom.lib(openf.obj)
 .rodata.str1.1
                0x0000000000000b84        0xc ../lib/freecom.lib(pr_prmpt.obj)
 .rodata.str1.1
                0x0000000000000b90        0x4 ../lib/freecom.lib(pr_time.obj)
 .rodata.str1.1
                0x0000000000000b94       0x1f ../lib/freecom.lib(prf.obj)
 .rodata.str1.1
                0x0000000000000bb3        0xc ../lib/freecom.lib(prprompt.obj)
 .rodata.str1.1
                0x0000000000000bbf        0x9 ../lib/freecom.lib(res_r.obj)
 .rodata.str1.1
                0x0000000000000bc8        0x4 ../lib/freecom.lib(resfile.obj)
 .rodata.str1.1
                0x0000000000000bcc        0x4 ../lib/freecom.lib(rtrimcl.obj)
 .rodata.str1.1
                0x0000000000000bd0        0x8 ../lib/freecom.lib(scanopt.obj)
 .rodata.str1.1
                0x0000000000000bd8        0x6 ../lib/freecom.lib(showcmds.obj)
 .rodata.str1.1
                0x0000000000000bde        0x6 ../lib/freecom.lib(skqwd.obj)
 .rodata.str1.1
                0x0000000000000be4       0x25 ../lib/freecom.lib(tmpnam.obj)
 .rodata.str1.1
                0x0000000000000c09        0x2 ../lib/freecom.lib(unquote.obj)
 .rodata.str1.1
                0x0000000000000c0b       0x11 ../lib/freecom.lib(where.obj)
 .rodata.str1.1
                0x0000000000000c1c        0x9 ../lib/freecom.lib(comfile.obj)
 .rodata.str1.1
                0x0000000000000c25        0x8 ../lib/freecom.lib(dispexit.obj)
 .rodata.str1.1
                0x0000000000000c2d        0x9 ../lib/freecom.lib(mktmpfil.obj)
 .rodata.str1.1
                0x0000000000000c36        0xc ../lib/freecom.lib(msg_dflt.obj)
 .rodata.str1.1
                0x0000000000000c42        0x2 ../suppl/suppl_s.lib(dfnfullp.obj)
 .rodata.str1.1
                0x0000000000000c44        0x1 ../suppl/suppl_s.lib(env_ovrw.obj)
 .rodata.str1.1
                0x0000000000000c45        0x2 ../suppl/suppl_s.lib(dstrchar.obj)
 .rodata.str1.1
                0x0000000000000c47        0x2 /home/evln/proj/build-ia16.202501/prefix/bin/../lib/gcc/ia16-elf/6.3.0/../../../../ia16-elf/lib/regparmcall/libc.a(lib_a-impure.o)
 .rodata.str1.1
                0x0000000000000c49       0x11 /home/evln/proj/build-ia16.202501/prefix/bin/../lib/gcc/ia16-elf/6.3.0/../../../../ia16-elf/lib/regparmcall/libc.a(lib_a-abort.o)
 *(.autofloat_stdio.__ia16_have_printf_float.dprintf.v2)
 *(.autofloat_stdio.__ia16_have_printf_float._dprintf_r.v2)
 *(.autofloat_stdio.__ia16_have_printf_float.vdprintf.v2)
 *(.autofloat_stdio.__ia16_have_printf_float._vdprintf_r.v2)
 *(.autofloat_stdio.__ia16_have_printf_float.sprintf.v2)
 *(.autofloat_stdio.__ia16_have_printf_float._sprintf_r.v2)
 *(.autofloat_stdio.__ia16_have_printf_float.fprintf.v2)
 *(.autofloat_stdio.__ia16_have_printf_float._fprintf_r.v2)
 *(.autofloat_stdio.__ia16_have_printf_float.printf.v2)
 *(.autofloat_stdio.__ia16_have_printf_float._printf_r.v2)
 *(.autofloat_stdio.__ia16_have_printf_float.snprintf.v2)
 *(.autofloat_stdio.__ia16_have_printf_float._snprintf_r.v2)
 *(.autofloat_stdio.__ia16_have_printf_float.asprintf.v2)
 *(.autofloat_stdio.__ia16_have_printf_float._asprintf_r.v2)
 *(.autofloat_stdio.__ia16_have_printf_float.asnprintf.v2)
 *(.autofloat_stdio.__ia16_have_printf_float._asnprintf_r.v2)
 *(.autofloat_stdio.__ia16_have_printf_float.vprintf.v2)
 *(.autofloat_stdio.__ia16_have_printf_float._vprintf_r.v2)
 *(.autofloat_stdio.__ia16_have_printf_float.vfprintf.v2)
 *(.autofloat_stdio.__ia16_have_printf_float._vfprintf_r.v2)
 *(.autofloat_stdio.__ia16_have_printf_float.vsprintf.v2)
 *(.autofloat_stdio.__ia16_have_printf_float._vsprintf_r.v2)
 *(.autofloat_stdio.__ia16_have_printf_float.vsnprintf.v2)
 *(.autofloat_stdio.__ia16_have_printf_float._vsnprintf_r.v2)
 *(.autofloat_stdio.__ia16_have_printf_float.vasprintf.v2)
 *(.autofloat_stdio.__ia16_have_printf_float._vasprintf_r.v2)
 *(.autofloat_stdio.__ia16_have_printf_float.vasnprintf.v2)
 *(.autofloat_stdio.__ia16_have_printf_float._vasnprintf_r.v2)
 *(.autofloat_stdio.__ia16_have_scanf_float.sscanf.v2)
 *(.autofloat_stdio.__ia16_have_scanf_float._sscanf_r.v2)
 *(.autofloat_stdio.__ia16_have_scanf_float.fscanf.v2)
 *(.autofloat_stdio.__ia16_have_scanf_float._fscanf_r.v2)
 *(.autofloat_stdio.__ia16_have_scanf_float.scanf.v2)
 *(.autofloat_stdio.__ia16_have_scanf_float._scanf_r.v2)
 *(.autofloat_stdio.__ia16_have_scanf_float.vscanf.v2)
 *(.autofloat_stdio.__ia16_have_scanf_float._vscanf_r.v2)
 *(.autofloat_stdio.__ia16_have_scanf_float.vfscanf.v2)
 *(.autofloat_stdio.__ia16_have_scanf_float._vfscanf_r.v2)
 *(.autofloat_stdio.__ia16_have_scanf_float.vsscanf.v2)
 *(.autofloat_stdio.__ia16_have_scanf_float._vsscanf_r.v2)
                0x0000000000000c5a                . = .
 *(.data)
 *fill*         0x0000000000000c5a        0x2 
 .data          0x0000000000000c5c        0x1 cswap.obj
 .data          0x0000000000000c5d        0x0 cswapc.obj
 *fill*         0x0000000000000c5d        0x1 
 .data          0x0000000000000c5e        0x2 batch.obj
                0x0000000000000c5e                echo
 .data          0x0000000000000c60      0x1a0 cmdtable.obj
                0x0000000000000c60                internalCommands
 .data          0x0000000000000e00        0xa command.obj
                0x0000000000000e00                __supportlfns
                0x0000000000000e02                swapContext
                0x0000000000000e04                inInit
                0x0000000000000e06                oldoutfd
                0x0000000000000e08                oldinfd
 .data          0x0000000000000e0a        0x0 expalias.obj
 .data          0x0000000000000e0a        0x2 init.obj
 .data          0x0000000000000e0c        0x0 kswap.obj
 .data          0x0000000000000e0c        0x0 loadhigh.obj
 .data          0x0000000000000e0c        0x0 module.obj
 .data          0x0000000000000e0c        0x0 redir.obj
 .data          0x0000000000000e0c        0x0 ver.obj
 .data          0x0000000000000e0c        0x0 ../cmd/cmds.lib(alias.obj)
 .data          0x0000000000000e0c        0x0 ../cmd/cmds.lib(beep.obj)
 .data          0x0000000000000e0c        0x0 ../cmd/cmds.lib(break.obj)
 .data          0x0000000000000e0c        0x0 ../cmd/cmds.lib(call.obj)
 .data          0x0000000000000e0c        0x0 ../cmd/cmds.lib(cdd.obj)
 .data          0x0000000000000e0c        0x0 ../cmd/cmds.lib(chcp.obj)
 .data          0x0000000000000e0c        0x0 ../cmd/cmds.lib(chdir.obj)
 .data          0x0000000000000e0c        0x0 ../cmd/cmds.lib(cls.obj)
 .data          0x0000000000000e0c        0x0 ../cmd/cmds.lib(copy.obj)
 .data          0x0000000000000e0c        0x0 ../cmd/cmds.lib(ctty.obj)
 .data          0x0000000000000e0c        0x0 ../cmd/cmds.lib(date.obj)
 .data          0x0000000000000e0c        0x0 ../cmd/cmds.lib(del.obj)
 .data          0x0000000000000e0c        0x4 ../cmd/cmds.lib(dir.obj)
 .data          0x0000000000000e10        0x0 ../cmd/cmds.lib(dirs.obj)
 .data          0x0000000000000e10        0x0 ../cmd/cmds.lib(doskey.obj)
 .data          0x0000000000000e10        0x0 ../cmd/cmds.lib(echo.obj)
 .data          0x0000000000000e10        0x0 ../cmd/cmds.lib(exit.obj)
 .data          0x0000000000000e10        0x0 ../cmd/cmds.lib(for.obj)
 .data          0x0000000000000e10        0x0 ../cmd/cmds.lib(goto.obj)
 .data          0x0000000000000e10        0x0 ../cmd/cmds.lib(history.obj)
 .data          0x0000000000000e10        0x0 ../cmd/cmds.lib(if.obj)
 .data          0x0000000000000e10        0x0 ../cmd/cmds.lib(lfnfor.obj)
 .data          0x0000000000000e10        0x0 ../cmd/cmds.lib(memory.obj)
 .data          0x0000000000000e10        0x0 ../cmd/cmds.lib(mkdir.obj)
 .data          0x0000000000000e10        0x0 ../cmd/cmds.lib(path.obj)
 .data          0x0000000000000e10        0x0 ../cmd/cmds.lib(pause.obj)
 .data          0x0000000000000e10        0x0 ../cmd/cmds.lib(popd.obj)
 .data          0x0000000000000e10        0x0 ../cmd/cmds.lib(prompt.obj)
 .data          0x0000000000000e10        0x0 ../cmd/cmds.lib(pushd.obj)
 .data          0x0000000000000e10        0x0 ../cmd/cmds.lib(rem.obj)
 .data          0x0000000000000e10        0x0 ../cmd/cmds.lib(ren.obj)
 .data          0x0000000000000e10        0x0 ../cmd/cmds.lib(rmdir.obj)
 .data          0x0000000000000e10        0x0 ../cmd/cmds.lib(set.obj)
 .data          0x0000000000000e10        0x0 ../cmd/cmds.lib(shift.obj)
 .data          0x0000000000000e10        0x0 ../cmd/cmds.lib(time.obj)
 .data          0x0000000000000e10        0x0 ../cmd/cmds.lib(truename.obj)
 .data          0x0000000000000e10        0x0 ../cmd/cmds.lib(type.obj)
 .data          0x0000000000000e10        0x0 ../cmd/cmds.lib(verify.obj)
 .data          0x0000000000000e10        0x0 ../cmd/cmds.lib(which.obj)
 .data          0x0000000000000e10        0x0 ../lib/freecom.lib(absfile.obj)
 .data          0x0000000000000e10        0x0 ../lib/freecom.lib(app_get.obj)
 .data          0x0000000000000e10        0x0 ../lib/freecom.lib(app_set.obj)
 .data          0x0000000000000e10        0x0 ../lib/freecom.lib(beep_n.obj)
 .data          0x0000000000000e10        0x0 ../lib/freecom.lib(brk_get.obj)
 .data          0x0000000000000e10        0x0 ../lib/freecom.lib(brk_set.obj)
 .data          0x0000000000000e10        0xd ../lib/freecom.lib(cbreak.obj)
 .data          0x0000000000000e1d        0x0 ../lib/freecom.lib(cd_dir.obj)
 .data          0x0000000000000e1d        0x0 ../lib/freecom.lib(cgetch.obj)
 .data          0x0000000000000e1d        0x0 ../lib/freecom.lib(chgctxt.obj)
 .data          0x0000000000000e1d        0x0 ../lib/freecom.lib(chgdrv.obj)
 .data          0x0000000000000e1d        0x0 ../lib/freecom.lib(chgenv.obj)
 .data          0x0000000000000e1d        0x0 ../lib/freecom.lib(chgenvc.obj)
 .data          0x0000000000000e1d        0x0 ../lib/freecom.lib(chgenvr.obj)
 .data          0x0000000000000e1d        0x0 ../lib/freecom.lib(cmdinput.obj)
 .data          0x0000000000000e1d        0x0 ../lib/freecom.lib(critrchk.obj)
 .data          0x0000000000000e1d        0x0 ../lib/freecom.lib(ctxt.obj)
 .data          0x0000000000000e1d        0x0 ../lib/freecom.lib(ctxt_clr.obj)
 .data          0x0000000000000e1d        0x0 ../lib/freecom.lib(ctxt_get.obj)
 *fill*         0x0000000000000e1d        0x1 
 .data          0x0000000000000e1e       0x30 ../lib/freecom.lib(ctxt_inf.obj)
                0x0000000000000e1e                ctxt_info
 .data          0x0000000000000e4e        0x0 ../lib/freecom.lib(ctxt_mk.obj)
 .data          0x0000000000000e4e        0x0 ../lib/freecom.lib(ctxt_mkb.obj)
 .data          0x0000000000000e4e        0x0 ../lib/freecom.lib(ctxt_mkn.obj)
 .data          0x0000000000000e4e        0x0 ../lib/freecom.lib(ctxt_pop.obj)
 .data          0x0000000000000e4e        0x0 ../lib/freecom.lib(ctxt_psh.obj)
 .data          0x0000000000000e4e        0x0 ../lib/freecom.lib(ctxt_rnu.obj)
 .data          0x0000000000000e4e        0x0 ../lib/freecom.lib(ctxt_set.obj)
 .data          0x0000000000000e4e        0x0 ../lib/freecom.lib(ctxt_vw.obj)
 .data          0x0000000000000e4e        0x0 ../lib/freecom.lib(curdatel.obj)
 .data          0x0000000000000e4e        0x0 ../lib/freecom.lib(curtime.obj)
 .data          0x0000000000000e4e        0x0 ../lib/freecom.lib(cwd.obj)
 .data          0x0000000000000e4e        0x0 ../lib/freecom.lib(dateget.obj)
 .data          0x0000000000000e4e        0x0 ../lib/freecom.lib(dateset.obj)
 .data          0x0000000000000e4e        0x0 ../lib/freecom.lib(devopen.obj)
 .data          0x0000000000000e4e        0x0 ../lib/freecom.lib(dfn_err.obj)
 .data          0x0000000000000e4e        0x0 ../lib/freecom.lib(dispcnt.obj)
 .data          0x0000000000000e4e        0x0 ../lib/freecom.lib(drvnum.obj)
 .data          0x0000000000000e4e        0x0 ../lib/freecom.lib(exec.obj)
 .data          0x0000000000000e4e        0x0 ../lib/freecom.lib(exec1.obj)
 .data          0x0000000000000e4e        0x0 ../lib/freecom.lib(farread.obj)
 .data          0x0000000000000e4e        0x0 ../lib/freecom.lib(filecomp.obj)
 .data          0x0000000000000e4e        0x0 ../lib/freecom.lib(fdattr.obj)
 .data          0x0000000000000e4e        0x0 ../lib/freecom.lib(fdsattr.obj)
 .data          0x0000000000000e4e        0x0 ../lib/freecom.lib(fillcomp.obj)
 .data          0x0000000000000e4e        0x0 ../lib/freecom.lib(find.obj)
 .data          0x0000000000000e4e        0x0 ../lib/freecom.lib(freep.obj)
 .data          0x0000000000000e4e        0x0 ../lib/freecom.lib(gallstr.obj)
 .data          0x0000000000000e4e        0x0 ../lib/freecom.lib(get1mcb.obj)
 .data          0x0000000000000e4e        0x0 ../lib/freecom.lib(getenv.obj)
 .data          0x0000000000000e4e        0x0 ../lib/freecom.lib(goxy.obj)
 .data          0x0000000000000e4e        0x0 ../lib/freecom.lib(grabfcom.obj)
 .data          0x0000000000000e4e        0x0 ../lib/freecom.lib(gumblink.obj)
 .data          0x0000000000000e4e        0x0 ../lib/freecom.lib(hdlrctxt.obj)
 .data          0x0000000000000e4e        0x0 ../lib/freecom.lib(hist_get.obj)
 .data          0x0000000000000e4e        0x0 ../lib/freecom.lib(hist_set.obj)
 .data          0x0000000000000e4e        0x0 ../lib/freecom.lib(is_empty.obj)
 .data          0x0000000000000e4e        0x0 ../lib/freecom.lib(is_fnamc.obj)
 .data          0x0000000000000e4e        0x0 ../lib/freecom.lib(is_fnstr.obj)
 .data          0x0000000000000e4e        0x0 ../lib/freecom.lib(is_pchr.obj)
 .data          0x0000000000000e4e        0x0 ../lib/freecom.lib(isadev.obj)
 .data          0x0000000000000e4e        0x0 ../lib/freecom.lib(lastdget.obj)
 .data          0x0000000000000e4e        0x0 ../lib/freecom.lib(lastdset.obj)
 .data          0x0000000000000e4e        0x0 ../lib/freecom.lib(leadopt.obj)
 .data          0x0000000000000e4e        0x0 ../lib/freecom.lib(lfnfuncs.obj)
 .data          0x0000000000000e4e        0x0 ../lib/freecom.lib(ltrimcl.obj)
 .data          0x0000000000000e4e        0x0 ../lib/freecom.lib(match.obj)
 .data          0x0000000000000e4e        0x2 ../lib/freecom.lib(messages.obj)
 .data          0x0000000000000e50        0x0 ../lib/freecom.lib(mk_rddir.obj)
 .data          0x0000000000000e50        0x0 ../lib/freecom.lib(msg_dps.obj)
 .data          0x0000000000000e50        0x0 ../lib/freecom.lib(msg_fstr.obj)
 .data          0x0000000000000e50        0x0 ../lib/freecom.lib(msg_gpt.obj)
 .data          0x0000000000000e50        0x0 ../lib/freecom.lib(msg_mkey.obj)
 .data          0x0000000000000e50        0x0 ../lib/freecom.lib(msg_prmp.obj)
 .data          0x0000000000000e50        0x0 ../lib/freecom.lib(mux_ae.obj)
 .data          0x0000000000000e50        0x0 ../lib/freecom.lib(myperror.obj)
 .data          0x0000000000000e50        0x0 ../lib/freecom.lib(nls.obj)
 .data          0x0000000000000e50        0x0 ../lib/freecom.lib(nls_date.obj)
 .data          0x0000000000000e50        0x0 ../lib/freecom.lib(nls_time.obj)
 .data          0x0000000000000e50        0x0 ../lib/freecom.lib(num_fmt.obj)
 .data          0x0000000000000e50        0x0 ../lib/freecom.lib(onoff.obj)
 .data          0x0000000000000e50        0x0 ../lib/freecom.lib(openf.obj)
 .data          0x0000000000000e50        0x0 ../lib/freecom.lib(optsb.obj)
 .data          0x0000000000000e50        0x0 ../lib/freecom.lib(optsi.obj)
 .data          0x0000000000000e50        0x0 ../lib/freecom.lib(optss.obj)
 .data          0x0000000000000e50        0x0 ../lib/freecom.lib(pr_date.obj)
 .data          0x0000000000000e50        0x0 ../lib/freecom.lib(pr_prmpt.obj)
 .data          0x0000000000000e50        0x0 ../lib/freecom.lib(pr_time.obj)
 .data          0x0000000000000e50        0x4 ../lib/freecom.lib(prf.obj)
                0x0000000000000e50                stderr
                0x0000000000000e52                stdout
 .data          0x0000000000000e54        0x0 ../lib/freecom.lib(prprompt.obj)
 .data          0x0000000000000e54        0x2 ../lib/freecom.lib(readcmd.obj)
 .data          0x0000000000000e56        0x0 ../lib/freecom.lib(realnum.obj)
 .data          0x0000000000000e56        0x0 ../lib/freecom.lib(res.obj)
 .data          0x0000000000000e56        0x0 ../lib/freecom.lib(res_r.obj)
 .data          0x0000000000000e56        0x0 ../lib/freecom.lib(res_vald.obj)
 .data          0x0000000000000e56        0x0 ../lib/freecom.lib(resfile.obj)
 .data          0x0000000000000e56        0x0 ../lib/freecom.lib(rmtmpfil.obj)
 .data          0x0000000000000e56        0x0 ../lib/freecom.lib(rtrimcl.obj)
 .data          0x0000000000000e56        0x0 ../lib/freecom.lib(rtrimsp.obj)
 .data          0x0000000000000e56        0x0 ../lib/freecom.lib(salloc.obj)
 .data          0x0000000000000e56        0x0 ../lib/freecom.lib(samefile.obj)
 .data          0x0000000000000e56        0x0 ../lib/freecom.lib(scancmd.obj)
 .data          0x0000000000000e56        0x0 ../lib/freecom.lib(scanopt.obj)
 .data          0x0000000000000e56        0x0 ../lib/freecom.lib(session.obj)
 .data          0x0000000000000e56        0x0 ../lib/freecom.lib(showcmds.obj)
 .data          0x0000000000000e56        0x0 ../lib/freecom.lib(skqwd.obj)
 .data          0x0000000000000e56        0x0 ../lib/freecom.lib(spfnam.obj)
 .data          0x0000000000000e56        0x0 ../lib/freecom.lib(split.obj)
 .data          0x0000000000000e56        0x0 ../lib/freecom.lib(sumblink.obj)
 .data          0x0000000000000e56        0x0 ../lib/freecom.lib(timeget.obj)
 .data          0x0000000000000e56        0x0 ../lib/freecom.lib(timeset.obj)
 .data          0x0000000000000e56        0x4 ../lib/freecom.lib(tmpnam.obj)
 .data          0x0000000000000e5a        0x0 ../lib/freecom.lib(trimsp.obj)
 .data          0x0000000000000e5a        0x0 ../lib/freecom.lib(truepath.obj)
 .data          0x0000000000000e5a        0x0 ../lib/freecom.lib(truncate.obj)
 .data          0x0000000000000e5a        0x0 ../lib/freecom.lib(txtlend.obj)
 .data          0x0000000000000e5a        0x0 ../lib/freecom.lib(unquote.obj)
 .data          0x0000000000000e5a        0x0 ../lib/freecom.lib(vcgetch.obj)
 .data          0x0000000000000e5a        0x0 ../lib/freecom.lib(where.obj)
 .data          0x0000000000000e5a        0x0 ../lib/freecom.lib(delay.obj)
 .data          0x0000000000000e5a        0x0 ../lib/freecom.lib(err2.obj)
 .data          0x0000000000000e5a        0x0 ../lib/freecom.lib(err3.obj)
 .data          0x0000000000000e5a        0x0 ../lib/freecom.lib(err5.obj)
 .data          0x0000000000000e5a        0x0 ../lib/freecom.lib(err6.obj)
 .data          0x0000000000000e5a        0x0 ../lib/freecom.lib(err7.obj)
 .data          0x0000000000000e5a        0x0 ../lib/freecom.lib(err8.obj)
 .data          0x0000000000000e5a        0x0 ../lib/freecom.lib(err10.obj)
 .data          0x0000000000000e5a        0x0 ../lib/freecom.lib(err11.obj)
 .data          0x0000000000000e5a        0x0 ../lib/freecom.lib(err13.obj)
 .data          0x0000000000000e5a        0x0 ../lib/freecom.lib(err14.obj)
 .data          0x0000000000000e5a        0x0 ../lib/freecom.lib(err15.obj)
 .data          0x0000000000000e5a        0x0 ../lib/freecom.lib(err16.obj)
 .data          0x0000000000000e5a        0x0 ../lib/freecom.lib(err17.obj)
 .data          0x0000000000000e5a        0x0 ../lib/freecom.lib(err18.obj)
 .data          0x0000000000000e5a        0x0 ../lib/freecom.lib(err19.obj)
 .data          0x0000000000000e5a        0x0 ../lib/freecom.lib(err20.obj)
 .data          0x0000000000000e5a        0x0 ../lib/freecom.lib(err21.obj)
 .data          0x0000000000000e5a        0x0 ../lib/freecom.lib(err22.obj)
 .data          0x0000000000000e5a        0x0 ../lib/freecom.lib(err23.obj)
 .data          0x0000000000000e5a        0x0 ../lib/freecom.lib(err25.obj)
 .data          0x0000000000000e5a        0x0 ../lib/freecom.lib(err26.obj)
 .data          0x0000000000000e5a        0x0 ../lib/freecom.lib(err27.obj)
 .data          0x0000000000000e5a        0x0 ../lib/freecom.lib(err28.obj)
 .data          0x0000000000000e5a        0x0 ../lib/freecom.lib(err29.obj)
 .data          0x0000000000000e5a        0x0 ../lib/freecom.lib(err30.obj)
 .data          0x0000000000000e5a        0x0 ../lib/freecom.lib(err31.obj)
 .data          0x0000000000000e5a        0x0 ../lib/freecom.lib(err32.obj)
 .data          0x0000000000000e5a        0x0 ../lib/freecom.lib(err33.obj)
 .data          0x0000000000000e5a        0x0 ../lib/freecom.lib(err34.obj)
 .data          0x0000000000000e5a        0x0 ../lib/freecom.lib(err35.obj)
 .data          0x0000000000000e5a        0x0 ../lib/freecom.lib(err36.obj)
 .data          0x0000000000000e5a        0x0 ../lib/freecom.lib(err37.obj)
 .data          0x0000000000000e5a        0x0 ../lib/freecom.lib(err38.obj)
 .data          0x0000000000000e5a        0x0 ../lib/freecom.lib(err39.obj)
 .data          0x0000000000000e5a        0x0 ../lib/freecom.lib(err41.obj)
 .data          0x0000000000000e5a        0x0 ../lib/freecom.lib(err42.obj)
 .data          0x0000000000000e5a        0x0 ../lib/freecom.lib(err45.obj)
 .data          0x0000000000000e5a        0x0 ../lib/freecom.lib(err46.obj)
 .data          0x0000000000000e5a        0x0 ../lib/freecom.lib(err47.obj)
 .data          0x0000000000000e5a        0x0 ../lib/freecom.lib(err50.obj)
 .data          0x0000000000000e5a        0x0 ../lib/freecom.lib(err51.obj)
 .data          0x0000000000000e5a        0x0 ../lib/freecom.lib(err53.obj)
 .data          0x0000000000000e5a        0x0 ../lib/freecom.lib(err54.obj)
 .data          0x0000000000000e5a        0x0 ../lib/freecom.lib(err58.obj)
 .data          0x0000000000000e5a        0x0 ../lib/freecom.lib(err59.obj)
 .data          0x0000000000000e5a        0x0 ../lib/freecom.lib(err60.obj)
 .data          0x0000000000000e5a        0x0 ../lib/freecom.lib(err61.obj)
 .data          0x0000000000000e5a        0x0 ../lib/freecom.lib(err63.obj)
 .data          0x0000000000000e5a        0x0 ../lib/freecom.lib(err64.obj)
 .data          0x0000000000000e5a        0x0 ../lib/freecom.lib(err65.obj)
 .data          0x0000000000000e5a        0x0 ../lib/freecom.lib(err67.obj)
 .data          0x0000000000000e5a        0x0 ../lib/freecom.lib(err68.obj)
 .data          0x0000000000000e5a        0x0 ../lib/freecom.lib(err69.obj)
 .data          0x0000000000000e5a        0x0 ../lib/freecom.lib(err70.obj)
 .data          0x0000000000000e5a        0x0 ../lib/freecom.lib(err71.obj)
 .data          0x0000000000000e5a        0x0 ../lib/freecom.lib(err72.obj)
 .data          0x0000000000000e5a        0x0 ../lib/freecom.lib(err73.obj)
 .data          0x0000000000000e5a        0x0 ../lib/freecom.lib(err74.obj)
 .data          0x0000000000000e5a        0x0 ../lib/freecom.lib(err75.obj)
 .data          0x0000000000000e5a        0x0 ../lib/freecom.lib(err76.obj)
 .data          0x0000000000000e5a        0x0 ../lib/freecom.lib(err77.obj)
 .data          0x0000000000000e5a        0x0 ../lib/freecom.lib(err78.obj)
 .data          0x0000000000000e5a        0x0 ../lib/freecom.lib(err79.obj)
 .data          0x0000000000000e5a        0x0 ../lib/freecom.lib(err80.obj)
 .data          0x0000000000000e5a        0x0 ../lib/freecom.lib(err81.obj)
 .data          0x0000000000000e5a        0x0 ../lib/freecom.lib(err82.obj)
 .data          0x0000000000000e5a        0x0 ../lib/freecom.lib(err83.obj)
 .data          0x0000000000000e5a        0x0 ../lib/freecom.lib(err84.obj)
 .data          0x0000000000000e5a        0x0 ../lib/freecom.lib(err85.obj)
 .data          0x0000000000000e5a        0x0 ../lib/freecom.lib(err86.obj)
 .data          0x0000000000000e5a        0x0 ../lib/freecom.lib(err87.obj)
 .data          0x0000000000000e5a        0x0 ../lib/freecom.lib(almemblk.obj)
 .data          0x0000000000000e5a        0x0 ../lib/freecom.lib(beep_l.obj)
 .data          0x0000000000000e5a        0x0 ../lib/freecom.lib(cbs.obj)
 .data          0x0000000000000e5a        0x0 ../lib/freecom.lib(comfile.obj)
 .data          0x0000000000000e5a        0x0 ../lib/freecom.lib(ctxt_as.obj)
 .data          0x0000000000000e5a        0x0 ../lib/freecom.lib(dispexit.obj)
 .data          0x0000000000000e5a       0xff ../lib/freecom.lib(inputdos.obj)
 .data          0x0000000000000f59        0x0 ../lib/freecom.lib(ltrimsp.obj)
 .data          0x0000000000000f59        0x0 ../lib/freecom.lib(mktmpfil.obj)
 .data          0x0000000000000f59        0x0 ../lib/freecom.lib(msg_dflt.obj)
 .data          0x0000000000000f59        0x0 ../lib/freecom.lib(msg_get.obj)
 .data          0x0000000000000f59        0x0 ../lib/freecom.lib(parsenum.obj)
 .data          0x0000000000000f59        0x0 ../strings/strings.lib(str0011.obj)
 .data          0x0000000000000f59        0x0 ../strings/strings.lib(str0018.obj)
 .data          0x0000000000000f59        0x0 ../strings/strings.lib(str003c.obj)
 .data          0x0000000000000f59        0x0 ../strings/strings.lib(str00b1.obj)
 .data          0x0000000000000f59        0x0 ../strings/strings.lib(str00b2.obj)
 .data          0x0000000000000f59        0x0 ../strings/strings.lib(str00f4.obj)
 .data          0x0000000000000f59        0x0 ../strings/strings.lib(str00f5.obj)
 .data          0x0000000000000f59        0x0 ../strings/strings.lib(str00f6.obj)
 .data          0x0000000000000f59        0x0 ../suppl/suppl_s.lib(byte2par.obj)
 .data          0x0000000000000f59        0xf ../suppl/suppl_s.lib(cntry.obj)
 .data          0x0000000000000f68        0x0 ../suppl/suppl_s.lib(dfnfnam.obj)
 .data          0x0000000000000f68        0x0 ../suppl/suppl_s.lib(dfnfullp.obj)
 .data          0x0000000000000f68        0x0 ../suppl/suppl_s.lib(dfnmerge.obj)
 .data          0x0000000000000f68        0x0 ../suppl/suppl_s.lib(dfnpath.obj)
 .data          0x0000000000000f68        0x0 ../suppl/suppl_s.lib(dfnstat.obj)
 .data          0x0000000000000f68        0x0 ../suppl/suppl_s.lib(dfntruen.obj)
 .data          0x0000000000000f68        0x0 ../suppl/suppl_s.lib(dosalloc.obj)
 .data          0x0000000000000f68        0x0 ../suppl/suppl_s.lib(dosfree.obj)
 .data          0x0000000000000f68        0x0 ../suppl/suppl_s.lib(dossize.obj)
 .data          0x0000000000000f68        0x0 ../suppl/suppl_s.lib(dstrfupr.obj)
 .data          0x0000000000000f68        0x0 ../suppl/suppl_s.lib(dstrtrim.obj)
 .data          0x0000000000000f68        0x0 ../suppl/suppl_s.lib(dstrupr.obj)
 .data          0x0000000000000f68        0x0 ../suppl/suppl_s.lib(enoallc.obj)
 .data          0x0000000000000f68        0x0 ../suppl/suppl_s.lib(enoreal.obj)
 .data          0x0000000000000f68        0x0 ../suppl/suppl_s.lib(enosetos.obj)
 .data          0x0000000000000f68        0x0 ../suppl/suppl_s.lib(env_chg.obj)
 .data          0x0000000000000f68        0x0 ../suppl/suppl_s.lib(env_dvar.obj)
 .data          0x0000000000000f68        0x0 ../suppl/suppl_s.lib(env_find.obj)
 .data          0x0000000000000f68        0x0 ../suppl/suppl_s.lib(env_fora.obj)
 .data          0x0000000000000f68        0x0 ../suppl/suppl_s.lib(env_free.obj)
 .data          0x0000000000000f68        0x0 ../suppl/suppl_s.lib(env_insv.obj)
 .data          0x0000000000000f68        0x0 ../suppl/suppl_s.lib(env_len.obj)
 .data          0x0000000000000f68        0x0 ../suppl/suppl_s.lib(env_mtch.obj)
 .data          0x0000000000000f68        0x0 ../suppl/suppl_s.lib(env_new.obj)
 .data          0x0000000000000f68        0x0 ../suppl/suppl_s.lib(env_nost.obj)
 .data          0x0000000000000f68        0x0 ../suppl/suppl_s.lib(env_ovrw.obj)
 .data          0x0000000000000f68        0x0 ../suppl/suppl_s.lib(env_repl.obj)
 .data          0x0000000000000f68        0x0 ../suppl/suppl_s.lib(env_rlsg.obj)
 .data          0x0000000000000f68        0x0 ../suppl/suppl_s.lib(env_scnt.obj)
 .data          0x0000000000000f68        0x0 ../suppl/suppl_s.lib(env_size.obj)
 .data          0x0000000000000f68        0x0 ../suppl/suppl_s.lib(env_strg.obj)
 .data          0x0000000000000f68        0x0 ../suppl/suppl_s.lib(env_sub.obj)
 .data          0x0000000000000f68        0x2 ../suppl/suppl_s.lib(env_var1.obj)
                0x0000000000000f68                env_resizeCtrl
 .data          0x0000000000000f6a        0x0 ../suppl/suppl_s.lib(env_var2.obj)
 .data          0x0000000000000f6a        0x0 ../suppl/suppl_s.lib(fstrdup.obj)
 .data          0x0000000000000f6a        0x0 ../suppl/suppl_s.lib(mcb_is.obj)
 .data          0x0000000000000f6a        0x0 ../suppl/suppl_s.lib(mcb_leng.obj)
 .data          0x0000000000000f6a        0x0 ../suppl/suppl_s.lib(mcb_nxt.obj)
 .data          0x0000000000000f6a        0x0 ../suppl/suppl_s.lib(mcb_walk.obj)
 .data          0x0000000000000f6a        0x0 ../suppl/suppl_s.lib(toupperx.obj)
 .data          0x0000000000000f6a        0x0 ../suppl/suppl_s.lib(filefind.obj)
 .data          0x0000000000000f6a        0x0 ../suppl/suppl_s.lib(invokedo.obj)
 .data          0x0000000000000f6a        0x0 ../suppl/suppl_s.lib(addu.obj)
 .data          0x0000000000000f6a        0x0 ../suppl/suppl_s.lib(dfndeli2.obj)
 .data          0x0000000000000f6a        0x0 ../suppl/suppl_s.lib(dfndelim.obj)
 .data          0x0000000000000f6a        0x0 ../suppl/suppl_s.lib(dfnexpan.obj)
 .data          0x0000000000000f6a        0x0 ../suppl/suppl_s.lib(dfnsplit.obj)
 .data          0x0000000000000f6a        0x0 ../suppl/suppl_s.lib(dfnsquee.obj)
 .data          0x0000000000000f6a        0x0 ../suppl/suppl_s.lib(dmemcmpf.obj)
 .data          0x0000000000000f6a        0x0 ../suppl/suppl_s.lib(dstrchar.obj)
 .data          0x0000000000000f6a        0x0 ../suppl/suppl_s.lib(dstrleft.obj)
 .data          0x0000000000000f6a        0x0 ../suppl/suppl_s.lib(dstrrepl.obj)
 .data          0x0000000000000f6a        0x0 ../suppl/suppl_s.lib(enosdup.obj)
 .data          0x0000000000000f6a        0x0 ../suppl/suppl_s.lib(env_del.obj)
 .data          0x0000000000000f6a        0x0 ../suppl/suppl_s.lib(mcb_1st.obj)
 .data          0x0000000000000f6a        0x0 /home/evln/proj/build-ia16.202501/prefix/bin/../lib/gcc/ia16-elf/6.3.0/../../../../ia16-elf/lib/regparmcall/libi86.a(fmemchr.o)
 .data          0x0000000000000f6a        0x0 /home/evln/proj/build-ia16.202501/prefix/bin/../lib/gcc/ia16-elf/6.3.0/../../../../ia16-elf/lib/regparmcall/libi86.a(fmemcmp.o)
 .data          0x0000000000000f6a        0x0 /home/evln/proj/build-ia16.202501/prefix/bin/../lib/gcc/ia16-elf/6.3.0/../../../../ia16-elf/lib/regparmcall/libi86.a(fmemcpy.o)
 .data          0x0000000000000f6a        0x0 /home/evln/proj/build-ia16.202501/prefix/bin/../lib/gcc/ia16-elf/6.3.0/../../../../ia16-elf/lib/regparmcall/libi86.a(fmemmove.o)
 .data          0x0000000000000f6a        0x0 /home/evln/proj/build-ia16.202501/prefix/bin/../lib/gcc/ia16-elf/6.3.0/../../../../ia16-elf/lib/regparmcall/libi86.a(fstrcpy.o)
 .data          0x0000000000000f6a        0x0 /home/evln/proj/build-ia16.202501/prefix/bin/../lib/gcc/ia16-elf/6.3.0/../../../../ia16-elf/lib/regparmcall/libi86.a(fstrlen.o)
 .data          0x0000000000000f6a        0x0 /home/evln/proj/build-ia16.202501/prefix/bin/../lib/gcc/ia16-elf/6.3.0/../../../../ia16-elf/lib/regparmcall/libi86.a(libi86-fmemmove-backward.o)
 .data          0x0000000000000f6a        0x0 /home/evln/proj/build-ia16.202501/prefix/bin/../lib/gcc/ia16-elf/6.3.0/../../../../ia16-elf/lib/regparmcall/libi86.a(getdcwd.o)
 .data          0x0000000000000f6a        0x0 /home/evln/proj/build-ia16.202501/prefix/bin/../lib/gcc/ia16-elf/6.3.0/../../../../ia16-elf/lib/regparmcall/libi86.a(getdrive.o)
 .data          0x0000000000000f6a        0x2 /home/evln/proj/build-ia16.202501/prefix/bin/../lib/gcc/ia16-elf/6.3.0/regparmcall/crtbegin.o
                0x0000000000000f6a                __dso_handle
 .data          0x0000000000000f6c        0x0 /home/evln/proj/build-ia16.202501/prefix/bin/../lib/gcc/ia16-elf/6.3.0/regparmcall/crtend.o
 .data          0x0000000000000f6c        0x0 /home/evln/proj/build-ia16.202501/prefix/bin/../lib/gcc/ia16-elf/6.3.0/../../../../ia16-elf/lib/regparmcall/dos-s-c0.o
 .data          0x0000000000000f6c        0x0 /home/evln/proj/build-ia16.202501/prefix/bin/../lib/gcc/ia16-elf/6.3.0/../../../../ia16-elf/lib/regparmcall/libc.a(lib_a-atexit.o)
 .data          0x0000000000000f6c        0x0 /home/evln/proj/build-ia16.202501/prefix/bin/../lib/gcc/ia16-elf/6.3.0/../../../../ia16-elf/lib/regparmcall/libc.a(lib_a-atol.o)
 .data          0x0000000000000f6c        0x2 /home/evln/proj/build-ia16.202501/prefix/bin/../lib/gcc/ia16-elf/6.3.0/../../../../ia16-elf/lib/regparmcall/libc.a(lib_a-ctype_.o)
                0x0000000000000f6c                __ctype_ptr__
 .data          0x0000000000000f6e        0x0 /home/evln/proj/build-ia16.202501/prefix/bin/../lib/gcc/ia16-elf/6.3.0/../../../../ia16-elf/lib/regparmcall/libc.a(lib_a-errno.o)
 .data          0x0000000000000f6e        0x0 /home/evln/proj/build-ia16.202501/prefix/bin/../lib/gcc/ia16-elf/6.3.0/../../../../ia16-elf/lib/regparmcall/libc.a(lib_a-exit.o)
 .data          0x0000000000000f6e       0x32 /home/evln/proj/build-ia16.202501/prefix/bin/../lib/gcc/ia16-elf/6.3.0/../../../../ia16-elf/lib/regparmcall/libc.a(lib_a-impure.o)
                0x0000000000000f6e                _impure_ptr
 .data          0x0000000000000fa0        0x0 /home/evln/proj/build-ia16.202501/prefix/bin/../lib/gcc/ia16-elf/6.3.0/../../../../ia16-elf/lib/regparmcall/libc.a(lib_a-malloc.o)
 .data          0x0000000000000fa0        0x0 /home/evln/proj/build-ia16.202501/prefix/bin/../lib/gcc/ia16-elf/6.3.0/../../../../ia16-elf/lib/regparmcall/libc.a(lib_a-memchr.o)
 .data          0x0000000000000fa0        0x0 /home/evln/proj/build-ia16.202501/prefix/bin/../lib/gcc/ia16-elf/6.3.0/../../../../ia16-elf/lib/regparmcall/libc.a(lib_a-memcmp.o)
 .data          0x0000000000000fa0        0x0 /home/evln/proj/build-ia16.202501/prefix/bin/../lib/gcc/ia16-elf/6.3.0/../../../../ia16-elf/lib/regparmcall/libc.a(lib_a-memcpy.o)
 .data          0x0000000000000fa0        0x0 /home/evln/proj/build-ia16.202501/prefix/bin/../lib/gcc/ia16-elf/6.3.0/../../../../ia16-elf/lib/regparmcall/libc.a(lib_a-memmove.o)
 .data          0x0000000000000fa0        0x0 /home/evln/proj/build-ia16.202501/prefix/bin/../lib/gcc/ia16-elf/6.3.0/../../../../ia16-elf/lib/regparmcall/libc.a(lib_a-memset.o)
 .data          0x0000000000000fa0        0x0 /home/evln/proj/build-ia16.202501/prefix/bin/../lib/gcc/ia16-elf/6.3.0/../../../../ia16-elf/lib/regparmcall/libc.a(lib_a-nano-freer.o)
 .data          0x0000000000000fa0        0x0 /home/evln/proj/build-ia16.202501/prefix/bin/../lib/gcc/ia16-elf/6.3.0/../../../../ia16-elf/lib/regparmcall/libc.a(lib_a-nano-mallocr.o)
 .data          0x0000000000000fa0        0x0 /home/evln/proj/build-ia16.202501/prefix/bin/../lib/gcc/ia16-elf/6.3.0/../../../../ia16-elf/lib/regparmcall/libc.a(lib_a-qsort.o)
 .data          0x0000000000000fa0        0x0 /home/evln/proj/build-ia16.202501/prefix/bin/../lib/gcc/ia16-elf/6.3.0/../../../../ia16-elf/lib/regparmcall/libc.a(lib_a-realloc.o)
 .data          0x0000000000000fa0        0x0 /home/evln/proj/build-ia16.202501/prefix/bin/../lib/gcc/ia16-elf/6.3.0/../../../../ia16-elf/lib/regparmcall/libc.a(lib_a-remove.o)
 .data          0x0000000000000fa0        0x0 /home/evln/proj/build-ia16.202501/prefix/bin/../lib/gcc/ia16-elf/6.3.0/../../../../ia16-elf/lib/regparmcall/libc.a(lib_a-setjmp.o)
 .data          0x0000000000000fa0        0x0 /home/evln/proj/build-ia16.202501/prefix/bin/../lib/gcc/ia16-elf/6.3.0/../../../../ia16-elf/lib/regparmcall/libc.a(lib_a-stpcpy.o)
 .data          0x0000000000000fa0        0x0 /home/evln/proj/build-ia16.202501/prefix/bin/../lib/gcc/ia16-elf/6.3.0/../../../../ia16-elf/lib/regparmcall/libc.a(lib_a-strcasecmp.o)
 .data          0x0000000000000fa0        0x0 /home/evln/proj/build-ia16.202501/prefix/bin/../lib/gcc/ia16-elf/6.3.0/../../../../ia16-elf/lib/regparmcall/libc.a(lib_a-strcat.o)
 .data          0x0000000000000fa0        0x0 /home/evln/proj/build-ia16.202501/prefix/bin/../lib/gcc/ia16-elf/6.3.0/../../../../ia16-elf/lib/regparmcall/libc.a(lib_a-strchr.o)
 .data          0x0000000000000fa0        0x0 /home/evln/proj/build-ia16.202501/prefix/bin/../lib/gcc/ia16-elf/6.3.0/../../../../ia16-elf/lib/regparmcall/libc.a(lib_a-strcmp.o)
 .data          0x0000000000000fa0        0x0 /home/evln/proj/build-ia16.202501/prefix/bin/../lib/gcc/ia16-elf/6.3.0/../../../../ia16-elf/lib/regparmcall/libc.a(lib_a-strcpy.o)
 .data          0x0000000000000fa0        0x0 /home/evln/proj/build-ia16.202501/prefix/bin/../lib/gcc/ia16-elf/6.3.0/../../../../ia16-elf/lib/regparmcall/libc.a(lib_a-strdup.o)
 .data          0x0000000000000fa0        0x0 /home/evln/proj/build-ia16.202501/prefix/bin/../lib/gcc/ia16-elf/6.3.0/../../../../ia16-elf/lib/regparmcall/libc.a(lib_a-strdup_r.o)
 .data          0x0000000000000fa0        0x0 /home/evln/proj/build-ia16.202501/prefix/bin/../lib/gcc/ia16-elf/6.3.0/../../../../ia16-elf/lib/regparmcall/libc.a(lib_a-strlen.o)
 .data          0x0000000000000fa0        0x0 /home/evln/proj/build-ia16.202501/prefix/bin/../lib/gcc/ia16-elf/6.3.0/../../../../ia16-elf/lib/regparmcall/libc.a(lib_a-strlwr.o)
 .data          0x0000000000000fa0        0x0 /home/evln/proj/build-ia16.202501/prefix/bin/../lib/gcc/ia16-elf/6.3.0/../../../../ia16-elf/lib/regparmcall/libc.a(lib_a-strncasecmp.o)
 .data          0x0000000000000fa0        0x0 /home/evln/proj/build-ia16.202501/prefix/bin/../lib/gcc/ia16-elf/6.3.0/../../../../ia16-elf/lib/regparmcall/libc.a(lib_a-strncpy.o)
 .data          0x0000000000000fa0        0x0 /home/evln/proj/build-ia16.202501/prefix/bin/../lib/gcc/ia16-elf/6.3.0/../../../../ia16-elf/lib/regparmcall/libc.a(lib_a-strpbrk.o)
 .data          0x0000000000000fa0        0x0 /home/evln/proj/build-ia16.202501/prefix/bin/../lib/gcc/ia16-elf/6.3.0/../../../../ia16-elf/lib/regparmcall/libc.a(lib_a-strrchr.o)
 .data          0x0000000000000fa0        0x0 /home/evln/proj/build-ia16.202501/prefix/bin/../lib/gcc/ia16-elf/6.3.0/../../../../ia16-elf/lib/regparmcall/libc.a(lib_a-strspn.o)
 .data          0x0000000000000fa0        0x0 /home/evln/proj/build-ia16.202501/prefix/bin/../lib/gcc/ia16-elf/6.3.0/../../../../ia16-elf/lib/regparmcall/libc.a(lib_a-strtok.o)
 .data          0x0000000000000fa0        0x0 /home/evln/proj/build-ia16.202501/prefix/bin/../lib/gcc/ia16-elf/6.3.0/../../../../ia16-elf/lib/regparmcall/libc.a(lib_a-strtok_r.o)
 .data          0x0000000000000fa0        0x0 /home/evln/proj/build-ia16.202501/prefix/bin/../lib/gcc/ia16-elf/6.3.0/../../../../ia16-elf/lib/regparmcall/libc.a(lib_a-strtol.o)
 .data          0x0000000000000fa0        0x0 /home/evln/proj/build-ia16.202501/prefix/bin/../lib/gcc/ia16-elf/6.3.0/../../../../ia16-elf/lib/regparmcall/libc.a(lib_a-sysisatty.o)
 .data          0x0000000000000fa0        0x0 /home/evln/proj/build-ia16.202501/prefix/bin/../lib/gcc/ia16-elf/6.3.0/../../../../ia16-elf/lib/regparmcall/libc.a(lib_a-syslseek.o)
 .data          0x0000000000000fa0        0x0 /home/evln/proj/build-ia16.202501/prefix/bin/../lib/gcc/ia16-elf/6.3.0/../../../../ia16-elf/lib/regparmcall/libc.a(lib_a-sysunlink.o)
 .data          0x0000000000000fa0        0x0 /home/evln/proj/build-ia16.202501/prefix/bin/../lib/gcc/ia16-elf/6.3.0/../../../../ia16-elf/lib/regparmcall/libc.a(lib_a-syswrite.o)
 .data          0x0000000000000fa0        0x0 /home/evln/proj/build-ia16.202501/prefix/bin/../lib/gcc/ia16-elf/6.3.0/../../../../ia16-elf/lib/regparmcall/libc.a(lib_a-toupper.o)
 .data          0x0000000000000fa0        0x0 /home/evln/proj/build-ia16.202501/prefix/bin/../lib/gcc/ia16-elf/6.3.0/../../../../ia16-elf/lib/regparmcall/libc.a(lib_a-__atexit.o)
 .data          0x0000000000000fa0        0x0 /home/evln/proj/build-ia16.202501/prefix/bin/../lib/gcc/ia16-elf/6.3.0/../../../../ia16-elf/lib/regparmcall/libc.a(lib_a-__call_atexit.o)
 .data          0x0000000000000fa0        0x0 /home/evln/proj/build-ia16.202501/prefix/bin/../lib/gcc/ia16-elf/6.3.0/../../../../ia16-elf/lib/regparmcall/libc.a(lib_a-nano-reallocr.o)
 .data          0x0000000000000fa0        0x0 /home/evln/proj/build-ia16.202501/prefix/bin/../lib/gcc/ia16-elf/6.3.0/../../../../ia16-elf/lib/regparmcall/libc.a(lib_a-nano-msizer.o)
 .data          0x0000000000000fa0        0x0 /home/evln/proj/build-ia16.202501/prefix/bin/../lib/gcc/ia16-elf/6.3.0/regparmcall/libgcc.a(udivsi3.o)
 .data          0x0000000000000fa0        0x0 /home/evln/proj/build-ia16.202501/prefix/bin/../lib/gcc/ia16-elf/6.3.0/regparmcall/libgcc.a(umodsi3.o)
 .data          0x0000000000000fa0        0x0 /home/evln/proj/build-ia16.202501/prefix/bin/../lib/gcc/ia16-elf/6.3.0/regparmcall/libgcc.a(ia16-ldivmodu.o)
 .data          0x0000000000000fa0        0x0 /home/evln/proj/build-ia16.202501/prefix/bin/../lib/gcc/ia16-elf/6.3.0/../../../../ia16-elf/lib/regparmcall/libdos-s.a(dos-isattyr.o)
 .data          0x0000000000000fa0        0x0 /home/evln/proj/build-ia16.202501/prefix/bin/../lib/gcc/ia16-elf/6.3.0/../../../../ia16-elf/lib/regparmcall/libdos-s.a(dos-lseekr.o)
 .data          0x0000000000000fa0        0x2 /home/evln/proj/build-ia16.202501/prefix/bin/../lib/gcc/ia16-elf/6.3.0/../../../../ia16-elf/lib/regparmcall/libdos-s.a(dos-sbrkr.o)
 .data          0x0000000000000fa2        0x0 /home/evln/proj/build-ia16.202501/prefix/bin/../lib/gcc/ia16-elf/6.3.0/../../../../ia16-elf/lib/regparmcall/libdos-s.a(dos-unlinkr.o)
 .data          0x0000000000000fa2        0x0 /home/evln/proj/build-ia16.202501/prefix/bin/../lib/gcc/ia16-elf/6.3.0/../../../../ia16-elf/lib/regparmcall/libdos-s.a(dos-writer.o)
 .data          0x0000000000000fa2        0x0 /home/evln/proj/build-ia16.202501/prefix/bin/../lib/gcc/ia16-elf/6.3.0/../../../../ia16-elf/lib/regparmcall/libdos-s.a(dos-msmmabort.o)
 .data          0x0000000000000fa2        0x2 /home/evln/proj/build-ia16.202501/prefix/bin/../lib/gcc/ia16-elf/6.3.0/../../../../ia16-elf/lib/regparmcall/libdos-s.a(dos-heaplen.o)
                0x0000000000000fa2                _heaplen
 .data          0x0000000000000fa4        0x0 /home/evln/proj/build-ia16.202501/prefix/bin/../lib/gcc/ia16-elf/6.3.0/../../../../ia16-elf/lib/regparmcall/libdos-s.a(dos-near-data-segment.o)
 .data          0x0000000000000fa4        0x0 /home/evln/proj/build-ia16.202501/prefix/bin/../lib/gcc/ia16-elf/6.3.0/../../../../ia16-elf/lib/regparmcall/libc.a(lib_a-abort.o)
 *(.data.*)
 *(.gcc_except_table)
                0x0000000000000fa4                __edata = .
                0x0000000000000fa4                . = (. == __sdata)?(. + 0x1):.
                0x0000000000000fb0                . = ALIGN (0x10)
 *fill*         0x0000000000000fa4        0xc 
                0x0000000000000fb0                __edata_padded = .

.bss            0x0000000000000fb0      0x50c load address 0x000000000000f1b0
                0x0000000000000fb0                __sbss = .
 *(.bss)
 .bss           0x0000000000000fb0       0x16 cswap.obj
                0x0000000000000fb0                SwapResidentSize
                0x0000000000000fb2                XMSsave
 .bss           0x0000000000000fc6        0x4 cswapc.obj
 .bss           0x0000000000000fca        0x6 batch.obj
                0x0000000000000fca                tracemode
                0x0000000000000fcc                bc
 .bss           0x0000000000000fd0        0x0 cmdtable.obj
 .bss           0x0000000000000fd0       0x16 command.obj
                0x0000000000000fd0                defaultToSwap
                0x0000000000000fd2                swapOnExec
                0x0000000000000fd4                isSwapFile
                0x0000000000000fd6                autofail
                0x0000000000000fd8                forceLow
                0x0000000000000fda                errorlevel
                0x0000000000000fdc                exitflag
                0x0000000000000fde                interactive_command
                0x0000000000000fe0                persistentMSGs
 .bss           0x0000000000000fe6        0x0 expalias.obj
 .bss           0x0000000000000fe6       0x10 init.obj
                0x0000000000000fe6                dispExitcode
 .bss           0x0000000000000ff6        0x0 kswap.obj
 .bss           0x0000000000000ff6       0x10 loadhigh.obj
 .bss           0x0000000000001006        0x0 module.obj
 .bss           0x0000000000001006        0x0 redir.obj
 .bss           0x0000000000001006        0x8 ver.obj
 .bss           0x000000000000100e        0x0 ../cmd/cmds.lib(alias.obj)
 .bss           0x000000000000100e        0x0 ../cmd/cmds.lib(beep.obj)
 .bss           0x000000000000100e        0x0 ../cmd/cmds.lib(break.obj)
 .bss           0x000000000000100e        0x4 ../cmd/cmds.lib(call.obj)
 .bss           0x0000000000001012        0x0 ../cmd/cmds.lib(cdd.obj)
 .bss           0x0000000000001012        0x0 ../cmd/cmds.lib(chcp.obj)
 .bss           0x0000000000001012        0x0 ../cmd/cmds.lib(chdir.obj)
 .bss           0x0000000000001012        0x0 ../cmd/cmds.lib(cls.obj)
 .bss           0x0000000000001012       0x14 ../cmd/cmds.lib(copy.obj)
 .bss           0x0000000000001026        0x0 ../cmd/cmds.lib(ctty.obj)
 .bss           0x0000000000001026        0x2 ../cmd/cmds.lib(date.obj)
 .bss           0x0000000000001028        0x4 ../cmd/cmds.lib(del.obj)
 .bss           0x000000000000102c       0x2a ../cmd/cmds.lib(dir.obj)
 .bss           0x0000000000001056        0x0 ../cmd/cmds.lib(dirs.obj)
 .bss           0x0000000000001056        0x0 ../cmd/cmds.lib(doskey.obj)
 .bss           0x0000000000001056        0x0 ../cmd/cmds.lib(echo.obj)
 .bss           0x0000000000001056        0x0 ../cmd/cmds.lib(exit.obj)
 .bss           0x0000000000001056        0x0 ../cmd/cmds.lib(for.obj)
 .bss           0x0000000000001056        0x0 ../cmd/cmds.lib(goto.obj)
 .bss           0x0000000000001056        0x0 ../cmd/cmds.lib(history.obj)
 .bss           0x0000000000001056        0x0 ../cmd/cmds.lib(if.obj)
 .bss           0x0000000000001056        0x2 ../cmd/cmds.lib(lfnfor.obj)
                0x0000000000001056                lfncomplete
                0x0000000000001057                lfnfor
 .bss           0x0000000000001058        0x0 ../cmd/cmds.lib(memory.obj)
 .bss           0x0000000000001058        0x0 ../cmd/cmds.lib(mkdir.obj)
 .bss           0x0000000000001058        0x0 ../cmd/cmds.lib(path.obj)
 .bss           0x0000000000001058        0x0 ../cmd/cmds.lib(pause.obj)
 .bss           0x0000000000001058        0x0 ../cmd/cmds.lib(popd.obj)
 .bss           0x0000000000001058        0x0 ../cmd/cmds.lib(prompt.obj)
 .bss           0x0000000000001058        0x0 ../cmd/cmds.lib(pushd.obj)
 .bss           0x0000000000001058        0x0 ../cmd/cmds.lib(rem.obj)
 .bss           0x0000000000001058        0x0 ../cmd/cmds.lib(ren.obj)
 .bss           0x0000000000001058      0x20a ../cmd/cmds.lib(rmdir.obj)
 .bss           0x0000000000001262        0x8 ../cmd/cmds.lib(set.obj)
 .bss           0x000000000000126a        0x0 ../cmd/cmds.lib(shift.obj)
 .bss           0x000000000000126a        0x2 ../cmd/cmds.lib(time.obj)
 .bss           0x000000000000126c        0x0 ../cmd/cmds.lib(truename.obj)
 .bss           0x000000000000126c        0x0 ../cmd/cmds.lib(type.obj)
 .bss           0x000000000000126c        0x0 ../cmd/cmds.lib(verify.obj)
 .bss           0x000000000000126c        0x0 ../cmd/cmds.lib(which.obj)
 .bss           0x000000000000126c        0x0 ../lib/freecom.lib(absfile.obj)
 .bss           0x000000000000126c        0x0 ../lib/freecom.lib(app_get.obj)
 .bss           0x000000000000126c        0x0 ../lib/freecom.lib(app_set.obj)
 .bss           0x000000000000126c        0x0 ../lib/freecom.lib(beep_n.obj)
 .bss           0x000000000000126c        0x0 ../lib/freecom.lib(brk_get.obj)
 .bss           0x000000000000126c        0x0 ../lib/freecom.lib(brk_set.obj)
 .bss           0x000000000000126c        0x2 ../lib/freecom.lib(cbreak.obj)
 .bss           0x000000000000126e        0x0 ../lib/freecom.lib(cd_dir.obj)
 .bss           0x000000000000126e        0x0 ../lib/freecom.lib(cgetch.obj)
 .bss           0x000000000000126e        0x0 ../lib/freecom.lib(chgctxt.obj)
 .bss           0x000000000000126e        0x0 ../lib/freecom.lib(chgdrv.obj)
 .bss           0x000000000000126e        0x0 ../lib/freecom.lib(chgenv.obj)
 .bss           0x000000000000126e        0x0 ../lib/freecom.lib(chgenvc.obj)
 .bss           0x000000000000126e        0x0 ../lib/freecom.lib(chgenvr.obj)
 .bss           0x000000000000126e        0x4 ../lib/freecom.lib(cmdinput.obj)
 .bss           0x0000000000001272        0x2 ../lib/freecom.lib(critrchk.obj)
 .bss           0x0000000000001274        0x2 ../lib/freecom.lib(ctxt.obj)
                0x0000000000001274                ctxt
 .bss           0x0000000000001276        0x0 ../lib/freecom.lib(ctxt_clr.obj)
 .bss           0x0000000000001276        0x0 ../lib/freecom.lib(ctxt_get.obj)
 .bss           0x0000000000001276        0x0 ../lib/freecom.lib(ctxt_inf.obj)
 .bss           0x0000000000001276        0x0 ../lib/freecom.lib(ctxt_mk.obj)
 .bss           0x0000000000001276        0x0 ../lib/freecom.lib(ctxt_mkb.obj)
 .bss           0x0000000000001276        0x0 ../lib/freecom.lib(ctxt_mkn.obj)
 .bss           0x0000000000001276        0x0 ../lib/freecom.lib(ctxt_pop.obj)
 .bss           0x0000000000001276        0x0 ../lib/freecom.lib(ctxt_psh.obj)
 .bss           0x0000000000001276        0x0 ../lib/freecom.lib(ctxt_rnu.obj)
 .bss           0x0000000000001276        0x0 ../lib/freecom.lib(ctxt_set.obj)
 .bss           0x0000000000001276        0x0 ../lib/freecom.lib(ctxt_vw.obj)
 .bss           0x0000000000001276        0x0 ../lib/freecom.lib(curdatel.obj)
 .bss           0x0000000000001276        0x0 ../lib/freecom.lib(curtime.obj)
 .bss           0x0000000000001276        0x0 ../lib/freecom.lib(cwd.obj)
 .bss           0x0000000000001276        0x0 ../lib/freecom.lib(dateget.obj)
 .bss           0x0000000000001276        0x0 ../lib/freecom.lib(dateset.obj)
 .bss           0x0000000000001276        0x0 ../lib/freecom.lib(devopen.obj)
 .bss           0x0000000000001276        0x0 ../lib/freecom.lib(dfn_err.obj)
 .bss           0x0000000000001276        0x0 ../lib/freecom.lib(dispcnt.obj)
 .bss           0x0000000000001276        0x0 ../lib/freecom.lib(drvnum.obj)
 .bss           0x0000000000001276        0x0 ../lib/freecom.lib(exec.obj)
 .bss           0x0000000000001276        0x0 ../lib/freecom.lib(exec1.obj)
 .bss           0x0000000000001276        0x0 ../lib/freecom.lib(farread.obj)
 .bss           0x0000000000001276        0x0 ../lib/freecom.lib(filecomp.obj)
 .bss           0x0000000000001276        0x0 ../lib/freecom.lib(fdattr.obj)
 .bss           0x0000000000001276        0x0 ../lib/freecom.lib(fdsattr.obj)
 .bss           0x0000000000001276        0x0 ../lib/freecom.lib(fillcomp.obj)
 .bss           0x0000000000001276        0x0 ../lib/freecom.lib(find.obj)
 .bss           0x0000000000001276        0x0 ../lib/freecom.lib(freep.obj)
 .bss           0x0000000000001276        0x0 ../lib/freecom.lib(gallstr.obj)
 .bss           0x0000000000001276        0x0 ../lib/freecom.lib(get1mcb.obj)
 .bss           0x0000000000001276        0x0 ../lib/freecom.lib(getenv.obj)
 .bss           0x0000000000001276        0x0 ../lib/freecom.lib(goxy.obj)
 .bss           0x0000000000001276        0x0 ../lib/freecom.lib(grabfcom.obj)
 .bss           0x0000000000001276        0x0 ../lib/freecom.lib(gumblink.obj)
 .bss           0x0000000000001276        0x0 ../lib/freecom.lib(hdlrctxt.obj)
 .bss           0x0000000000001276        0x0 ../lib/freecom.lib(hist_get.obj)
 .bss           0x0000000000001276        0x0 ../lib/freecom.lib(hist_set.obj)
 .bss           0x0000000000001276        0x0 ../lib/freecom.lib(is_empty.obj)
 .bss           0x0000000000001276        0x0 ../lib/freecom.lib(is_fnamc.obj)
 .bss           0x0000000000001276        0x0 ../lib/freecom.lib(is_fnstr.obj)
 .bss           0x0000000000001276        0x0 ../lib/freecom.lib(is_pchr.obj)
 .bss           0x0000000000001276        0x0 ../lib/freecom.lib(isadev.obj)
 .bss           0x0000000000001276        0x0 ../lib/freecom.lib(lastdget.obj)
 .bss           0x0000000000001276        0x0 ../lib/freecom.lib(lastdset.obj)
 .bss           0x0000000000001276        0x0 ../lib/freecom.lib(leadopt.obj)
 .bss           0x0000000000001276       0x80 ../lib/freecom.lib(lfnfuncs.obj)
 .bss           0x00000000000012f6        0x0 ../lib/freecom.lib(ltrimcl.obj)
 .bss           0x00000000000012f6        0x0 ../lib/freecom.lib(match.obj)
 .bss           0x00000000000012f6        0x4 ../lib/freecom.lib(messages.obj)
                0x00000000000012f6                strCnt
                0x00000000000012f8                msgSegm
 .bss           0x00000000000012fa        0x4 ../lib/freecom.lib(mk_rddir.obj)
 .bss           0x00000000000012fe        0x0 ../lib/freecom.lib(msg_dps.obj)
 .bss           0x00000000000012fe        0x0 ../lib/freecom.lib(msg_fstr.obj)
 .bss           0x00000000000012fe        0x0 ../lib/freecom.lib(msg_gpt.obj)
 .bss           0x00000000000012fe        0x0 ../lib/freecom.lib(msg_mkey.obj)
 .bss           0x00000000000012fe        0x0 ../lib/freecom.lib(msg_prmp.obj)
 .bss           0x00000000000012fe        0x0 ../lib/freecom.lib(mux_ae.obj)
 .bss           0x00000000000012fe        0x0 ../lib/freecom.lib(myperror.obj)
 .bss           0x00000000000012fe        0x2 ../lib/freecom.lib(nls.obj)
                0x00000000000012fe                nlsBuf
 .bss           0x0000000000001300        0x0 ../lib/freecom.lib(nls_date.obj)
 .bss           0x0000000000001300        0x0 ../lib/freecom.lib(nls_time.obj)
 .bss           0x0000000000001300        0x0 ../lib/freecom.lib(num_fmt.obj)
 .bss           0x0000000000001300        0x0 ../lib/freecom.lib(onoff.obj)
 .bss           0x0000000000001300        0x0 ../lib/freecom.lib(openf.obj)
 .bss           0x0000000000001300        0x0 ../lib/freecom.lib(optsb.obj)
 .bss           0x0000000000001300        0x0 ../lib/freecom.lib(optsi.obj)
 .bss           0x0000000000001300        0x0 ../lib/freecom.lib(optss.obj)
 .bss           0x0000000000001300        0x0 ../lib/freecom.lib(pr_date.obj)
 .bss           0x0000000000001300        0x0 ../lib/freecom.lib(pr_prmpt.obj)
 .bss           0x0000000000001300        0x0 ../lib/freecom.lib(pr_time.obj)
 .bss           0x0000000000001300        0x6 ../lib/freecom.lib(prf.obj)
                0x0000000000001300                stdin
 .bss           0x0000000000001306        0x0 ../lib/freecom.lib(prprompt.obj)
 .bss           0x0000000000001306        0x0 ../lib/freecom.lib(readcmd.obj)
 .bss           0x0000000000001306        0x0 ../lib/freecom.lib(realnum.obj)
 .bss           0x0000000000001306        0x0 ../lib/freecom.lib(res.obj)
 .bss           0x0000000000001306        0x0 ../lib/freecom.lib(res_r.obj)
 .bss           0x0000000000001306        0x0 ../lib/freecom.lib(res_vald.obj)
 .bss           0x0000000000001306        0x0 ../lib/freecom.lib(resfile.obj)
 .bss           0x0000000000001306        0x0 ../lib/freecom.lib(rmtmpfil.obj)
 .bss           0x0000000000001306        0x0 ../lib/freecom.lib(rtrimcl.obj)
 .bss           0x0000000000001306        0x0 ../lib/freecom.lib(rtrimsp.obj)
 .bss           0x0000000000001306        0x0 ../lib/freecom.lib(salloc.obj)
 .bss           0x0000000000001306        0x0 ../lib/freecom.lib(samefile.obj)
 .bss           0x0000000000001306        0x0 ../lib/freecom.lib(scancmd.obj)
 .bss           0x0000000000001306        0x2 ../lib/freecom.lib(scanopt.obj)
                0x0000000000001306                currCmdHelpScreen
 .bss           0x0000000000001308        0x4 ../lib/freecom.lib(session.obj)
 .bss           0x000000000000130c        0x0 ../lib/freecom.lib(showcmds.obj)
 .bss           0x000000000000130c        0x0 ../lib/freecom.lib(skqwd.obj)
 .bss           0x000000000000130c        0x0 ../lib/freecom.lib(spfnam.obj)
 .bss           0x000000000000130c        0x0 ../lib/freecom.lib(split.obj)
 .bss           0x000000000000130c        0x0 ../lib/freecom.lib(sumblink.obj)
 .bss           0x000000000000130c        0x0 ../lib/freecom.lib(timeget.obj)
 .bss           0x000000000000130c        0x0 ../lib/freecom.lib(timeset.obj)
 .bss           0x000000000000130c        0x0 ../lib/freecom.lib(tmpnam.obj)
 .bss           0x000000000000130c        0x0 ../lib/freecom.lib(trimsp.obj)
 .bss           0x000000000000130c        0x0 ../lib/freecom.lib(truepath.obj)
 .bss           0x000000000000130c        0x0 ../lib/freecom.lib(truncate.obj)
 .bss           0x000000000000130c        0x0 ../lib/freecom.lib(txtlend.obj)
 .bss           0x000000000000130c        0x0 ../lib/freecom.lib(unquote.obj)
 .bss           0x000000000000130c        0x0 ../lib/freecom.lib(vcgetch.obj)
 .bss           0x000000000000130c        0x2 ../lib/freecom.lib(where.obj)
 .bss           0x000000000000130e        0x0 ../lib/freecom.lib(delay.obj)
 .bss           0x000000000000130e        0x0 ../lib/freecom.lib(err2.obj)
 .bss           0x000000000000130e        0x0 ../lib/freecom.lib(err3.obj)
 .bss           0x000000000000130e        0x0 ../lib/freecom.lib(err5.obj)
 .bss           0x000000000000130e        0x0 ../lib/freecom.lib(err6.obj)
 .bss           0x000000000000130e        0x0 ../lib/freecom.lib(err7.obj)
 .bss           0x000000000000130e        0x0 ../lib/freecom.lib(err8.obj)
 .bss           0x000000000000130e        0x0 ../lib/freecom.lib(err10.obj)
 .bss           0x000000000000130e        0x0 ../lib/freecom.lib(err11.obj)
 .bss           0x000000000000130e        0x0 ../lib/freecom.lib(err13.obj)
 .bss           0x000000000000130e        0x0 ../lib/freecom.lib(err14.obj)
 .bss           0x000000000000130e        0x0 ../lib/freecom.lib(err15.obj)
 .bss           0x000000000000130e        0x0 ../lib/freecom.lib(err16.obj)
 .bss           0x000000000000130e        0x0 ../lib/freecom.lib(err17.obj)
 .bss           0x000000000000130e        0x0 ../lib/freecom.lib(err18.obj)
 .bss           0x000000000000130e        0x0 ../lib/freecom.lib(err19.obj)
 .bss           0x000000000000130e        0x0 ../lib/freecom.lib(err20.obj)
 .bss           0x000000000000130e        0x0 ../lib/freecom.lib(err21.obj)
 .bss           0x000000000000130e        0x0 ../lib/freecom.lib(err22.obj)
 .bss           0x000000000000130e        0x0 ../lib/freecom.lib(err23.obj)
 .bss           0x000000000000130e        0x0 ../lib/freecom.lib(err25.obj)
 .bss           0x000000000000130e        0x0 ../lib/freecom.lib(err26.obj)
 .bss           0x000000000000130e        0x0 ../lib/freecom.lib(err27.obj)
 .bss           0x000000000000130e        0x0 ../lib/freecom.lib(err28.obj)
 .bss           0x000000000000130e        0x0 ../lib/freecom.lib(err29.obj)
 .bss           0x000000000000130e        0x0 ../lib/freecom.lib(err30.obj)
 .bss           0x000000000000130e        0x0 ../lib/freecom.lib(err31.obj)
 .bss           0x000000000000130e        0x0 ../lib/freecom.lib(err32.obj)
 .bss           0x000000000000130e        0x0 ../lib/freecom.lib(err33.obj)
 .bss           0x000000000000130e        0x0 ../lib/freecom.lib(err34.obj)
 .bss           0x000000000000130e        0x0 ../lib/freecom.lib(err35.obj)
 .bss           0x000000000000130e        0x0 ../lib/freecom.lib(err36.obj)
 .bss           0x000000000000130e        0x0 ../lib/freecom.lib(err37.obj)
 .bss           0x000000000000130e        0x0 ../lib/freecom.lib(err38.obj)
 .bss           0x000000000000130e        0x0 ../lib/freecom.lib(err39.obj)
 .bss           0x000000000000130e        0x0 ../lib/freecom.lib(err41.obj)
 .bss           0x000000000000130e        0x0 ../lib/freecom.lib(err42.obj)
 .bss           0x000000000000130e        0x0 ../lib/freecom.lib(err45.obj)
 .bss           0x000000000000130e        0x0 ../lib/freecom.lib(err46.obj)
 .bss           0x000000000000130e        0x0 ../lib/freecom.lib(err47.obj)
 .bss           0x000000000000130e        0x0 ../lib/freecom.lib(err50.obj)
 .bss           0x000000000000130e        0x0 ../lib/freecom.lib(err51.obj)
 .bss           0x000000000000130e        0x0 ../lib/freecom.lib(err53.obj)
 .bss           0x000000000000130e        0x0 ../lib/freecom.lib(err54.obj)
 .bss           0x000000000000130e        0x0 ../lib/freecom.lib(err58.obj)
 .bss           0x000000000000130e        0x0 ../lib/freecom.lib(err59.obj)
 .bss           0x000000000000130e        0x0 ../lib/freecom.lib(err60.obj)
 .bss           0x000000000000130e        0x0 ../lib/freecom.lib(err61.obj)
 .bss           0x000000000000130e        0x0 ../lib/freecom.lib(err63.obj)
 .bss           0x000000000000130e        0x0 ../lib/freecom.lib(err64.obj)
 .bss           0x000000000000130e        0x0 ../lib/freecom.lib(err65.obj)
 .bss           0x000000000000130e        0x0 ../lib/freecom.lib(err67.obj)
 .bss           0x000000000000130e        0x0 ../lib/freecom.lib(err68.obj)
 .bss           0x000000000000130e        0x0 ../lib/freecom.lib(err69.obj)
 .bss           0x000000000000130e        0x0 ../lib/freecom.lib(err70.obj)
 .bss           0x000000000000130e        0x0 ../lib/freecom.lib(err71.obj)
 .bss           0x000000000000130e        0x0 ../lib/freecom.lib(err72.obj)
 .bss           0x000000000000130e        0x0 ../lib/freecom.lib(err73.obj)
 .bss           0x000000000000130e        0x0 ../lib/freecom.lib(err74.obj)
 .bss           0x000000000000130e        0x0 ../lib/freecom.lib(err75.obj)
 .bss           0x000000000000130e        0x0 ../lib/freecom.lib(err76.obj)
 .bss           0x000000000000130e        0x0 ../lib/freecom.lib(err77.obj)
 .bss           0x000000000000130e        0x0 ../lib/freecom.lib(err78.obj)
 .bss           0x000000000000130e        0x0 ../lib/freecom.lib(err79.obj)
 .bss           0x000000000000130e        0x0 ../lib/freecom.lib(err80.obj)
 .bss           0x000000000000130e        0x0 ../lib/freecom.lib(err81.obj)
 .bss           0x000000000000130e        0x0 ../lib/freecom.lib(err82.obj)
 .bss           0x000000000000130e        0x0 ../lib/freecom.lib(err83.obj)
 .bss           0x000000000000130e        0x0 ../lib/freecom.lib(err84.obj)
 .bss           0x000000000000130e        0x0 ../lib/freecom.lib(err85.obj)
 .bss           0x000000000000130e        0x0 ../lib/freecom.lib(err86.obj)
 .bss           0x000000000000130e        0x0 ../lib/freecom.lib(err87.obj)
 .bss           0x000000000000130e        0x0 ../lib/freecom.lib(almemblk.obj)
 .bss           0x000000000000130e        0x0 ../lib/freecom.lib(beep_l.obj)
 .bss           0x000000000000130e        0x0 ../lib/freecom.lib(cbs.obj)
 .bss           0x000000000000130e        0x0 ../lib/freecom.lib(comfile.obj)
 .bss           0x000000000000130e        0x0 ../lib/freecom.lib(ctxt_as.obj)
 .bss           0x000000000000130e        0x0 ../lib/freecom.lib(dispexit.obj)
 .bss           0x000000000000130e        0x0 ../lib/freecom.lib(inputdos.obj)
 .bss           0x000000000000130e        0x0 ../lib/freecom.lib(ltrimsp.obj)
 .bss           0x000000000000130e        0x0 ../lib/freecom.lib(mktmpfil.obj)
 .bss           0x000000000000130e        0x0 ../lib/freecom.lib(msg_dflt.obj)
 .bss           0x000000000000130e        0x0 ../lib/freecom.lib(msg_get.obj)
 .bss           0x000000000000130e        0x0 ../lib/freecom.lib(parsenum.obj)
 .bss           0x000000000000130e        0x0 ../strings/strings.lib(str0011.obj)
 .bss           0x000000000000130e        0x0 ../strings/strings.lib(str0018.obj)
 .bss           0x000000000000130e        0x0 ../strings/strings.lib(str003c.obj)
 .bss           0x000000000000130e        0x0 ../strings/strings.lib(str00b1.obj)
 .bss           0x000000000000130e        0x0 ../strings/strings.lib(str00b2.obj)
 .bss           0x000000000000130e        0x0 ../strings/strings.lib(str00f4.obj)
 .bss           0x000000000000130e        0x0 ../strings/strings.lib(str00f5.obj)
 .bss           0x000000000000130e        0x0 ../strings/strings.lib(str00f6.obj)
 .bss           0x000000000000130e        0x0 ../suppl/suppl_s.lib(byte2par.obj)
 .bss           0x000000000000130e       0x42 ../suppl/suppl_s.lib(cntry.obj)
 .bss           0x0000000000001350        0x0 ../suppl/suppl_s.lib(dfnfnam.obj)
 .bss           0x0000000000001350        0x0 ../suppl/suppl_s.lib(dfnfullp.obj)
 .bss           0x0000000000001350        0x0 ../suppl/suppl_s.lib(dfnmerge.obj)
 .bss           0x0000000000001350        0x0 ../suppl/suppl_s.lib(dfnpath.obj)
 .bss           0x0000000000001350        0x0 ../suppl/suppl_s.lib(dfnstat.obj)
 .bss           0x0000000000001350        0x0 ../suppl/suppl_s.lib(dfntruen.obj)
 .bss           0x0000000000001350        0x0 ../suppl/suppl_s.lib(dosalloc.obj)
 .bss           0x0000000000001350        0x0 ../suppl/suppl_s.lib(dosfree.obj)
 .bss           0x0000000000001350        0x0 ../suppl/suppl_s.lib(dossize.obj)
 .bss           0x0000000000001350        0x0 ../suppl/suppl_s.lib(dstrfupr.obj)
 .bss           0x0000000000001350        0x0 ../suppl/suppl_s.lib(dstrtrim.obj)
 .bss           0x0000000000001350        0x0 ../suppl/suppl_s.lib(dstrupr.obj)
 .bss           0x0000000000001350        0x0 ../suppl/suppl_s.lib(enoallc.obj)
 .bss           0x0000000000001350        0x0 ../suppl/suppl_s.lib(enoreal.obj)
 .bss           0x0000000000001350        0x0 ../suppl/suppl_s.lib(enosetos.obj)
 .bss           0x0000000000001350        0x0 ../suppl/suppl_s.lib(env_chg.obj)
 .bss           0x0000000000001350        0x0 ../suppl/suppl_s.lib(env_dvar.obj)
 .bss           0x0000000000001350        0x0 ../suppl/suppl_s.lib(env_find.obj)
 .bss           0x0000000000001350        0x0 ../suppl/suppl_s.lib(env_fora.obj)
 .bss           0x0000000000001350        0x0 ../suppl/suppl_s.lib(env_free.obj)
 .bss           0x0000000000001350        0x0 ../suppl/suppl_s.lib(env_insv.obj)
 .bss           0x0000000000001350        0x0 ../suppl/suppl_s.lib(env_len.obj)
 .bss           0x0000000000001350        0x0 ../suppl/suppl_s.lib(env_mtch.obj)
 .bss           0x0000000000001350        0x0 ../suppl/suppl_s.lib(env_new.obj)
 .bss           0x0000000000001350        0x0 ../suppl/suppl_s.lib(env_nost.obj)
 .bss           0x0000000000001350        0x0 ../suppl/suppl_s.lib(env_ovrw.obj)
 .bss           0x0000000000001350        0x0 ../suppl/suppl_s.lib(env_repl.obj)
 .bss           0x0000000000001350        0x0 ../suppl/suppl_s.lib(env_rlsg.obj)
 .bss           0x0000000000001350        0x0 ../suppl/suppl_s.lib(env_scnt.obj)
 .bss           0x0000000000001350        0x0 ../suppl/suppl_s.lib(env_size.obj)
 .bss           0x0000000000001350        0x0 ../suppl/suppl_s.lib(env_strg.obj)
 .bss           0x0000000000001350        0x0 ../suppl/suppl_s.lib(env_sub.obj)
 .bss           0x0000000000001350        0x0 ../suppl/suppl_s.lib(env_var1.obj)
 .bss           0x0000000000001350        0x2 ../suppl/suppl_s.lib(env_var2.obj)
                0x0000000000001350                suppl_dfltEnvSegm
 .bss           0x0000000000001352        0x0 ../suppl/suppl_s.lib(fstrdup.obj)
 .bss           0x0000000000001352        0x0 ../suppl/suppl_s.lib(mcb_is.obj)
 .bss           0x0000000000001352        0x0 ../suppl/suppl_s.lib(mcb_leng.obj)
 .bss           0x0000000000001352        0x0 ../suppl/suppl_s.lib(mcb_nxt.obj)
 .bss           0x0000000000001352        0x0 ../suppl/suppl_s.lib(mcb_walk.obj)
 .bss           0x0000000000001352        0x0 ../suppl/suppl_s.lib(toupperx.obj)
 .bss           0x0000000000001352        0x0 ../suppl/suppl_s.lib(filefind.obj)
 .bss           0x0000000000001352        0x0 ../suppl/suppl_s.lib(invokedo.obj)
 .bss           0x0000000000001352        0x0 ../suppl/suppl_s.lib(addu.obj)
 .bss           0x0000000000001352        0x0 ../suppl/suppl_s.lib(dfndeli2.obj)
 .bss           0x0000000000001352        0x0 ../suppl/suppl_s.lib(dfndelim.obj)
 .bss           0x0000000000001352        0x0 ../suppl/suppl_s.lib(dfnexpan.obj)
 .bss           0x0000000000001352        0x0 ../suppl/suppl_s.lib(dfnsplit.obj)
 .bss           0x0000000000001352        0x0 ../suppl/suppl_s.lib(dfnsquee.obj)
 .bss           0x0000000000001352        0x0 ../suppl/suppl_s.lib(dmemcmpf.obj)
 .bss           0x0000000000001352        0x0 ../suppl/suppl_s.lib(dstrchar.obj)
 .bss           0x0000000000001352        0x0 ../suppl/suppl_s.lib(dstrleft.obj)
 .bss           0x0000000000001352        0x0 ../suppl/suppl_s.lib(dstrrepl.obj)
 .bss           0x0000000000001352        0x0 ../suppl/suppl_s.lib(enosdup.obj)
 .bss           0x0000000000001352        0x0 ../suppl/suppl_s.lib(env_del.obj)
 .bss           0x0000000000001352        0x0 ../suppl/suppl_s.lib(mcb_1st.obj)
 .bss           0x0000000000001352        0x0 /home/evln/proj/build-ia16.202501/prefix/bin/../lib/gcc/ia16-elf/6.3.0/../../../../ia16-elf/lib/regparmcall/libi86.a(fmemchr.o)
 .bss           0x0000000000001352        0x0 /home/evln/proj/build-ia16.202501/prefix/bin/../lib/gcc/ia16-elf/6.3.0/../../../../ia16-elf/lib/regparmcall/libi86.a(fmemcmp.o)
 .bss           0x0000000000001352        0x0 /home/evln/proj/build-ia16.202501/prefix/bin/../lib/gcc/ia16-elf/6.3.0/../../../../ia16-elf/lib/regparmcall/libi86.a(fmemcpy.o)
 .bss           0x0000000000001352        0x0 /home/evln/proj/build-ia16.202501/prefix/bin/../lib/gcc/ia16-elf/6.3.0/../../../../ia16-elf/lib/regparmcall/libi86.a(fmemmove.o)
 .bss           0x0000000000001352        0x0 /home/evln/proj/build-ia16.202501/prefix/bin/../lib/gcc/ia16-elf/6.3.0/../../../../ia16-elf/lib/regparmcall/libi86.a(fstrcpy.o)
 .bss           0x0000000000001352        0x0 /home/evln/proj/build-ia16.202501/prefix/bin/../lib/gcc/ia16-elf/6.3.0/../../../../ia16-elf/lib/regparmcall/libi86.a(fstrlen.o)
 .bss           0x0000000000001352        0x0 /home/evln/proj/build-ia16.202501/prefix/bin/../lib/gcc/ia16-elf/6.3.0/../../../../ia16-elf/lib/regparmcall/libi86.a(libi86-fmemmove-backward.o)
 .bss           0x0000000000001352        0x0 /home/evln/proj/build-ia16.202501/prefix/bin/../lib/gcc/ia16-elf/6.3.0/../../../../ia16-elf/lib/regparmcall/libi86.a(getdcwd.o)
 .bss           0x0000000000001352        0x0 /home/evln/proj/build-ia16.202501/prefix/bin/../lib/gcc/ia16-elf/6.3.0/../../../../ia16-elf/lib/regparmcall/libi86.a(getdrive.o)
 .bss           0x0000000000001352        0x4 /home/evln/proj/build-ia16.202501/prefix/bin/../lib/gcc/ia16-elf/6.3.0/regparmcall/crtbegin.o
 .bss           0x0000000000001356        0x0 /home/evln/proj/build-ia16.202501/prefix/bin/../lib/gcc/ia16-elf/6.3.0/regparmcall/crtend.o
 *fill*         0x0000000000001356        0x2 
 .bss           0x0000000000001358       0x80 /home/evln/proj/build-ia16.202501/prefix/bin/../lib/gcc/ia16-elf/6.3.0/../../../../ia16-elf/lib/regparmcall/dos-s-c0.o
 .bss           0x00000000000013d8        0x0 /home/evln/proj/build-ia16.202501/prefix/bin/../lib/gcc/ia16-elf/6.3.0/../../../../ia16-elf/lib/regparmcall/libc.a(lib_a-atexit.o)
 .bss           0x00000000000013d8        0x0 /home/evln/proj/build-ia16.202501/prefix/bin/../lib/gcc/ia16-elf/6.3.0/../../../../ia16-elf/lib/regparmcall/libc.a(lib_a-atol.o)
 .bss           0x00000000000013d8        0x0 /home/evln/proj/build-ia16.202501/prefix/bin/../lib/gcc/ia16-elf/6.3.0/../../../../ia16-elf/lib/regparmcall/libc.a(lib_a-ctype_.o)
 .bss           0x00000000000013d8        0x0 /home/evln/proj/build-ia16.202501/prefix/bin/../lib/gcc/ia16-elf/6.3.0/../../../../ia16-elf/lib/regparmcall/libc.a(lib_a-errno.o)
 .bss           0x00000000000013d8        0x0 /home/evln/proj/build-ia16.202501/prefix/bin/../lib/gcc/ia16-elf/6.3.0/../../../../ia16-elf/lib/regparmcall/libc.a(lib_a-exit.o)
 .bss           0x00000000000013d8        0x0 /home/evln/proj/build-ia16.202501/prefix/bin/../lib/gcc/ia16-elf/6.3.0/../../../../ia16-elf/lib/regparmcall/libc.a(lib_a-impure.o)
 .bss           0x00000000000013d8        0x0 /home/evln/proj/build-ia16.202501/prefix/bin/../lib/gcc/ia16-elf/6.3.0/../../../../ia16-elf/lib/regparmcall/libc.a(lib_a-malloc.o)
 .bss           0x00000000000013d8        0x0 /home/evln/proj/build-ia16.202501/prefix/bin/../lib/gcc/ia16-elf/6.3.0/../../../../ia16-elf/lib/regparmcall/libc.a(lib_a-memchr.o)
 .bss           0x00000000000013d8        0x0 /home/evln/proj/build-ia16.202501/prefix/bin/../lib/gcc/ia16-elf/6.3.0/../../../../ia16-elf/lib/regparmcall/libc.a(lib_a-memcmp.o)
 .bss           0x00000000000013d8        0x0 /home/evln/proj/build-ia16.202501/prefix/bin/../lib/gcc/ia16-elf/6.3.0/../../../../ia16-elf/lib/regparmcall/libc.a(lib_a-memcpy.o)
 .bss           0x00000000000013d8        0x0 /home/evln/proj/build-ia16.202501/prefix/bin/../lib/gcc/ia16-elf/6.3.0/../../../../ia16-elf/lib/regparmcall/libc.a(lib_a-memmove.o)
 .bss           0x00000000000013d8        0x0 /home/evln/proj/build-ia16.202501/prefix/bin/../lib/gcc/ia16-elf/6.3.0/../../../../ia16-elf/lib/regparmcall/libc.a(lib_a-memset.o)
 .bss           0x00000000000013d8        0x0 /home/evln/proj/build-ia16.202501/prefix/bin/../lib/gcc/ia16-elf/6.3.0/../../../../ia16-elf/lib/regparmcall/libc.a(lib_a-nano-freer.o)
 .bss           0x00000000000013d8        0x4 /home/evln/proj/build-ia16.202501/prefix/bin/../lib/gcc/ia16-elf/6.3.0/../../../../ia16-elf/lib/regparmcall/libc.a(lib_a-nano-mallocr.o)
                0x00000000000013d8                __malloc_sbrk_start
                0x00000000000013da                __malloc_free_list
 .bss           0x00000000000013dc        0x0 /home/evln/proj/build-ia16.202501/prefix/bin/../lib/gcc/ia16-elf/6.3.0/../../../../ia16-elf/lib/regparmcall/libc.a(lib_a-qsort.o)
 .bss           0x00000000000013dc        0x0 /home/evln/proj/build-ia16.202501/prefix/bin/../lib/gcc/ia16-elf/6.3.0/../../../../ia16-elf/lib/regparmcall/libc.a(lib_a-realloc.o)
 .bss           0x00000000000013dc        0x0 /home/evln/proj/build-ia16.202501/prefix/bin/../lib/gcc/ia16-elf/6.3.0/../../../../ia16-elf/lib/regparmcall/libc.a(lib_a-remove.o)
 .bss           0x00000000000013dc        0x0 /home/evln/proj/build-ia16.202501/prefix/bin/../lib/gcc/ia16-elf/6.3.0/../../../../ia16-elf/lib/regparmcall/libc.a(lib_a-setjmp.o)
 .bss           0x00000000000013dc        0x0 /home/evln/proj/build-ia16.202501/prefix/bin/../lib/gcc/ia16-elf/6.3.0/../../../../ia16-elf/lib/regparmcall/libc.a(lib_a-stpcpy.o)
 .bss           0x00000000000013dc        0x0 /home/evln/proj/build-ia16.202501/prefix/bin/../lib/gcc/ia16-elf/6.3.0/../../../../ia16-elf/lib/regparmcall/libc.a(lib_a-strcasecmp.o)
 .bss           0x00000000000013dc        0x0 /home/evln/proj/build-ia16.202501/prefix/bin/../lib/gcc/ia16-elf/6.3.0/../../../../ia16-elf/lib/regparmcall/libc.a(lib_a-strcat.o)
 .bss           0x00000000000013dc        0x0 /home/evln/proj/build-ia16.202501/prefix/bin/../lib/gcc/ia16-elf/6.3.0/../../../../ia16-elf/lib/regparmcall/libc.a(lib_a-strchr.o)
 .bss           0x00000000000013dc        0x0 /home/evln/proj/build-ia16.202501/prefix/bin/../lib/gcc/ia16-elf/6.3.0/../../../../ia16-elf/lib/regparmcall/libc.a(lib_a-strcmp.o)
 .bss           0x00000000000013dc        0x0 /home/evln/proj/build-ia16.202501/prefix/bin/../lib/gcc/ia16-elf/6.3.0/../../../../ia16-elf/lib/regparmcall/libc.a(lib_a-strcpy.o)
 .bss           0x00000000000013dc        0x0 /home/evln/proj/build-ia16.202501/prefix/bin/../lib/gcc/ia16-elf/6.3.0/../../../../ia16-elf/lib/regparmcall/libc.a(lib_a-strdup.o)
 .bss           0x00000000000013dc        0x0 /home/evln/proj/build-ia16.202501/prefix/bin/../lib/gcc/ia16-elf/6.3.0/../../../../ia16-elf/lib/regparmcall/libc.a(lib_a-strdup_r.o)
 .bss           0x00000000000013dc        0x0 /home/evln/proj/build-ia16.202501/prefix/bin/../lib/gcc/ia16-elf/6.3.0/../../../../ia16-elf/lib/regparmcall/libc.a(lib_a-strlen.o)
 .bss           0x00000000000013dc        0x0 /home/evln/proj/build-ia16.202501/prefix/bin/../lib/gcc/ia16-elf/6.3.0/../../../../ia16-elf/lib/regparmcall/libc.a(lib_a-strlwr.o)
 .bss           0x00000000000013dc        0x0 /home/evln/proj/build-ia16.202501/prefix/bin/../lib/gcc/ia16-elf/6.3.0/../../../../ia16-elf/lib/regparmcall/libc.a(lib_a-strncasecmp.o)
 .bss           0x00000000000013dc        0x0 /home/evln/proj/build-ia16.202501/prefix/bin/../lib/gcc/ia16-elf/6.3.0/../../../../ia16-elf/lib/regparmcall/libc.a(lib_a-strncpy.o)
 .bss           0x00000000000013dc        0x0 /home/evln/proj/build-ia16.202501/prefix/bin/../lib/gcc/ia16-elf/6.3.0/../../../../ia16-elf/lib/regparmcall/libc.a(lib_a-strpbrk.o)
 .bss           0x00000000000013dc        0x0 /home/evln/proj/build-ia16.202501/prefix/bin/../lib/gcc/ia16-elf/6.3.0/../../../../ia16-elf/lib/regparmcall/libc.a(lib_a-strrchr.o)
 .bss           0x00000000000013dc        0x0 /home/evln/proj/build-ia16.202501/prefix/bin/../lib/gcc/ia16-elf/6.3.0/../../../../ia16-elf/lib/regparmcall/libc.a(lib_a-strspn.o)
 .bss           0x00000000000013dc        0x0 /home/evln/proj/build-ia16.202501/prefix/bin/../lib/gcc/ia16-elf/6.3.0/../../../../ia16-elf/lib/regparmcall/libc.a(lib_a-strtok.o)
 .bss           0x00000000000013dc        0x0 /home/evln/proj/build-ia16.202501/prefix/bin/../lib/gcc/ia16-elf/6.3.0/../../../../ia16-elf/lib/regparmcall/libc.a(lib_a-strtok_r.o)
 .bss           0x00000000000013dc        0x0 /home/evln/proj/build-ia16.202501/prefix/bin/../lib/gcc/ia16-elf/6.3.0/../../../../ia16-elf/lib/regparmcall/libc.a(lib_a-strtol.o)
 .bss           0x00000000000013dc        0x0 /home/evln/proj/build-ia16.202501/prefix/bin/../lib/gcc/ia16-elf/6.3.0/../../../../ia16-elf/lib/regparmcall/libc.a(lib_a-sysisatty.o)
 .bss           0x00000000000013dc        0x0 /home/evln/proj/build-ia16.202501/prefix/bin/../lib/gcc/ia16-elf/6.3.0/../../../../ia16-elf/lib/regparmcall/libc.a(lib_a-syslseek.o)
 .bss           0x00000000000013dc        0x0 /home/evln/proj/build-ia16.202501/prefix/bin/../lib/gcc/ia16-elf/6.3.0/../../../../ia16-elf/lib/regparmcall/libc.a(lib_a-sysunlink.o)
 .bss           0x00000000000013dc        0x0 /home/evln/proj/build-ia16.202501/prefix/bin/../lib/gcc/ia16-elf/6.3.0/../../../../ia16-elf/lib/regparmcall/libc.a(lib_a-syswrite.o)
 .bss           0x00000000000013dc        0x0 /home/evln/proj/build-ia16.202501/prefix/bin/../lib/gcc/ia16-elf/6.3.0/../../../../ia16-elf/lib/regparmcall/libc.a(lib_a-toupper.o)
 .bss           0x00000000000013dc       0x46 /home/evln/proj/build-ia16.202501/prefix/bin/../lib/gcc/ia16-elf/6.3.0/../../../../ia16-elf/lib/regparmcall/libc.a(lib_a-__atexit.o)
 .bss           0x0000000000001422        0x2 /home/evln/proj/build-ia16.202501/prefix/bin/../lib/gcc/ia16-elf/6.3.0/../../../../ia16-elf/lib/regparmcall/libc.a(lib_a-__call_atexit.o)
                0x0000000000001422                _global_atexit
 .bss           0x0000000000001424        0x0 /home/evln/proj/build-ia16.202501/prefix/bin/../lib/gcc/ia16-elf/6.3.0/../../../../ia16-elf/lib/regparmcall/libc.a(lib_a-nano-reallocr.o)
 .bss           0x0000000000001424        0x0 /home/evln/proj/build-ia16.202501/prefix/bin/../lib/gcc/ia16-elf/6.3.0/../../../../ia16-elf/lib/regparmcall/libc.a(lib_a-nano-msizer.o)
 .bss           0x0000000000001424        0x0 /home/evln/proj/build-ia16.202501/prefix/bin/../lib/gcc/ia16-elf/6.3.0/regparmcall/libgcc.a(udivsi3.o)
 .bss           0x0000000000001424        0x0 /home/evln/proj/build-ia16.202501/prefix/bin/../lib/gcc/ia16-elf/6.3.0/regparmcall/libgcc.a(umodsi3.o)
 .bss           0x0000000000001424        0x0 /home/evln/proj/build-ia16.202501/prefix/bin/../lib/gcc/ia16-elf/6.3.0/regparmcall/libgcc.a(ia16-ldivmodu.o)
 .bss           0x0000000000001424        0x0 /home/evln/proj/build-ia16.202501/prefix/bin/../lib/gcc/ia16-elf/6.3.0/../../../../ia16-elf/lib/regparmcall/libdos-s.a(dos-isattyr.o)
 .bss           0x0000000000001424        0x0 /home/evln/proj/build-ia16.202501/prefix/bin/../lib/gcc/ia16-elf/6.3.0/../../../../ia16-elf/lib/regparmcall/libdos-s.a(dos-lseekr.o)
 .bss           0x0000000000001424        0x0 /home/evln/proj/build-ia16.202501/prefix/bin/../lib/gcc/ia16-elf/6.3.0/../../../../ia16-elf/lib/regparmcall/libdos-s.a(dos-sbrkr.o)
 .bss           0x0000000000001424        0x0 /home/evln/proj/build-ia16.202501/prefix/bin/../lib/gcc/ia16-elf/6.3.0/../../../../ia16-elf/lib/regparmcall/libdos-s.a(dos-unlinkr.o)
 .bss           0x0000000000001424        0x0 /home/evln/proj/build-ia16.202501/prefix/bin/../lib/gcc/ia16-elf/6.3.0/../../../../ia16-elf/lib/regparmcall/libdos-s.a(dos-writer.o)
 .bss           0x0000000000001424       0x80 /home/evln/proj/build-ia16.202501/prefix/bin/../lib/gcc/ia16-elf/6.3.0/../../../../ia16-elf/lib/regparmcall/libdos-s.a(dos-msmmabort.o)
 .bss           0x00000000000014a4        0x0 /home/evln/proj/build-ia16.202501/prefix/bin/../lib/gcc/ia16-elf/6.3.0/../../../../ia16-elf/lib/regparmcall/libdos-s.a(dos-heaplen.o)
 .bss           0x00000000000014a4        0x0 /home/evln/proj/build-ia16.202501/prefix/bin/../lib/gcc/ia16-elf/6.3.0/../../../../ia16-elf/lib/regparmcall/libdos-s.a(dos-near-data-segment.o)
 .bss           0x00000000000014a4        0x0 /home/evln/proj/build-ia16.202501/prefix/bin/../lib/gcc/ia16-elf/6.3.0/../../../../ia16-elf/lib/regparmcall/libc.a(lib_a-abort.o)
 *(.bss.*)
 *(COMMON)
 COMMON         0x00000000000014a4       0x14 command.obj
                0x00000000000014a4                jmp_beginning
 COMMON         0x00000000000014b8        0x2 init.obj
                0x00000000000014b8                ComPath
 COMMON         0x00000000000014ba        0x2 ../lib/freecom.lib(dispexit.obj)
                0x00000000000014ba                exitReason
                0x00000000000014bc                __ebss = .
                0x00000000000014c0                __heap_end_minimum = ALIGN (0x8)
                0x0000000000000001                ASSERT ((. <= 0xfd00), Error: too large for a small-model .exe file.)
                0x0000000000000001                ASSERT (((LOADADDR (.bss) + SIZEOF (.bss)) <= 0xa0000), Error: too large for a .exe file.)
                0x0000000000000001                ASSERT ((ABSOLUTE (DEFINED (main!)?main!:0x0) == 0x0), Error: using non-segelf ld script with segelf program.)
                0x0000000000000001                ASSERT ((ABSOLUTE (DEFINED (environ!)?environ!:0x0) == 0x0), Error: using non-segelf ld script with segelf library.)
                0x0000000000000f84                __ldata = (__edata - __sdata)
                0x000000000000050c                __lbss0 = (__ebss - __sbss)
                0x000000000000050d                __lbss1 = (__lbss0 + 0x1)
                0x0000000000000286                __lbss = (__lbss1 / 0x2)
                0x0000000000001e25                __msdos_initial_alloc_paras = (((((LOADADDR (.data) / 0x10) - (LOADADDR (.text) / 0x10)) + 0x10) + 0x1000) - (ADDR (.data) / 0x10))

.tail
 *(.tail)
 *(SORT_BY_NAME(.tail.*))
 *(.zip)
 *(SORT_BY_NAME(.zip.*))
 *(.ov)
 *(SORT_BY_NAME(.ov.*))
 *(.ov0)
 *(SORT_BY_NAME(.ov0.*))
 *(.ov1)
 *(SORT_BY_NAME(.ov1.*))
 *(.ov2)
 *(SORT_BY_NAME(.ov2.*))
 *(.ov3)
 *(SORT_BY_NAME(.ov3.*))
 *(.ov4)
 *(SORT_BY_NAME(.ov4.*))
 *(.ov5)
 *(SORT_BY_NAME(.ov5.*))
 *(.ov6)
 *(SORT_BY_NAME(.ov6.*))
 *(.ov7)
 *(SORT_BY_NAME(.ov7.*))

/DISCARD/
 *(.*)
OUTPUT(command.exe binary)
